S32508008000888700206981000863D3000891C7000861D300089D970008F91B010800000000FE
S3250800802000000000000000000000000069E700087DB200080000000051DB0008FDEE00087C
S32508008040E51C010883810008838100088381000883810008838100088381000883810008B4
S32508008060838100088381000883810008838100088381000883810008838100088381000892
S3250800808083810008838100088381000829980008A197000883810008C1970008838100082D
S325080080A0838100088381000883810008838100088381000831F00008838100088381000835
S325080080C08381000883810008838100088381000883810008110D01088D0D01085D0E010818
S325080080E083810008838100088381000800000000000000000000000000000000000000004E
S325080081000000000000000000838100088381000845FF000839000108838100088381000893
S3250800812083810008838100088381000883810008838100088381000883810008F19A00084A
S32508008140838100081D9A0008599A000883810008DFF810D000F07AFC00480047A94A010897
S32508008160AFF30080888700200648804706480047FEE7FEE7FEE7FEE7FEE7FEE7FEE7FEE7CE
S32508008180FEE7FEE791EF000851810008202A04DB203A00FA02F1002070479140C2F12003B7
S325080081A020FA03F3194390407047202A04DB203A21FA02F00021704721FA02F3D040C2F183
S325080081C02002914008431946704740EA01039B0703D009E008C9121F08C0042AFAD203E00A
S325080081E011F8013B00F8013B521EF9D27047D2B201E000F8012B491EFBD270470022F6E793
S3250800820010B513460A4604461946FFF7F0FF204610BD30B505462A460B4612F8010B13F80F
S32508008220014B08B1A042F8D01CB1002802D06D1CF1E7284630BD421C10F8011B0029FBD187
S32508008240801A704730B504460020034600E05B1C934203D2E05CCD5C401BF8D030BDF0B40D
S3250800826080EA0102D40F4200B2EB410F02D20246084611464A0042D0C30DDDB2C1F3C75228
S32508008280AD1A202D35DAC1F3160141F4000204B15242C5F1200602FA06F12A411044B3EB36
S325080082A0D05F23D0C4B1012DA0EBC35009DCF0BC4FF0004202EAC352DBB200F5000000F0C8
S325080082C009BB400000F1807000EBC350A0F1807040EAD170490009E0490841EAC071A0EB57
S325080082E0C35000F50000400800EBC350F0BC00F0E8BA6142012202EB4101001BF6E7F0BC4B
S32508008300704781F00041AAE780F00040A7E780EA010210B502F00043400022D04A001FD045
S32508008320010E01EB1261C0F35600C2F3560240F4000042F40002A0FB022000047F391404AE
S3250800834000D0401C50EA124001D44000491EC2B20C0604EBD010401C4008802A02D003E083
S32508008360002010BD20F00100002900DA0020184310BD30B480EA010202F0004530F00042BC
S3250800838021F0004013D090B1C30DD40DC2F31601C0F31600E41A41F4000140F400027D34F9
S325080083A0914201D3641C00E04900002C02DA30BC002070474FF400000023914201D3891AE4
S325080083C0034340084FEA4101F7D151B1914202D14FF0004105E002D24FF0010101E06FF05C
S325080083E0010103EBC450284430BC00F06ABA2DE9FE4F804681EA0300C00F0C46009021F0A6
S32508008400004123F00045B8EB0200A94105D24046214690461C460B46024623F000401043EB
S3250800842047D0270DC7F30A00C3F30A510290401A019040286BDAC3F3130040F4801B0098B4
S32508008440924620B10023D2EB030A63EB0B0B01985946C0F140025046FFF798FE06460D4628
S3250800846050465946019A00F01AFA10EB08006141002487EA115284EAE7731A4340D0009AAE
S3250800848062B3019A012A4FEA075215DC001B61EB02014FF0004202EA0752CDE90042001C2C
S325080084A041F5801132462B4600F051FA03B0BDE8F08F40462146F9E7001B61EB0201001C99
S325080084C041F5801300185B412018A2F5001747EB030140EAD570B6196D4111E06D084FEA6A
S325080084E0360645EAC0754FEA0752001B61EB0201001C41F5801149084FEA3000001951418A
S3250800850032462B4603B0BDE8F04F00F011BA0098012240000023D0EB020263EBE0730098FC
S3250800852021464FEAE074B8EB000061EB0401E9E783F000435BE781F0004158E72DE9FE4F29
S3250800854081EA030404F0004421F0004100944FF0000B23F0004350EA01045ED052EA03042D
S325080085605BD0C3F30A54C1F30A552C44A4F2F3340194A0FB0254C1F3130141F48011C3F3A4
S32508008580130343F4801301FB024400FB034E840A970A44EA815447EA8357A4FB076802957D
S325080085A08D0A05FB07854FEA932C04FB0C542705029D4FEA065847EA1637B5EB08056EEB4D
S325080085C0070C870E920E47EA811742EA8312A7FB0201B6EB0B0164EB00042B0D43EA0C3372
S325080085E05E1844EB1C50DA465146E7FB0201C5F313044FEA0B3343EA14534FEA0432019CDA
S3250800860043EA0603A4F10C040294009CCDE900B400F09DF903B0BDE8F08F00200146F9E731
S325080086202DE9F04D81EA030404F0004B21F0004514464FF0000A23F0004150EA050220D0AA
S3250800864054EA01021DD0C5F30A570246C5F31303C1F31300C1F30A5640F4801543F4801341
S32508008660A7EB0608101BD64608F2FD3873EB050002D308F1010801E092185B41B8F1000FBD
S3250800868003DA00200146BDE8F08D00204FF48011064684460EE0171B73EB050705D3121BCD
S325080086A063EB050306434CEA010C49084FEA300092185B4150EA0107EDD152EA030012D0A9
S325080086C082EA040083EA0501084305D0101BAB4106D20122002306E000224FF0004302E0E8
S325080086E06FF0010253101AEB06004CEB085110EB0A0041EB0B01BDE8F04D00F019B970B506
S3250800870021F0004303430CD0C1F30A550024D5EB040564EB0403D617AD1AB34102DB0020DA
S32508008720014670BD201841EB025170BDC10F80EAE0700844CA079623002100F0CBB8962326
S325080087400022114600F0C6B80EB540F2334102910021CDE900110A460B4600F0F8F803B00C
S3250800876000BD20F00040C10DC0F3160040F400007F2901DA00207047962903DCC1F19601D2
S32508008780C840704796398840704700F0004230F000400AD0C10D01F56071C0F3160042EAC8
S325080087A00151C20840071143704700200146704701F0004330B421F0004150EA010206D0A2
S325080087C00A0DA2F56072C1F31301002A02DC30BC00207047440F44EAC104C100E01830BC8D
S325080087E000EBC25000F06DB8002801DBC0F10040002901DBC1F1004181427047002801DBEE
S32508008800C0F10040002901DBC1F100418842704730B50B46014600202022012409E021FAD8
S3250800882002F59D4205D303FA02F5491B04FA02F52844151EA2F10102F1DC30BD2DE9F05FDB
S325080088400546002092469B4688460646814640241BE02846414647462246FFF7A6FC53468B
S325080088605A46C01A914110D3114618462246FFF78DFC2D1A67EB01084F462246012000213E
S32508008880FFF784FC17EB00094E41201EA4F10104DFDC484631462A464346BDE8F09F202AAB
S325080088A006DBCB17203A41FA02F043EAE07306E041FA02F3D040C2F120029140084319466A
S325080088C070470029A8BF7047401C490008BF20F00100704710B4B0FA80FC00FA0CF050EA3E
S325080088E0010404BF10BC704749B1CCF1200421FA04F411FA0CF118BF012121430843A3EBF3
S325080089000C01CB1D4FEA00614FEA102042BF002010BC704700EBC35010440029A4BF10BC03
S325080089207047401C490008BF20F0010010BC704710B5141E73F1000408DA401C41F10001A2
S3250800894092185B411A4301D120F0010010BD2DE9F04D92469B4611B1B1FA81F202E0B0FA3E
S3250800896080F220329046FFF711FC04460F4640EA0A0041EA0B0153465A46084313D0114684
S3250800898053EA010019D0C8F140025046FFF70DFC05460E46504659464246FFF7F7FB084383
S325080089A005D0012004E020463946BDE8F08D0020054346EAE0762C4337430A986305E40AF9
S325080089C0A0EB08000022FD0A44EA47540A3002D500200146E9E7010510196941DDE90845D0
S325080089E000196941BDE8F04DA2E7C1F30A52C1F3130140F2FF3341F480119A4202DA002061
S32508008A000146704740F233439A42A2F2334202DC5242FFF7CABBFFF7B9BB000030B5041E5F
S32508008A2071F1000404DB4FF00044404264EB0101141E73F1000405DB1C464FF0004352429B
S32508008A4063EB0403994208BF904230BD064C074D06E0E06840F0010394E8070098471034A4
S32508008A60AC42F6D3FFF778FB088001082880010870B58C1810F8015B15F0070301D110F870
S32508008A80013B2A1106D110F8012B03E010F8016B01F8016B5B1EF9D12B0705D40023521EA9
S32508008AA00DD401F8013BFAE710F8013BCB1A921C03E013F8015B01F8015B521EF9D5A1421A
S32508008AC0D8D3002070BD0078704700002DE9F0411E4804F08DFB1E4D0126002769791D4C34
S32508008AE0884205D0207818B9042002F06FFE88B1164804F07DFB6979884202D1207800B112
S32508008B002770154804F074FBA97988420BD0607828B108E02670042009F014FEF1E70320D0
S32508008B2002F054FE58B10C4804F062FBA979884203D16078002800D06770BDE8F0816670E2
S32508008B40BDE8F041052009F0FDBD0000A00900209023002040070020A80900200029816873
S32508008B6002D041F0010101E021F00101816070470029816802D041F4807101E021F4807165
S32508008B8081607047014600208968490700D501207047014600208968090700D501207047C5
S32508008BA010B542680E4B0C791A400B6842EA04221343436083680B4A1340D1E9024222434C
S32508008BC04C7943EA44031A438260C26A097C22F47002491EC9B242EA0151C16210BD000086
S32508008BE0FFFEF0FFFDF7F1FF70B5072409290AD9C568A1F10A0606EB4606B440A543B34057
S32508008C001D43C56007E0056901EB4106B440A543B3401D4305611F23072A09D2446B521E37
S32508008C2002EB820293409C4391400C43446370BD0D2A09D2046BD21F02EB820293409C437A
S32508008C4091400C43046370BDC46A0D3A02EB820293409C4391400C43C46270BD816841F02D
S32508008C600801816070470029816802D041F4A00101E021F4A00181607047816841F004013D
S32508008C808160704738B590228DF8002001228DF801208DF802108DF803000B480024C0F8D3
S32508008CA0982103F03FFE6D46285D03F079FE0A20401E0004000CFBD1641CE4B2042CF3D3AB
S32508008CC003F052FE38BD00000080214208B50121082005F0A3FBC020ADF8000003208DF8A4
S32508008CE0020010208DF803006946054802F052FF04480121C0F89C11C0F8981108BD000074
S32508008D00000C01400080214210B5084C207B18B100206074012010BD607C20B9012060740C
S32508008D2005F062FCA060002010BD00003024002070B5012192B0084605F04CFB012140F20A
S32508008D40112005F06BFB4FF4004005F039FB3920ADF8400000248DF8434010A9334802F03D
S32508008D6019FF4FF460200B94CDE90D0401208DF831002F4E04258DF830008DF83C500BA9AD
S32508008D803046FFF70DFF052301220A213046FFF72BFF052302220D213046FFF725FF05230F
S32508008DA003220E213046FFF71FFF052304220F213046FFF719FF1E4869464C30009080150F
S32508008DC006901C480190280207908020CDE9044020200890CDE90245C001CDE90904164CE4
S32508008DE0204602F0A2F90121204602F093F901213046FFF7BDFE01213046FFF7AFFE304672
S32508008E00FFF72CFF34462046FFF7C3FE0028FAD12046FFF732FF2046FFF7B4FE0028FAD10B
S32508008E2001212046FFF71FFF12B070BD0010014000240140500000200800024070B50446BA
S32508008E400D460C200CF070F82988018069684160216809B1626806E0012121726060806035
S32508008E60206070BD19468B689342FBD188602168816070BD10B50D4C0D49207851F8200050
S32508008E8080470B492078203151F8200080472178074A01EB4101C03A02EBC10151F8201056
S32508008EA0002901D08847207010BD0000682300205806002000F00F01000900EB800001EBF5
S32508008EC04000C0B2704710B5012005F0B3FABDE81040002005F0AEBA00B50D48A1B041F293
S32508008EE00401A0F805102021418000F5C371087C401C087407A008F051FF20AA6946044877
S32508008F0002F030F90021084806F02AFF21B000BD2A1F002073656E6420436861726765206D
S32508008F20646174610A0D0000E001002010B50C4C94F86C00642809D0206F0169884738B146
S32508008F40206F8169884728B1012010BD062002E01C2000E0212002F047FC002010BD00006D
S32508008F60CC06002000B50B48A1B041F20901A0F805101221418000F5C371087C401C087435
S32508008F8005A008F00BFF20AA6946024802F0EAF821B000BD2A1F002053656E6420436861D8
S32508008FA07267696E6744617461200A0D0000000000B5A1B00020ADF880000F4841F2030102
S32508008FC0A0F805100D49097881720421418000F5C370017C491C017409A008F0DFFE20AA5F
S32508008FE06946054802F0BEF804480021503006F0B7FE21B000BD00002A1F00208C01002083
S3250800900073656E642073746174652064617461200A0D000010B5242002F0C8FB002104483B
S3250800902006F09EFEBDE81040002001F029BE00009C23002010B5124CA2B041F22100A4F85F
S325080090400500A4F246404069E071010A2172010C6172000EA072042004F5C3716080087C94
S32508009060401C087407A008F099FE20AA6946204602F078F80421E01D0AF0D4FE22B010BD06
S325080090802A1F00200A0D7368656E676A6979696E676461200A0D000010B50F4CA2B04FF4F2
S325080090A08150A4F805005520E071AA202072022004F5C3716080087C401C087407A008F0E4
S325080090C06DFE20AA6946204602F04CF80221E01D0AF0A8FE22B010BD2A1F00204F54412036
S325080090E041434B200A0D000000B51848A1B041F20801A0F8051016A100F2BE220B6816A15A
S32508009100D36209681163A0F1420242F8493F516000F2EA229168C1730B0A03740B0C43745A
S32508009120090E8174117BC1740D21418000F5C371087C401C08740AA008F030FE20AA694697
S32508009140024802F00FF821B000BD00002A1F00205332303100000000574C494E4700000060
S3250800916073656E6420626D732076657273696F6E0A0D00000549088A401C80B20882C828B0
S3250800918001D3AA2070470020704700006823002010B501214FF0C05005F028F9BDE81040A9
S325080091A0012004F0B5B9000070B5094D130AD2B205F5807606E000BF10F8014B5C402B5DF5
S325080091C05340325D491E89B2F6D242EA032070BDAC74010870B5094DFF22134605F580766B
S325080091E006E000BF10F8014B54402A5D5A40335D491E89B2F6D243EA022070BDAC74010814
S32508009200022101A005F0C6B9415400000A2101A005F0C0B941542B53544154453D3F00007C
S3250800922010B588B0044620216846FEF7E7FF20216846FEF7E3FF224606A1684608F0BEFDD9
S325080092406846FEF7F8FF0146684605F0A3F908B010BD000041542B4E414D453D25730000A5
S32508009260092101A005F096B941542B4E414D453D3F0000000D2101A005F08CB941542B5556
S325080092804152545F4346473D3F0000000B2101A005F080B941542B564552494F4E3D3F0024
S325080092A070B5214D687801283DD1204C2078062830D2DFE800F003130B2F1A2307221CA198
S325080092C01D48FEF7BFFF28BB022015E00A221BA11948FEF7B7FFE8B901200DE01A4916480A
S325080092E0FEF797FFB0B1042006E00B2217A11248FEF7A8FF70B9052020700BE00E486060B0
S32508009300E88920810C480188A1F5B442A53A01D10BF05CFE00206870E881BDE87040802167
S325080093200548FEF76BBF70BD8C010020B020002041542B4F4B0D0A00D41B002041542B4F5A
S325080093404B0D0A30333033003815002041542B4F4B0D0A30310D0A0010B5114C2078062899
S3250800936019D2DFE800F0030B07180F19BDE81040FFF746BFBDE8104000F0F0B9BDE8104075
S3250800938000F0B0B900F0D6F9064890F8760008B1012800D1A07010BDBDE8104000F004B82A
S325080093A0B0200020281500202DE9F041424E4348002596F8A810037C01290DD0404C4FF430
S325080093C07A7132462186012792F87620142B0CD942B1012A08D008E00A2B01D386F8A850AC
S325080093E0BDE8F081857000E087708378052BF7D2DFE803F004080B035500F1E7BDE8F041B2
S3250800940000F040B900F0FEF8E8E72D48403006F0A7FC0128E4D1E08D401C80B2E0850928B3
S3250800942000D9E58526480021403006F099FCE08DA8B1012817D0022819D00328D0D0042871
S3250800944019D005281BD006281DD007281FD0082821D00928C4D1BDE8F04109F081BABDE82E
S32508009460F04100F0A3B8BDE8F041FFF735BDBDE8F041FFF79DBDBDE8F04100F023B8BDE838
S32508009480F041FFF731BEBDE8F041FFF76BBDBDE8F04109F099BABDE8F04109F037BA417C15
S325080094A04B1C437414299BD905701AB1012A97D1877095E7857093E728150020B0200020CD
S325080094C08C01002030B5A1B000202F4CADF8800041F20700A4F805002C4842F21075818BC7
S325080094E0C28BE17101FB02F393FBF5F3090A21726272110AA172E37290F82910217390F87E
S32508009500281061732021A1735F21E173C27E2274C18C6174090AA174E274B0F8091021753B
S32508009520090A6175B0F80B10A175090AE175B0F801102176090A6176B0F80510A176090AD1
S32508009540E176C1792177418A6177090AA17790F82A10E17790F82B0084F820000CA008F0F9
S325080095601DFC1A20608020AA6946204601F0FAFD04F5C370017C491C01740021094806F0F8
S32508009580EFFB21B030BD00002A1F0020800C002073656E64204443444320646174610A0D57
S325080095A000000000E401002004F0E8BF00B5A1B00020ADF880000AA008F0F0FB0E493A2074
S325080095C020AA488069460C4801F0CCFD0B48017C491C017400210A4806F0C2FB21B000BDD0
S325080095E073656E64206865617274626561742064617461200A0D00002A1F0020B020002099
S32508009600D801002010B592B00020ADF8400040F6B831134806F0A4FB01281FD1114C41F27F
S325080096200100A4F8050010A008F0B8FB1349A4F14200CA6E40F8492F096F416010490A6820
S3250800964082604968C1601020608010AA6946204601F088FD0021024806F082FB12B010BD86
S32508009660D40100202A1F002073656E64204C6F67696E20646174610D0A000000281500208D
S32508009680BC73010810B592B00024ADF8404041F288310C4806F064FB012810D101030A483F
S325080096A0A0F80510448009A008F078FB10AA6946054801F057FD0021024806F051FB12B0AD
S325080096C010BD0000D00100202A1F002053656E6420526567697374657265642064617461E3
S325080096E00A0D000010B54FF47A71104806F038FB012819D10D4C383CA07A20B1012804D009
S32508009700022807D00AE0012007E00948FFF788FD022002E0FFF7A4FD0020A072BDE81040BA
S325080097200021024806F01CBB10BD0000C40100203815002010B540F6B831074806F010FB90
S32508009740012807D1FFF762FDBDE810400021024806F006BB10BD0000C801002010B54FF4D0
S325080097607A710D4806F0FCFA012814D10A4C343C607A10B1012804D007E0FFF787FD0120C1
S3250800978002E0FFF777FD00206072BDE810400021014806F0E5BA10BDC0010020FEE70000F6
S325080097A000B585B06A460021044800F089FD6946002009F02FFF05B000BD00000064004012
S325080097C070B5174C4FF400752946204600F0B0FB01280CD11349204600F08FFB012802D18D
S325080097E0002009F0B7FF2946204600F0D1F94FF480652946204600F09BFB01280FD109491F
S325080098002046891C00F079FB012802D1002009F0B9FF29462046BDE8704000F0B9B970BD45
S32508009820006400400200F01010B51A4C0021204600F004FE022806D0012824D00022002170
S32508009840084609F013FF0121204600F0F7FD022806D0012819D000220121002009F006FFC1
S325080098600221204600F0EAFD022806D001280ED000220221002009F0F9FE2046BDE81040C3
S32508009880012100F085B90122D9E70122E4E70122EFE700000064004070B58AB004F065FF45
S325080098A00121092004F0BAFD0121480604F09EFD0121880604F09AFD504E0021304600F045
S325080098C0B9FC7014ADF8200003208DF8220018204B4C8DF8230008A9204602F05BF9A0142A
S325080098E0ADF8200048208DF8230008A9204602F051F9002401258DF80A408DF80B50082011
S325080099008DF808008DF80C408DF806408DF80D408DF8075006208DF80E40ADF804008DF83B
S325080099200F508DF8095001A9304600F05DFB3548407BB0B10E208DF81A008DF81B408DF8A9
S325080099401C50ADF81040ADF81440ADF81240ADF81640ADF818508DF81D5004A800F0AAF96F
S3250800996003E02949002000F0B7FA01221021304600F032FB41208DF800008DF801508DF89B
S3250800998002408DF80350684603F0FCFC01221146304600F021FB01225102304600F01CFB17
S325080099A001229102304600F017FB0122D103304600F012FB0121304600F03CFC3F208DF85D
S325080099C000008DF801508DF802408DF80350684603F0D8FC42208DF800008DF801508DF84D
S325080099E002408DF80350684603F0CCFC04F0BFFE06A008F0D3F90AB0002070BD006800400C
S32508009A00000C0140302400201005002063616E2032206F70656E210A0000000000B50B49B8
S32508009A2085B0012088730A4804F0DEFE6A460121084800F045FC9DF80900002803D1694609
S32508009A40012009F0E7FD05B000BD000030240020BC3400200068004070B5214C4FF4007512
S32508009A602946204600F064FA012810D11D4E2046314600F042FA012805D109F06BFE31465F
S32508009A80204600F06DF82946204600F081F84FF480652946204600F04BFA01281ED1114E16
S32508009AA02046B61C314600F028FA0F4A012807D00020107429462046BDE8704000F068B8A0
S32508009AC0107C401C1074094804F08EFE012009F059FE3146204600F043F8EBE770BD0000C3
S32508009AE0006800400200F01030240020C434002010B51A4C0021204600F0A0FC022806D0E4
S32508009B00012824D000220021012009F0AFFD0121204600F093FC022806D0012819D00022D6
S32508009B200121084609F0A2FD0221204600F086FC022806D001280ED000220221012009F0AE
S32508009B4095FD2046BDE81040012100F021B80122D9E70122E4E70122EFE7000000680040AD
S32508009B600A4A914202D1002181617047C1F313028B0101D5C26070474B0101D502617047E3
S32508009B80090101D582607047426070477000F03030B5082310240422B1F5007F1DD010DCED
S32508009BA0202929D007DC012921D0042922D0082900D1C46030BD402920D0B1F5807FF9D15D
S32508009BC00BE00025B1F5004F06D008DCB1F5806F03D0B1F5006FEDD18561426030BDB1F562
S32508009BE0803F0DD0B1F5003FF8D1446030BD0549816030BDC36030BD036130BD046130BDAD
S32508009C00436030BD01010100094910B588424FF0010101D14C0601E04FF08064204604F0FF
S32508009C20F1FB2046BDE81040002104F0EBBB00000064004030B41446002819D0002202728B
S32508009C4002604260B1F5006F03D304250572416001E00272016043B13CB14272837221461F
S32508009C6030BC1A460B30FEF7B0BA82720221417230BC704730B41446002819D0002202729E
S32508009C8002604260B1F5006F03D304250572416001E00272016043B13CB1427283722146DF
S32508009CA030BC1A460B30FEF790BA82720221417230BC7047F0B5827A012191402E4A1368DC
S32508009CC043F0010313602C4B1C331C688C431C60294D067B294C0C35A6B92E688E432E6036
S32508009CE04688C78846EA0746877A04EBC707C7F840660688878846EA0746877A04EBC707C1
S32508009D00C7F84466067B012E12D12E680E432E60867A056804EBC6064FEA3545C6F8405695
S32508009D20867A456804EBC6044FEA3545C4F84456114CC57A241D002D256806D00D43256064
S32508009D400D4C0589143415B104E08D43F7E725688D4325600589012D02D125680D4325609B
S32508009D60407B012802D1186808431860106820F001001060F0BD00000066004000600040EF
S32508009D802DE9FF41064601250F460024284600F0DFFA01208DF80A508DF80B008DF80C001C
S32508009DA0ADF808008DF80D0000254FF0040831E004EBD47020F00100201A401C012802D000
S32508009DC002281BD10DE056F8351008EBC101090CADF8001036F8351008EBC100ADF8020092
S32508009DE00CE056F8351008EBC101090CADF8041036F8351008EBC100ADF80600641CE0071A
S32508009E0007D16846FFF756FF9DF80A00401C8DF80A006D1CBD42CBDBE00702D06846FFF74E
S32508009E2049FFBDE8FF812DE9FF41804601250E460024284600F08CFA01208DF80A500021E8
S32508009E408DF80B008DF80C10ADF808008DF80D000D464FF6FF7736E0E01704EB907020F06A
S32508009E600300201A401C012806D002280BD0032810D004281BD114E038F8350007EA40107A
S32508009E80ADF8000013E038F8350007EA4010ADF802000CE038F8350007EA4010ADF8040094
S32508009EA005E038F8350007EA4010ADF80600641CA00707D16846FFF7FDFE9DF80A00401CC5
S32508009EC08DF80A006D1CB542C6DBA00702D06846FFF7F0FEBDE8FF8110B50A46102118B185
S32508009EE0012805D0002010BD1046FFF79CFF02E01046FFF745FF012010BD0246002011F4B5
S32508009F00700F03D0926904E001207047CB0104D552680A401103F7D170470B0101D5926812
S32508009F20F7E78B0101D5D268F3E71269F1E700000246002053690B424AD0B1F5807F3BD031
S32508009F4013DC08292ED007DC012926D0022927D004293DD1D0682BE0102925D0202926D0C5
S32508009F60402935D11069102130E0B1F5004F2BD00BDCB1F5007F22D0B1F5806F22D0B1F58F
S32508009F80006F25D19069702120E0B1F5803F11D0B1F5003F1CD15068E5E790680D4915E0E5
S32508009FA0D06802E0D068DEE7106903210EE0106908210BE05068FBE79069012106E09069D0
S32508009FC0022103E0906900E05068042100F0D2BD7047000001010100002A426901D00A438B
S32508009FE000E08A434261704710B50368002223F002030360036843F0010303604FF6FF73C3
S3250800A00000E0521C4468E40701D19A42F9D14268D2073ED08A79012A02683CD022F080020C
S3250800A0200260CA79012A026838D022F0400202600A7A012A026834D022F0200202604A7AA3
S3250800A040012A026830D022F0100202608A7A012A02682CD022F008020260CA7A012A0268EB
S3250800A06028D022F0040202608A78CC78920742EA04620C7942EA04424C79098842EA045220
S3250800A080491E0A43C261016821F001010160002114E0002010BD42F08002C1E742F040022C
S3250800A0A0C5E742F02002C9E742F01002CDE742F00802D1E742F00402D5E7491C4268D2071A
S3250800A0C001D09942F9D14068C007E2D1012010BD10460B0001D00021184770470846D1B2B2
S3250800A0E0C0B20AF0C1BA000070B58AB00121052004F094F90121480604F078F9474E0021B9
S3250800A100304600F097F8B014ADF8200003208DF822001820424C8DF8230008A9204601F073
S3250800A12039FDE014ADF8200048208DF8230008A9204601F02FFD00248DF81A4001258DF830
S3250800A1401B500C208DF818008DF816408DF817400920ADF8140007948DF8195005A9304677
S3250800A160FFF742FF8DF80E408DF80F408DF81050ADF80440ADF80840ADF80640ADF80A405E
S3250800A180ADF80C408DF8115001A8FFF793FD012202213046FFF720FF14208DF800008DF89C
S3250800A1A001508DF802408DF80350684603F0EAF8012211463046FFF70FFF0122510230463E
S3250800A1C0FFF70AFF012291023046FFF705FF0122D1033046FFF700FF0121304600F02AF840
S3250800A1E013208DF800008DF801508DF802408DF80350684603F0C6F816208DF800008DF885
S3250800A20001508DF802408DF80350684603F0BAF804A007F0C3FD0AB0002070BD00640040E7
S3250800A2200008014063616E2031206F70656E210A0000000000234FF6FF7221B1012917D08B
S3250800A240022924D03AE0016821F0020141F00101016000E0521E416801F00301012901D0BD
S3250800A260002AF7D1406800F00300012823D124E0016821F00301016000E0521E41688907BA
S3250800A28001D0002AF9D14068800714D115E0016821F0010141F00201016000E0521E4168D8
S3250800A2A001F00301022901D0002AF7D1406800F00300022801D0002300E0012318467047DB
S3250800A2C010B500EB0113D3F8B04114F004041472D3F8B04134D0E408C2F80440D3F8B041F8
S3250800A2E004F002045472D3F8B44104F00F049472D3F8B441240AD474D3F8B841D472D3F8B8
S3250800A300B841240A1473D3F8B841240C5473D3F8B841240E9473D3F8BC41D473D3F8BC41F2
S3250800A320240A1474D3F8BC41240C5474D3F8BC311B0E937439B1016941F02001016110BDDC
S3250800A340640D1460CAE7C16841F02001C16010BD09490A6842F001020A600A6843F60E7361
S3250800A3609A430A600A6842EA00200860086820F001000860704700000066004030B50246EF
S3250800A380002093685B0108D49068000101D5012003E09068C00044D5022002EB0012D2F8CD
S3250800A3A0803103F00103C2F880310B7AC3B3D2F880414D681C434B7A43EAC5031C43C2F80F
S3250800A3C080418B7A03F00F038B72D2F8843123F00F03C2F88431D2F884318C7A2343C2F8EF
S3250800A3E08431CB7A8C7B0D7B43EA04634C7B240444EA05242343C2F88831CB7B8C7C43EA98
S3250800A40004634C7C097C240444EA01210B43C2F88C31D2F8801141F00101C2F8801130BD77
S3250800A42001E00420FBE7D2F880314C7A23430C8843EA4453C2F88031C3E70000002221B11F
S3250800A440012905D0022906D112E08268114801E08268114802401149501A8A4214D00ADCF8
S3250800A460A2B16FF0806010180FD002280CD10FE082680B48EEE7B0F5007F09D00949401886
S3250800A48003D0B0F5003F03D000207047022070470120704703000004000300080001000881
S3250800A4A0000003100001FFF770B5124881888288A0F1300400253038616AC06971B13C212D
S3250800A4C0B0FBF1F0C000FEF73AF90B49FDF751FF0A4908606562E561256270BDA16A3C2976
S3250800A4E004D2491C1044A162E06170BD0120C4E9090570BD5000002000401C46400C0020C7
S3250800A500054810B590F8210008B1012010BD292001F06AF9002010BD040D002010B50178D2
S3250800A520427801EB0221144AA2F81B108178C37801EB032109B2B1F57A6F02DDA1F57A6143
S3250800A54001E0C1F57A6109B20B4C8BB23D34A2F81D300A2902DBA4F8073002E00021A4F852
S3250800A56007100179437901EB032122F81F1F80799070012010BD0000040D002000B5024603
S3250800A5800078FEF797FC134BD8725078FEF792FC18739078FEF78EFC5873D078FEF78AFC1A
S3250800A5A098731079FEF786FCD8735079FEF782FC18749079FEF77EFC064958744839D1F892
S3250800A5C0532041F8012FB1F856208A808871012000BD0000040D002010B508A007F0DEFB23
S3250800A5E000F0A0F900F074F900F092F902F06CFF044802F00EFE012010BD000054310D0ABB
S3250800A600000000008809002010B502A007F0C6FB022010BD5431300D0A00000010B502A03A
S3250800A62007F0BCFB062010BD5431310D0A00000010B502A007F0B2FB062010BD5431320DDC
S3250800A6400A00000010B504A007F0A8FB02F01CFF00F068F9002010BD5431330D0A000000C5
S3250800A66010B503A007F09AFB00F05CF9012010BD5431340D0A00000010B509A007F08EFBE7
S3250800A68002F002FF084C01202072084802F0C1FD0020E071064802F09CFD072010BD000074
S3250800A6A05431350D0A00000090230020800900207009002010B509A007F070FB094802F093
S3250800A6C088FD00F025F902F0FFFE074900200870064908700649087010BD00005431360DDF
S3250800A6E00A000000880900202100002020000020100B002010B503A007F050FB02F0E4FE57
S3250800A700022010BD54320D0A0000000010B502A007F044FB032010BD54330D0A0000000074
S3250800A720044810B50021C174018203A007F036FB042010BD6823002054340D0A000000001B
S3250800A74010B502A007F02AFB052010BD54350D0A0000000010B502A007F020FB062010BD6A
S3250800A76054360D0A0000000010B506A007F016FB06490020487100F0D5F802F085FE00203D
S3250800A78010BD000054370D0A000000007C23002010B502A007F002FB022010BD54380D0A90
S3250800A7A00000000010B502A007F0F8FA022010BD54390D0A0000000010B5252000F0F6FFB9
S3250800A7C00021044805F0CCFABDE81040012000F057BA0000A023002010B5154C606A002831
S3250800A7E001DA14A01CE0606A400001D515A017E0606A800001D518A012E0606AC00001D50A
S3250800A8001AA00DE0606A000101D51BA008E0606A400101D51CA003E0606A800102D51DA0E0
S3250800A82007F0BCFA606A40F08070606210BD000000100240B5CDB9A6BAC4B8B4CEBB0D0A27
S3250800A84000000000B4B0BFDABFB4C3C5B9B7B8B4CEBB0D0A00000000B6C0C1A2BFB4C3C5A2
S3250800A860B9B7B8B4CEBB0D0A00000000C8EDBCFEB8B4CEBB0D0A0000C9CFB5E72FB5F4B512
S3250800A880E7B8B4CEBB0D0A00D2FDBDC5B8B4CEBB0D0A0000424F52B8B4CEBB0D0A0000006B
S3250800A8A010B5094802F095FC012000F0E8FC074802F0AFFC4FF4FA7000F0E1FCBDE81040A1
S3250800A8C0024802F086BC0000C8090020D009002010B502F0AFFB4FF4FA7000F0D0FC02F046
S3250800A8E0C5FB044901204871BDE8104002A007F055BA000090230020434C4F53455F3132BB
S3250800A90056506F7765725265616C790D0A000000024900200872024802F05BBC90230020A7
S3250800A92080090020024900208871024802F051BC90230020600900200249002088710248A9
S3250800A94002F047BC902300206009002030B50C46054600F005F8024628190088504030BD9B
S3250800A96070B504464FF6FF7048F2050503460EE014F8012B80EA02200022491E060403EAE7
S3250800A980400000D56840521CD2B2082AF6D30029EED170BD0A48026FB0F84630B0F8480019
S3250800A9A0118801EB81014900B1FBF3F1494201EB81014FF2600303EB410108445080704709
S3250800A9C0CC0600200120704770B5124D124C2878072811D011480069804702280CD000205E
S3250800A9E020702878801E042801D801202070062000F0ECFE48B901E00320F1E7287806281A
S3250800AA0005D1074802F0F4FB08B902202070207870BD000068230020900500205800002012
S3250800AA20A80900200088322801D80120704700207047000010B506480649C08F898A88423F
S3250800AA4004D2282000F0D0FE002010BD012010BDCC060020040D00201D4810B5007920B19A
S3250800AA60012807D002280CD108E01121194801F02FF806E0174801F057F802E0112001F0A5
S3250800AA8063F8134832213038044605F069F9012805D108F0D9F80021204605F061F90E49A1
S3250800AAA0886BC20612D520F0100088630848FA212838044605F054F9012807D108F01EFB72
S3250800AAC02046BDE81040002105F04AB910BD00007C230020752D0108040D002070B5204DFA
S3250800AAE00026A889401C80B2A8810A2802D3AE8101F0EEFA1B491C4CA1F1FC008A88130AA2
S3250800AB0000F8E83F42708A790274C97941746889401C80B26881642814D36E81134D94F830
S3250800AB202800297881420DD0287008212846FFF717FF2872000A687200230A2229460C48D3
S3250800AB4000F062FD6078012808D1A078012805D16670A67001F016FE0120607170BD000097
S3250800AB60140B0020D4350020A8440020FE44002008450020024600200A4200D00120704728
S3250800AB80034900200978490700D5012070470000D4350020034900200978890700D5012021
S3250800ABA070470000D4350020034600201AB18B4200D0012070478B42FBD070470349002043
S3250800ABC0497A002900D0012070470000D43500200021012801D0032800D10121084670476C
S3250800ABE00021012805D0022803D0042801D00A2800D101210846704701460020090600D4BA
S3250800AC0001207047024600208A4200D1012070470120704770B517490020174E08601439DA
S3250800AC200446C87004EBC40006EB40050C3510212846FDF7E3FA10212846FFF791FE28742A
S3250800AC40000A641CE4B26874122CEBD30A494FF4A2740C3122460D4601F5A270FDF7B5FA9F
S3250800AC60002322462946054800F0CEFCBDE8704006F044BA280B0020EC35002091450020F2
S3250800AC80024A012110440172704700009C230020044810B500698047022801D0002010BDB2
S3250800ACA0012010BD5800002070B58F480521064603F088FD8D4C002518B12573304603F072
S3250800ACC093FD894805210830064603F07BFD18B1A573304603F088FD8348052110300646A4
S3250800ACE003F070FD18B12574304603F07DFD804CE06880477F49884203DA2A2000F066FDBA
S3250800AD0040B3E06880477C49884206DB2A2000F05DFD10B12A2000F049FDE068804777490F
S3250800AD20884203DD322000F051FDB8B1E06880477349884206DC322000F048FD10B1322051
S3250800AD4000F034FD6F4C94F84C00C0F30100032808D00AE02A2000F047FDDEE7322000F00B
S3250800AD6043FDEFE72E2000F03FFD606CC0F38160032802D10B2000F037FD606CC0F3017098
S3250800AD80032802D12B2000F02FFD606C800F032802D12C2000F028FD606CC0F3014003289B
S3250800ADA002D12D2000F020FD606CC0F38150032802D10C2000F018FD94F84400C0F3000056
S3250800ADC010B10D2000F010FDB4F84400C0F38130032802D10E2000F007FD94F84400C0F383
S3250800ADE0800010B10F2000F0FFFC94F84400C0F3C00010B1102000F0F7FC94F84400C0F350
S3250800AE00001010B1112000F0EFFC94F84400C0F3401010B1122000F0E7FC94F84400C0F32B
S3250800AE208110032802D1132000F0DEFC206CC0F3806010B1142000F0D7FC206CC0F3006002
S3250800AE4010B1152000F0D0FC206CC0F3406010B1162000F0C9FC206CC0F3007010B1172000
S3250800AE6000F0C2FC206CC00F02D0182000F0BCFC206CC0F3404010B1192000F0B5FC206C23
S3250800AE80C0F30150032802D11A2000F0ADFCB4F84000C0F3C02010B11B2000F0A5FC94F837
S3250800AEA05C00C0F3800010B11D2000F09DFC94F85C00C0F3C00010B11E2000F095FC94F807
S3250800AEC05C00C0F3401010B11F2000F08DFC94F85C00C0F3C010002804D0BDE87040202090
S3250800AEE000F082BC70BD0000B4340020302400205800002000000841000010410000944186
S3250800AF0000009041B822002070B51949194800F079FD0546174818490C3000F073FD164904
S3250800AF20164C1D39B1F81D10B9B1012D05D0B1F5A07F12D9032804D00FE0012000F054FC09
S3250800AF4012E00321204603F03DFC30B1052000F04BFC204603F048FC06E0204603F044FCE2
S3250800AF60032000F033FC08B1002070BD012070BD4C0C0020C0230020210D0020A43400206C
S3250800AF8010B52A2000F022FC08B9FDF79FFD114C60688047552803DB302000F025FC06E0A7
S3250800AFA060688047502802DC302000F0FFFB0A4890F90000552804DBBDE81040312000F0F7
S3250800AFC013BC502804DCBDE81040312000F0EEBB10BD000058000020902300200A4810B52E
S3250800AFE00078002448B1411E032901D8012404E0052801D0072800D1022400F0C9FB00B1B8
S3250800B0000324204610BD00006823002010B541F2883421460D4804F0A3FE012808D00B48C4
S3250800B0202146001F04F09CFE012806D0012010BD252000F0D9FB012003E0242000F0D4FBF1
S3250800B040002003F001FE002010BD0000A0230020007870472DE9FE4F01A9264800F0C4FAA8
S3250800B060254D264E264FDFF89C80DFF89C90002436F8140000F0A2FFFF2813D037F8100031
S3250800B08001992844029039F8140038F814B0084482465946FFF75AFC20B95A465146029828
S3250800B0A0FDF793F8641CE4B2092CE1D306F0FEF9104869460A3800F097FA08210098FFF796
S3250800B0C045FC124938B1002081F82900C87081F82800BDE8FE8F00980D4A0078107081F8B0
S3250800B0E028000328F5D30A2081F829000120C870EFE7000012450020D834002020790108E7
S3250800B100C07801084479010832790108A8440020FE4400200029016802D041F0010102E07F
S3250800B1204FF6FE7211400160704730B5036847F6F07293430C6A8A682243D1E904452C43DF
S3250800B14022438C692243CC6922434C6A22438C6A22431A430260CA6842600A68826049687A
S3250800B160C16030BD70B50C46050033D08CB36888A52121705A2161701930A070000AE070AF
S3250800B18020202071601D10221349FDF71EF868796075B5F805001726000AA0756A88022AD9
S3250800B1A007D304F11700E91DFDF70FF8A8781730C6B231462046FEF70DF8A055761CF1B2BA
S3250800B1C0000A6054491CC9B22046FEF7EDF9012070BDFFE70020FBE728150020F8B5694693
S3250800B1E0214800F001FA1226204F0024009804EBC40500EB4500B11EFFF7A8FB88B9009861
S3250800B200324600EB450107EB45000C30FCF7DDFF0098324600EB4501154800EB4500FCF774
S3250800B220D4FF07EB4500007B092805D111480121A14002680A430260641CE4B2122CD5D303
S3250800B24006F04AF90B494FF4FA701439888018314FF0FF30A1F1150208600749A1F5227011
S3250800B26003F0D0FDF8BD000091450020EC3500203C370020280B002080380020704710B5DA
S3250800B280044606E0142006F041FD01F0ABFC641EA4B2002CF6D110BD70B5044600F0B6FEC5
S3250800B2A00646FF2822D0204600F088FEFF281DD00F49114A0C5C0F4932F8100045182146BA
S3250800B2C02846FFF74DFB2855641C000A28550B48621C30F816100A48081803D0002329463A
S3250800B2E000F092F9BDE8704006F0E0B870BD0000E6780108D8340020C0780108327901082D
S3250800B300124500202DE9F8411C46002688468DF80060217815464A1C592322706B5421785E
S3250800B320194F4A1C227068546A463946404603F069FD22E037F816002178020A13484B1C27
S3250800B34050F8220023704FEA104C05F801C021784FEA102C4B1C237005F801C021784B1CC9
S3250800B3602370685402EBC20108EB410042782078411C2170761C2A54F6B29DF80000864237
S3250800B380D8D30020BDE8F88180380020507801082DE9F0434FF05908DDE90754002694F851
S3250800B3A000C04FF001090CF10107277005F80C80277807F1010C84F800C0E855224F21F0B2
S3250800B3C07F4000BF57F826C0604536D120784FEA114C471C277005F800C020784FEA112C0D
S3250800B3E0471C277005F800C02078471C2770295406EBC601267813F81170701C2070AF5577
S3250800B400012A01D0FF2A1CD103EB41014FF00009487BB0B120780123421C22702B542278AB
S3250800B4200823501C2070AB542078891C284403F0A5FC21780844207003E0761CF6B2122EC9
S3250800B440C0D34846BDE8F08350780108524B10B5524A18781168C40602D541F0200101E0F9
S3250800B46021F0200111608106116802D541F0400101E021F0400111604106116802D541F066
S3250800B480800101E021F080011160000602D541F4807001E021F4807010605878C1071168D0
S3250800B4A002D041F4007101E021F4007111608107116802D541F4806101E021F480611160F8
S3250800B4C04107116802D541F4006101E021F4006111600107116802D541F4805101E021F414
S3250800B4E080511160C106116802D541F4005101E021F4005111608106116802D541F48041DA
S3250800B50001E021F4804111604106116802D541F4004101E021F400411160000602D541F42E
S3250800B520803001E021F4803010609878C007106802D040F4003001E020F400301060FFF727
S3250800B5403DFB28B3587A082803D3106840F010001060FFF733FB002819D110481438C188A7
S3250800B560491C8BB20021C380C82B04D9136843F001031360C18003895B1C9BB20381B3F505
S3250800B580967F04D9136843F002031360018110BD106820F01000DBE7D4350020280B002060
S3250800B5A030B50C460F4A00EBC00102EB41030C4D0C33122813D21878A0420FD0092C0DD1F5
S3250800B5C0184603F011FC587818B92878401C28705870587BFF2801D0401C58731C7030BD97
S3250800B5E0170B0020EC350020064A824205D07F3A824202D00A3A824202D101200A60704765
S3250800B600002070479145002010B50BF081FB012010BD000001A006F0C1BB00004556454EE4
S3250800B620545F410D0A00000070B515A006F0B6FB164D00244FF4FA766879D0B101F024FFC0
S3250800B6403046FFF71CFE6879B0B101F01DFF3046FFF715FE0E4801F0CBFD697988420ED0EF
S3250800B660641CE4B2052CE7D3BDE87040042000F0BBB8FFF72DF9E3E7FFF72AF9E7E770BDE5
S3250800B6804556454E545F41430D0A000090230020A009002001A006F081BB00004556454E83
S3250800B6A0545F420D0A00000001A006F077BB00004556454E545F430D0A00000070B516A091
S3250800B6C006F06CFB174D00244FF4FA76A87901281BD001F00DFF3046FFF7D1FDA87901280E
S3250800B6E016D001F005FF3046FFF7C9FD0E4801F07FFDA97988420ED0641CE4B2052CE5D3A3
S3250800B700BDE87040032000F06FB8FFF715F9E2E7FFF712F9E7E770BD4556454E545F44435B
S3250800B7200D0A000090230020A809002010B510210548FCF763FD054900200860087108391A
S3250800B7400860486010BD0000202400203008002070B50A4C052604F108052068616888427F
S3250800B7600BD0295C06A006F019FB2068401C90FBF6F106FB11002060F0E770BD280800206F
S3250800B780457272204E554D2069732025640D0A00054900200A5C0AB101207047401CC0B271
S3250800B7A01028F7D3002070472024002010B5034600F00CF830B1DC08184600F079F902496C
S3250800B7C000200855012010BD20240020C20800F007010448805C01228A40104000D0012074
S3250800B7E0704700002024002010B50346FFF7EEFFA0B90B4AA2F10801486813540522401C4B
S3250800B80090FBF2F402FB140048600649D80803F007030A5C01249C4022430A54012010BDAC
S3250800B82030080020202400200149C860704700000020024070B50D4E0546304600F088F802
S3250800B840042811D10A4C206940F0020020616561206940F040002061304600F079F8216999
S3250800B86041F6FD721140216170BD0000FFFF0F000020024008490420CA68D20701D0012033
S3250800B8807047CA68520701D502207047C968C906FBD50320704700000020024002480169E9
S3250800B8A041F080010161704700200240F0B506464FF6FF770D46384600F04AF804280DD194
S3250800B8C0074C206940F0010020613580384600F03FF8216941F6FE7211402161F0BD0000C1
S3250800B8E0002002402DE9F841064600204FF6FF7700900D46384600F02BF8042817D10D4C81
S3250800B900206940F0010020613580B846384600F01FF841F6FE77042806D1B61C280C00965B
S3250800B9203080404600F014F8216939402161BDE8F88100000020024003480249416003493F
S3250800B940416070472301674500200240AB89EFCD00B50346FFF78EFF03E000BFFFF78AFFBD
S3250800B9605B1E012803D0002B00D1052000BD002BF4D1FAE70A290FD801EB41020749038871
S3250800B98021F8223001EB820183788B70C278CA7002790A718068886070470000A8230020ED
S3250800B9A000B501211648FFF7E5FF154802210C30FFF7E0FF124803211830FFF7DBFF1048EB
S3250800B9C004212430FFF7D6FF0D4805213030FFF7D1FF0B4806213C30FFF7CCFF0848072155
S3250800B9E04830FFF7C7FF064808215430FFF7C2FF0348092160305DF804EBFFF7BBBF00009A
S3250800BA00BC07002010B5044682680846904721790022814202D0A27020710CE0E378834217
S3250800BA2001D1A27007E0A078401CC0B2A0702288904200D3E170E07810BD00002DE9F04725
S3250800BA4081461A48184C00278088401E86B204EBC60041684846FCF7C7FE04D348466168B4
S3250800BA60FCF7CCFE18D240F6FF70BDE8F087B819450804EBC5084846D8F80410FCF7BEFE55
S3250800BA8002D26D1EAEB207E04846D8F80410FCF7ABFE06D26D1CAFB2B742E8D934F9370004
S3250800BAA0E3E734F93500E0E7186E010820000020064A0021535C834202D100205054704783
S3250800BAC0491CC9B20529F5D370470000300800202DE9F041074612480E466421804604F0F2
S3250800BAE03FF900250F4C012806D1B847E57200214046656004F034F9E07A11280ED1607C4F
S3250800BB00B0420BD1606841F6EC41B1EB104F05D103490120E572403165600871BDE8F081C3
S3250800BB203C230020540D002010B501460220884704490220087103480021BDE810403C383D
S3250800BB4004F00EB97C23002070B50F4900240F4DCA7A0F4E132A0CD14A7C824209D1486891
S3250800BB6041F6EC42B2EB104F03D1CC724C602C71B463064832213C3804F0F2F8012801D1F6
S3250800BB802C71B46370BD0000540D00207C230020040D0020F0B5CA78002502F00F03D2065D
S3250800BBA001D58A7813430A784FF00F0E12F0FF0F4FF001021CD004680F8802FA05F63740BC
S3250800BBC0B74211D14FEA850C0EFA0CF724EA070703FA0CF43C43CF78282F02D0482F02D056
S3250800BBE002E0466100E006616D1C082DE4D304600C88FF2C1ED944685FF0000606F10807D1
S3250800BC0002FA07F50F882F40AF420FD14FEA860C0EFA0CF7BC4303FA0CF73C43CF78282F55
S3250800BC2000D14561CF78482F00D10561761C082EE4D34460F0BD0000F0B5144C002801DAB2
S3250800BC40E36900E06368420D120185B2C0F301579540C0F30346032F05D0C2020AD503229B
S3250800BC60B240934307E023F07062636823F07063636002E0AB4343F0706201B12A43002892
S3250800BC8001DAE261F0BD6260F0BD0000000001400246002092680A4200D001207047416123
S3250800BCA070470161704700787047000070B50C4C206980470B4D02280BD10B480321064689
S3250800BCC002F080FD28B1304602F08EFDA068804704E020698047022801D00020287070BD38
S3250800BCE05800002090230020AC3400200C4810B540880B4A01211C3A05F0AEFF08483038E3
S3250800BD004069FCF742FD02460B4606480649FCF787FCFCF74DFDFFF791FE0449488110BDE9
S3250800BD20500000209A99999999991340400C00207CB5002328A40093246801946D4601ACFB
S3250800BD40012825D0C85CE65C7040E8545B1CDBB2042BF7D39DF800109DF8010001F00F0429
S3250800BD60034664F31F13137003099DF8020043EA001353709DF8033003F0F00444EA1010BD
S3250800BD80907003F00F0040EA1110D07000207CBDC85CE65C7040E8545B1CDBB2042BF7D360
S3250800BDA09DF801109DF8000001F0F00343EA001313700B019DF8021043EA1113537001F0DB
S3250800BDC0F0039DF8031043EA111301F00F01937061F31F10D9E700009023B02170B505462E
S3250800BDE005F072F94443601C01D01CB105E06FF0A90402E005F068F904462C70200C687021
S3250800BE00200AA870EC70002070BD0000FEB5002604468DF8086053783D480D460B2974D2FC
S3250800BE20DFE801F07306065960737173737306000A4602A9204600F0FDF802004FF05900E1
S3250800BE404FF0090115D18DF8086020709DF80820521CD2B28DF80820A5549DF80820521CA8
S3250800BE60D2B28DF80820A1549DF80820521C8DF80820012D49D18DF8086020709DF8080054
S3250800BE80401CC0B28DF8080025549DF80800401CC0B28DF8080021549DF80800401CC0B2E8
S3250800BEA08DF8080026549DF80800401CC1B218488DF808100C38C27A62549DF80810491CBC
S3250800BEC0C9B28DF80810807A60549DF80800401C8DF8080019E0014602AB22462846FFF74F
S3250800BEE011FA12E063F31741937863F30F21D378127963F3070102ABCDE900430346284667
S3250800BF00FFF746FA08B18DF808609DF80800FEBDF835002070B516490324164B91F82C20B1
S3250800BF2091F82B10144D02EB01218AB262210170110A41708270002135F81160964203D067
S3250800BF40491CC9B21329F7D313290ED0022C0AD00A4A2044555C0A4A32F811102A461944F6
S3250800BF60FCF733F92C44204670BD0224FBE70000A8440020D8340020FA780108E67801086F
S3250800BF80C078010800B5FEF7FBFD0B4A0028106802D040F0080001E020F008001060FEF753
S3250800BFA0F9FD0028106802D040F0040001E020F00400106000BD0000280B0020024610B555
S3250800BFC0FF20074B002100BF33F81140944201D1084610BD491CC9B21329F5D310BD000012
S3250800BFE0FA780108007A704700797047C079032801D000207047012070477047704770474E
S3250800C000533530385F44435532343031024610B5FF20074B002100BF33F81140944201D19E
S3250800C020084610BD491CC9B20929F5D310BD0000207901082DE9F043224C0027592567814A
S3250800C0400570427009258946857039465FF0030501EBC10604EB460C9CF80C601E4203D1BB
S3250800C0609E4201D00A2A23D1174E3668CE40F6071ED066890127761C6681144E56F82180FC
S3250800C0804FEA184800F805806D1C36F82180EDB24FEA182800F805806D1CEDB216F82160D8
S3250800C0A046556D1CEDB29CF80C6046556D1CEDB2491CC9B21229CBD389F800503846BDE83F
S3250800C0C0F0830000EC3500202C0B0020507801082DE9F0412F4DA88818B1401EA880BDE88F
S3250800C0E0F081FFF74FFFFFF7B1F92B4890F827000028F4D12748294F14300024D0F8006057
S3250800C10026FA04F0C00701D0092106E004EBC40007EB4000007B20F001012046FFF740FA4D
S3250800C120641CE4B2122CEBD32878122600EBC00007EB40041A4F14F80C1F17F810008142A4
S3250800C14014D010212046FEF70BFC2074000A60742878217800EBC002002307F81210114964
S3250800C160324606FB00102146FFF74EFA2878401CC1B200202970122900D328706978491C6F
S3250800C180C9B269706429AAD36870BDE8F04105F0A3B90000140B0020A8440020EC350020A8
S3250800C1A03C3700209145002000210D4A0CE0834206D101EB410000EBC10002EB001070475B
S3250800C1C0491CC9B2022908D201EB410303EBC10302EB03131B78FF2BE9D100207047000039
S3250800C1E0441300202DE9F0470026DFF80C81DFF80C91DFF80CA1434C4FF400474FF6FF7519
S3250800C200012804D0022817D0032854D070E0EB21822008F029FCA0F50041E080B94202D293
S3250800C220281AE08002E0A84200D3E680E088FCF78BFA42464B4652E0E321B22008F014FC40
S3250800C240E080B84204D301216180281AE08000E0668080B2FCF778FA42464B46FCF76EF92A
S3250800C26000225346FCF7DCF9FCF7A2FAFCF78DFA4FF03332244BFCF761F9244A244BFCF7F4
S3250800C280CFF9FCF795FAA0616088012830D11D484FF4FA61143003F063FD012807D11DA0DB
S3250800C2A005F07CFD17480021143003F059FDA06980F000401BE0E321B42008F0D5FBA0F50C
S3250800C2C00041E080B94202D2281AE08002E0A84200D3E680E088FCF737FA4246164BFCF7D1
S3250800C2E02DF900225346FCF79BF9FCF761FAA061A069BDE8F0870000FCA9F1D24D622040DD
S3250800C300E0FFEF407C000020F308CA40F6285C8FC2F513404E6567617469766520766F6CA9
S3250800C320746167652073616D706C65206661756C74210D0A000000004D6210408079012817
S3250800C34002D0002800D00020704700000148B0F90A007047400C0020014840687047000067
S3250800C360400C00202DE9F84F05462D4800248DF80040006F016B8847DFF8A89003462A49C8
S3250800C38099F80080012602200322284F6FF0814CDFF89CA02944AC44B8F1000F0AD0B8F1C2
S3250800C3A0010F1ED0234BB8F1020F1FD0B8F1030F2CD120E0DFF88080B94203D298F80F104C
S3250800C3C0022910D31D4929441D4DA94203D298F80F10022911D2D44515D3BBB188F80F404B
S3250800C3E014E0B94212D28DF8006011E0994204D3D44508D30AE0994202D28DF8002007E0BB
S3250800C40010498C4502D28DF8000001E08DF8004069460D48FFF7F6FA89F80000BDE8F88F4E
S3250800C420CC060020100B0020F528DCC3285C4F04FFFF3F00F5289C0368230020CCCCCCC066
S3250800C440CCCC8C00FFFF5F00B42300202DE9F0411448046814482146FBF753FF0546134999
S3250800C4602046FBF754FF2946FBF783FFFCF78DF90F4D8846044600222B46FCF75CF806460D
S3250800C4800F462046414600222B46FCF757F832463B46FCF7C5F8FCF78BF906490860BDE8FB
S3250800C4A0F0810000400C00200000A0403333A34000002440580000200148B0F908007047DB
S3250800C4C0400C00204079012802D0002800D000207047000001484078704700002000002067
S3250800C4E070B53F4E7088401C80B270800A286FD33C4C00257580B4F840004FF4FA7188428C
S3250800C50024D2401C80B2A4F8400088421ED12572607F032801D0022818D1257701206077DB
S3250800C52084F82250A5716574A4F8405084F824502C4884F8255084F827503838E57301795A
S3250800C540012901D18561057100F04AFB94F8241025480029017802D021F0030101E041F078
S3250800C5600301017094F825100029017802D021F00C0101E041F00C010170B4F8541031B163
S3250800C580491E0904090CA4F8541000D1E5733188491C89B2318064291AD3358094F82910DD
S3250800C5A079B1491E11F0FF0184F8291009D1E178012906D1E57094F8281011B1491E84F834
S3250800C5C02810217A0029017803D021F01001017070BD41F010010170BDE8704000F000BB92
S3250800C5E0B40B0020A8440020300B002000F00F00092801D93730704730307047000909286E
S3250800C60001D937307047303070470000074A30B45170064B0022083303E0845C9C54521C38
S3250800C620D2B28A42F9D330BC02F00ABEF40B0020064A10B5054B00215278083303E05C5CE5
S3250800C6404454491CC9B29142F9D310BDF40B002070B50C46054602F0A9FE02462146284651
S3250800C660BDE8704004F0D2BA074A30B45170064B0022083303E0845C9C54521CD2B28A42C2
S3250800C680F9D330BC02F034BEF40B002002F0E4BE10B504F037FB02490020087010BD0000A2
S3250800C6A0F40B00200148407870470000F40B00207FB50D496B464A6800928A788DF804204C
S3250800C6C0002104E0445C5D18491C6C71C9B29142F8D3064901208DF80D0048709DE80F0089
S3250800C6E003F0D4FB7FBD0000F40B0020A84400200149887070470000F40B0020024A40F26D
S3250800C700B471516070470000F40B002070B50D46064602F04BFE0A4C217800290ED17F21C9
S3250800C72001704670857003250020FFF7E7FF03F0C9F8284602F060FE0120207070BD00005B
S3250800C740F40B002070B50E46044602F02FFE0C4D2978002913D1002C11D0002203E0B15CA4
S3250800C7608154521C92B2A242F9D30020FFF7C6FF03F0A8F8204602F03FFE0120287070BD8B
S3250800C780F40B002002F022BD0078704700787047FEE700002DE9F0410427044600F1700635
S3250800C7A04FF001085FF0000594F89100062876D2DFE800F0031975424E5C94F854000328FD
S3250800C7C06DD330460AF05EF9002868D104F1940130460AF073F970B384F8918084F8905071
S3250800C7E084F8AC5050E0D4F808C094F89930207804F19A02D4F89410E04784F8980094F83A
S3250800C8009010491C84F89010FF280CD0022084F8910084F8AC5094F854008128C4D10320FE
S3250800C82084F85400C0E794F84400C9B2814236D384F891702CE027E094F8900094F84410D0
S3250800C840884202D384F891701EE084F891801BE084F89150D4F8A82022B10121D4F8A400D2
S3250800C860904711E0226D002AF7D10DE084F89150D4F8A81029B10220D4F8A42007F038F8E0
S3250800C88002E0216D0029F6D194F8910004288BD12278BDE8F0410421012007F029B8BDE852
S3250800C8A0F081000030B500201D49024604460125C1F8985105235B1E1B041B0CFBD140063B
S3250800C8C0D1F81C31000E0BB140F00100C1F8984105235B1E1B041B0CFBD1521CD2B2082AD0
S3250800C8E0E6D3C1F898410522521E1204120CFBD1C1F89C410522521E1204120CFBD1C1F862
S3250800C90098510522521E1204120CFBD1C1F898410522521E1204120CFBD1C1F89C5130BDCD
S3250800C920008021420F480122C0F89C210521491E0904090CFBD1C0F898210521491E090491
S3250800C940090CFBD10022C0F89C210521491E0904090CFBD1C0F898210520401E0004000CD2
S3250800C960FBD17047008021420C480021C0F89C110521491E0904090CFBD10122C0F898215A
S3250800C9800521491E0904090CFBD1C0F89C210520401E0004000CFBD17047000000802142A0
S3250800C9A030B516490024C1F8984122460123050602D5C1F89C3101E0C1F89C41C1F8983182
S3250800C9C005256D1E2D042D0CFBD1C1F8984105256D1E2D042D0CFBD14006521C000ED2B29B
S3250800C9E0082AE4D3C1F89C31C1F898310520401E0004000CFBD1C1F8984130BD0080214277
S3250800CA002DE9F041084D4FF400642C6007F039FF2F1F66103E6007F034FF2E6007F031FFC9
S3250800CA203C60BDE8F0810000140C014070B5084C4FF40060206007F024FF2515256007F069
S3250800CA4020FF201D0560BDE8704007F01ABF0000100C01402DE9F047144F0024DFF84C800E
S3250800CA6082462546A8F108083E1507F104096006040E3E6007F005FFD8F80000000501D5B8
S3250800CA80641CE4B2C9F8006007F0FBFE6D1CEDB2082DECD3BAF1000F04D0FFF7B1FF2046AB
S3250800CAA0BDE8F087FFF7C2FFF9E70000100C01402DE9F047DFF84890054600244FF48067C3
S3250800CAC04FF40068A9F104062806404601D5306001E0C9F8000007F0D4FE376007F0D1FE17
S3250800CAE0C9F80070072C01D1C6F800806806050E07F0C7FE641CE4B2082CE5D3BDE8F08759
S3250800CB00140C014070B509484FF4006505600415046007F0B6FE054E361D356007F0B1FE1A
S3250800CB203460BDE8704007F0ACBE0000100C014070B507484FF400640460054D00152D1F0E
S3250800CB40286007F09EFE2C60BDE8704007F099BE140C014070B50C4C4FF40060206007F085
S3250800CB6090FE2515256007F08CFE074808380068000501D5012400E000240348001D056011
S3250800CB8007F07FFE204670BD100C0140064A01880020B2F835308B4204D3B2F84320143224
S3250800CBA08A4200D803207047CC06002070B50B4D06680024B5F83900FBF7C1FD3146FBF7E9
S3250800CBC013FE01D2012407E0E88FFBF7B8FD3146FBF714FE00D20224204670BDCC06002041
S3250800CBE07047000003497F20086003490020087070470000002C0040780100200C48C169FF
S3250800CC0041F40061C1610B4940F2FF30086009487F21001F0160016841F0800101604FF005
S3250800CC20E020002180F800140121C0F80011704700100240042C00402DE9FE4342F20F78C3
S3250800CC40224CADF80080694621480194FCF7F6F840F6C315ADF8005069461D480194FCF706
S3250800CC60EDF841F64B561B4FADF80060694618480197FCF7E3F842F22730ADF80000694626
S3250800CC8013480194FCF7DAF840F2E730ADF800001148019069460E48FCF7D0F8ADF8006034
S3250800CCA069460B480194FCF7C9F8ADF80050694607480197FCF7C2F8ADF8008069460448C3
S3250800CCC00194FCF7BBF8BDE8FE83000045D80008CC34002055D90008C9EB00082DE9F04167
S3250800CCE00024154E5FF0FF0704EB440000EBC40006EB00100546B021FBF780FA641CE4B2C9
S3250800CD002F70022CF0D30D4C206818B90C4806F069FE206006F0C5FE18B90A21206806F05F
S3250800CD20B9FE0849012006F0FBFDBDE8F0410649022006F0F5BD000044130020D400002074
S3250800CD40B56D0108DDA00008D1A0000810B548210F48FBF753FA0E4828214830FBF74EFA87
S3250800CD600C4801F0C5FC010004D0094814224830FBF72BFA0748203001F0BAFC010006D097
S3250800CD8003481422BDE810405C30FBF71EBA10BD4C0F00207073010810B5284800F0B3F9B4
S3250800CDA02648083000F0AFF92448103000F0ABF92248183000F0A7F92048203000F0A3F961
S3250800CDC01E48283000F09FF91C48303000F09BF91A48383000F097F91848403000F093F921
S3250800CDE01648483000F08FF91448503000F08BF91248583000F087F91048603000F083F9E1
S3250800CE000E48683000F07FF90C48703000F07BF90A48783000F077F90848803000F073F9A0
S3250800CE200648883000F06FF90448903000F06BF90248BDE81040983000F065B96009002088
S3250800CE4070B51A4C1B491C486278194D09780069052A18D2DFE802F003091E101800E87BC0
S3250800CE6008B103200EE001200CE0072902D080470228F8D1022005E00729F2D08047022827
S3250800CE80EFD00420607070BD0729F3D080470228F7D1EFE700F022FB00266E606E7301F04F
S3250800CEA0A3FBA8606670267070BD0000380800203024002068230020580000202DE9F041E7
S3250800CEC016460D46FFF770F9040007D035B12EB1287818B194F85400012802D00020BDE88D
S3250800CEE0F08195F82000C00702D0A86A0028F6D095F8250084F8450010B9322084F845001E
S3250800CF00C0B200EB4000C00004F09AFFC4F88C00011EE4D094F84530182204F1700009F065
S3250800CF20C1FD95F82000C0070FD194F84500000104F086FFC4F88800011E2ED094F8453024
S3250800CF40102204F1580009F0ADFD286A206404F1200007462021FBF751F91F22294638467E
S3250800CF60FBF733F9E86AF862A86AB86295F8240087F82400286B38630B4830610B48F060A4
S3250800CF800B48B0600B4870600B4830600B487061022084F854000120A1E754F88C0F04F080
S3250800CFA021FF0020206099E7854E0108F54C0108674D0108774D0108EB4D0108614C01087C
S3250800CFC038B5044601213C2001F028FA0121084601F024FA01211248FEF72EFEA468B4B1EE
S3250800CFE02088ADF8000010208DF8030002208DF8020069466068FEF7CDFD207A01280AD0A2
S3250800D000002803D121886068FEF749FE38BD05A004F0C4FE38BD21886068FEF742FE38BD79
S3250800D020000230004F5053206973204E554C4C0D0A00000010B5044800F0CBF8BDE8104097
S3250800D040024800F0E6B80000C8090020D009002010B5044800F0BDF8BDE81040024800F01B
S3250800D060D8B80000D0090020C809002010B5044800F0AFF8BDE81040024800F0AAB80000EF
S3250800D080C8090020D009002010B5054800F0A1F8044800F09EF8BDE8104003A004F07EBE63
S3250800D0A0C8090020D0090020414320C8ABB5CD0010B5054800F0ADF8044800F0AAF8BDE8B5
S3250800D0C0104003A004F06ABEC8090020D0090020414320C8ABB8DF0038B504460121102012
S3250800D0E001F09CF9A06800280CD00188ADF8001004218DF8031003218DF802104068694683
S3250800D100FEF748FD38BD00680168002900D008477047000038B5044601213C2001F07EF9E5
S3250800D120A468B4B12088ADF8000010208DF8030002208DF8020069466068FEF72BFD207A94
S3250800D14001280AD0002803D121886068FEF7A7FD38BD04A004F022FE38BD21886068FEF7B0
S3250800D160A0FD38BD4F5053206973204E554C4C0D0A00000038B504460121042001F04EF9FA
S3250800D180A468002C15D02088ADF8000010208DF8030003208DF8020069466068FEF7FAFC53
S3250800D1A0207A012806D0002803D121886068FEF776FD38BD21886068FEF773FD38BD10B56E
S3250800D1C0044601884068FEF76AFD00202072012010BD10B500684168496819B180688847C2
S3250800D1E0012010BD002010BD01884068FEF750BD00684168896809B1806808470320704746
S3250800D20010B5044601884068FEF74BFD0120207210BD10B500684168096819B1806888473B
S3250800D220012010BD002010BD38B504460121102001F0F4F8A06800280CD00188ADF8001055
S3250800D24048218DF8031003218DF8021040686946FEF7A0FC38BD00000A4810B5C088094A75
S3250800D2600221203A04F0F8FC0648074930380069FBF74DF84FF07A51FAF7F1FF03494860B6
S3250800D28010BD00005000002000003041400C002030B504465FF0000014F8015B8D4203D1DD
S3250800D2A0012A08D0521ED2B2002B04D0401C5B1E80B29BB2F0E730BD124810B5C07E124C97
S3250800D2C0012813D04FF47A700146A0600E4802F047FD012814D1606810F0010F00F101005C
S3250800D2E060600A4804D0FFF774FF03E06420EBE7FFF78FFFBDE810400021034802F030BDD4
S3250800D30010BD0000800C00200000002098090020094B9A7A72B1094841780B44DB7A03B1B8
S3250800D3208380491CC9B241708A4201D8002141700079704700207047300B002090050020BD
S3250800D34003A004F02BFD04F0C1FC00F003FC0000476F20746F20536C6565700D0A00000077
S3250800D360FEE770474FF4A06000F03EB800F01F02012191404009800000F1E020C0F88011D3
S3250800D3807047000070B50F23C47801780122F4B1144C2468457804F4E064C4F5E064240AE4
S3250800D3A0C4F10406E3408478B5401C402C4301F1E021230181F80034007800F01F018A40AB
S3250800D3C04009800000F1E020C0F8002170BD01F01F0082404809800000F1E020C0F8802192
S3250800D3E070BD00000CED00E00249084302490860704700000000FA050CED00E0024A1140A4
S3250800D400014302480160704780FFFF1F08ED00E004480168044A01F4E06111430160BFF346
S3250800D4204F8FFEE70CED00E00400FA0504480168044A01F4E06111430160BFF34F8FFEE7DC
S3250800D4400CED00E00400FA054FF400720021014803F036BE0845002010B50948FFF7D9FE8C
S3250800D4600120FDF70CFF0748FFF7D3FE4FF4FA70FDF705FFBDE810400248FFF7AABE000026
S3250800D480C8090020D009002010B5FFF7E1FD4FF4FA70FDF7F4FEFFF7E9FD04490020487166
S3250800D4A0BDE8104002A004F079BC0000902300204F50454E5F313256506F7765725265615C
S3250800D4C06C790D0A0000000002490120C8710248FFF79FBE90230020700900200249012028
S3250800D4E0C8710248FFF795BE90230020700900200249012088710248FFF78BBE9023002025
S3250800D50060090020007808B10020704701207047014908627047000000000E4202490A681C
S3250800D52042EA8000086070470070004000B50B30034609F023FB18680D49C0F309300A2224
S3250800D54021F83C0F1868C0F3093090FBF2F081F830005868800C48805868800C488118682E
S3250800D5601A79800D62F38D208881012000BD0000CC06002070B50B30044609F0FFFA0A4DAF
S3250800D5806068296FC0F3C260496A8847296F2068C96AC0F3026088472068C0F3407085F827
S3250800D5A05900012070BD0000CC06002000B50B30034609F0E3FA98880A2280B290FBF2F0CA
S3250800D5C00A49A1F866005868000C90FBF2F0A1F868005868000C90FBF2F040F4805021F85B
S3250800D5E04A0F1868000C4871012000BDCC06002000B50B30034609F0C1FA98880B49000A44
S3250800D6000A3081F86A005868000E0A3081F86B009888000A01F8500F5868000E88705868EB
S3250800D620000C48701879C870012000BDCC06002010B50446FBF7EEFC0B34204609F09EFA5E
S3250800D64060684FF6FF71C0F3892000EB800001EA4000044921F8410F6068000D48800120D9
S3250800D66010BD0000CC06002000B500F10B03184609F084FA0348196801635968416301209E
S3250800D68000BD0000B822002000B500F10B03184609F074FA0348196881635968C163012096
S3250800D6A000BD0000B822002000B500F10B03184609F064FA03481968016459684164012084
S3250800D6C000BD0000B822002070B500F10B04204609F054FA2068154DC0F340400A2185F8EE
S3250800D6E045006068000C90FBF1F0A5F83300A088C0F38D002880207868712088000A85F817
S3250800D7003B00A088C0F38D00A5F83900296F2068C968C0F3004088472068C0F3004085F877
S3250800D7205A002068800C2881012070BDCC06002000B50B30034609F021FA98880549C0F316
S3250800D7408D00C8805868000DC0F57A60A1F83500012000BDCC06002000B50B30034609F0BA
S3250800D7600DFA18680549C0F38930A1F837000448196881655968C165012000BDCC06002020
S3250800D780B82200202DE9F0472348244F0122868A07F2FA2500206F6028703346202138464C
S3250800D7A0FFF776FD687004461DA0696804F0F6FAB4422AD0022025E0385D202828D02978D1
S3250800D7C0A14605EB810107EB090088603346424620211248FFF75CFD2A7815490446A0EB3F
S3250800D7E009005054297805EB8100826811A004F0D5FA2878401CC0B22870042805D208F1FC
S3250800D8000100C0B28046B442D6D10120BDE8F087641CA4B2F7E700008C0100209A1D0020AF
S3250800D820696E6F757420636D643A25730A000000AC200020256420706172616D3A25730AF9
S3250800D840000000002DE9FC4100203E4C00904FF44571019021606160207260720820A072C3
S3250800D860E84600F0EBFF054600F0FCFF019A65F3196265F39B6260F31D72334D60F39F72D3
S3250800D8800192287A10B3002060F311420192E879F0B1002060F393420192FDF79FFB009A24
S3250800D8A060F38B220092FDF78FF8DDE9006760F3155726480197C068FAF753FF80B20A2193
S3250800D8C0B0FBF1F0C82805D2002004E00120DBE70120DFE7C83860F35D561D48CDE9006791
S3250800D8E0006FB0F9020090FBF1F000F5FA7060F314360096FDF7CCF9009A60F3DF722420C7
S3250800D9000092FDF763FFDDE9002160F39E72687A60F34F31CDE90021687808B9A87800B1C9
S3250800D920012060F3D7514046019109F02EF9009844F80B0F01986060024806F0DBF8BDE806
S3250800D940FC8100002023002090230020400C0020CC0600202DE9FC410024374E00944FF4D5
S3250800D9607A70019430607060347274720820B072E8462820FDF72AFF58B92620FDF726FFE1
S3250800D98038B91C20FDF722FF18B92120FDF71EFF08B1012200E00022019962F38E31274A17
S3250800D9A0019113781B1F022B05D8D27C1AB1012262F3CF310191FDF707F8022803D0FDF7F1
S3250800D9C003F8032803D1019864F3CF3001901C4F78688047DDE90054283060F31F64194804
S3250800D9E019490078283060F3174401943868FAF78EFCFAF7B6FE42F21071884200D908463E
S3250800DA0060F30D041148807A60F30B25CDE90054FFF77EFC009960F307014046009109F040
S3250800DA20B4F8009846F80B0F01987060024806F061F8BDE8FC81000020230020682300200A
S3250800DA40580000209023002000007A44300B00207CB50021144B009140F23F400191186057
S3250800DA6058601972114C597208209872A2786846521CD2B2A270102A00D3A1700099012552
S3250800DA80A47865F3CF3164F30B21641C64F30701009109F07AF8009843F80B0F0198586068
S3250800DAA0014806F027F87CBD20230020900500201FB5104A012010720020A2F84000009B43
S3250800DAC09DF80410A3F5E0636846343B09D0AB2B06D140F2DF73A2F84E30401DFEF796FD90
S3250800DAE01FBD40F23473A2F84E30401DFEF7BCFD1FBD0000A844002000B50B30034609F026
S3250800DB003DF80648196801615968416104495868096F000C0880012000BD0000B82200203D
S3250800DB20CC06002070B50B30044609F027F8074D2068296FC0F30360C9698847296F606838
S3250800DB404969800F8847012070BD0000CC060020704700004FF0E020016921F00201016191
S3250800DB600220FFF703FC0320FFF700FC0420FFF7FDFB0520FFF7FAFB0620FFF7F7FB072014
S3250800DB80FFF7F4FB0820FFF7F1FB0920FFF7EEFB0A20FFF7EBFB0B20FFF7E8FB0C20FFF754
S3250800DBA0E5FB0D20FFF7E2FB0E20FFF7DFFB0F20FFF7DCFB1020FFF7D9FB1120FFF7D6FB8B
S3250800DBC01320FFF7D3FB1420FFF7D0FB1520FFF7CDFB1620FFF7CAFB1720FFF7C7FB182040
S3250800DBE0FFF7C4FB1920FFF7C1FB1A20FFF7BEFB1B20FFF7BBFB1C20FFF7B8FB1D20FFF78F
S3250800DC00B5FB1E20FFF7B2FB1F20FFF7AFFB2020FFF7ACFB2120FFF7A9FB2220FFF7A6FBF5
S3250800DC202320FFF7A3FB2420FFF7A0FB2520FFF79DFB2620FFF79AFB2720FFF797FBFEF7C2
S3250800DC40D1FF2820FFF792FB2920FFF78FFB2A20FFF78CFB3220FFF789FB3320FFF786FBF5
S3250800DC603420FFF783FB3520FFF780FB3620FFF77DFB3720FFF77AFB3820FFF777FB392069
S3250800DC80FFF774FB3A20FFF771FB3B20FFF76EFB3C20FFF76BFB3D20FFF768FB3E20FFF7D9
S3250800DCA065FB3F20FFF762FB4020FFF75FFB4120FFF75CFB4220FFF759FB4320FFF756FB90
S3250800DCC00020411E820002F1E022C2F88011401C0828F7DB0120FFF721FCFEF783FF09489B
S3250800DCE0FFF797FA0848C07B0028084802D0FFF790FA01E0FFF76DFA41F28830FDF7BFFA64
S3250800DD00FFF794FBF809002030240020F009002070B56249624E634C4868634D401C48602F
S3250800DD200521B0FBF1F201FB120005287AD2DFE800F0033347728F005CA004F02FF8287AAC
S3250800DD4008B165A105E0306980475449083151F8201064A004F022F8206F016A88474F49EF
S3250800DD604C3151F8201066A004F018F86A484B4994F86C200078143151F8201067A004F006
S3250800DD800DF894F8450008B16CA100E06FA173A0BDE8704004F002B8B4F84320B4F84110C7
S3250800DDA074A003F0FBFF7E48B0F81D20B0F81B107CA003F0F3FF206FB0F9021084A0E7E799
S3250800DDC0B06880470446706880470146224686A003F0E4FF8C48FFF70BFA08B18BA400E02B
S3250800DDE08DA48F48FFF704FA08B18BA100E087A122468CA003F0D2FF287A08B191A200E066
S3250800DE0091A2E87908B191A100E091A1BDE8704090A003F0C3BF974C6068FAF7B6FC0246D3
S3250800DE200B4600E038E094A003F0B8FFE068FAF7ACFC02460B4695A003F0B0FF3068FAF7D3
S3250800DE40A4FCBDE8704002460B4696A003F0A6BF206F016B88471149343151F8201097A05F
S3250800DE6003F09CFFA87808B19AA200E09BA2687808B198A100E099A19AA003F08FFFFAF73C
S3250800DE8043FF28B99D48D0E900219DA003F086FFBDE8704000F04AB970BD00004007002001
S3250800DEA058000020CC060020902300200D0AA1AAA1AAA1AAA1AAA1AAA1AAA1AAA1AAA1AA5D
S3250800DEC0A1AAA1AAA1AAA1AAA1AAA1AAA1AAA1AAA1AAA1AA0D0A000041435F436861726767
S3250800DEE0696E67000D0A4443555F576F726B696E674D6F6465203C25733E0D0A00000000D5
S3250800DF005643555F576F726B696E674D6F6465203C25733E0D0A00006823002043686172CE
S3250800DF2067696E675F5374616765203C25733E09534F43203C25643E0D0A0000436F6E73EE
S3250800DF4074616E74566F6C7461676500436F6E7374616E7443757272656E7400436861727F
S3250800DF6067696E675F4D6F646520203C25733E0D0A00000044656D616E645F766F6C7461D3
S3250800DF806765203C25643E0944656D616E645F63757272656E74203C25643E0D0A00000096
S3250800DFA0040D00204F75747075745F766F6C74616765203C25643E094F75747075745F63C1
S3250800DFC0757272656E74203C25643E0D0A0000004368617267696E6743757272656E742033
S3250800DFE03C25643E0D0A000054656D7031202020203C25643E092047554E5F54454D5020E7
S3250800E0003C25643E0D0A0000A0090020446973636F6E6E65637400004F70656E0000000073
S3250800E020A809002044435F52656C6179203C25733E202041435F52656C6179203C25733E9A
S3250800E0400D0A00004343000043433200434331004350000043502D4343312020203C257368
S3250800E0603E092043432D4343322020203C25733E0D0A0000400C00204B4C33305F566F6C41
S3250800E08074203C25663E0D0A0000000053616D706C5F766F6C74616765202020203C25662D
S3250800E0A03E0D0A0043435F52206973202020202020202020203C25663E0D0A004F42435F3B
S3250800E0C047756E436F6E6E6563742020203C25733E0D0A004E4F5F4C6F636B004C6F636BA7
S3250800E0E0000000004856494C203C25733E204856494C5F32203C25733E0D0A00302400200C
S3250800E100456E7465722046616C7365536C6565702049646C6520636F756E74202564204DF2
S3250800E12041582069732025640D0A00002DE9F047DFF84880DFF848900025464618F805001B
S3250800E140B0B1FDF705FB3327B04600244FEA090618F8052016F83410914205D106EBC400BB
S3250800E160416808A003F01AFE641CE4B2BC42EFD36D1CEDB2052DE0D3BDE8F08730080020DE
S3250800E180AC7601084572726F7220436F646520496E466F2069732025732D25640D0A000094
S3250800E1A02DE9F041264C207860B10026254D01280DD0022827D003283FD0BDE8F04122A05E
S3250800E1C003F0ECBDFAF7A0FD80F0010014E008F0ADFC012798B1012813D002280DD11D4817
S3250800E1E006721D48FEF7F5FFFFF72CFB4FF4FA70FDF745F86F7302202070BDE8F08127700F
S3250800E200FBE72670F9E76068401C6060A97B012905D0052803D303206660207003E0012809
S3250800E22001D1FBF739FBFEF70BFE287B0028E4D0FFF754F96E606E73E3E7FFF781F8000030
S3250800E240380800203024002045525220536C6565700D0A009023002080090020F0B5284F2B
S3250800E260284B4FF496623878002403EBC0062649B6F802E005464FF0010C96450CD317E013
S3250800E28033F830E0964505D203EBC00EBEF802E0964504D8401CC0B20528F1D301E00528AB
S3250800E2A000D304204C700A7802BB81F800C018E033F830E096450DD816E000BF33F830E042
S3250800E2C0964505D203EBC00EBEF802E0964503D8401EC0B20028F1D10C704A7832B981F818
S3250800E2E001C0F2884A8001E04C700C704A8812B1521E4A80F0BD8542FCD03870F0BD00008E
S3250800E300940B002048730108D0000020F0B52948807A00EB80004200B2F5AF7F43D3264965
S3250800E320264B00240878012703EBC0060546B6F802C094450CD316E033F830C0944505D2AA
S3250800E34003EBC00CBCF802C0944504D8401CC0B20528F1D301E0052800D30420CC708B78C7
S3250800E360EBB98F7016E033F830C094450CD814E033F830C0944505D203EBC00CBCF802C02F
S3250800E380944503D8401EC0B20028F1D18C70CB782BB9CF70F3888B8001E0CC708C708B88ED
S3250800E3A013B15B1E8B80F0BD8542FCD0322AFAD90870F0BDD4350020940B00209878010872
S3250800E3C0034A516821F44041014351607047000000100240044A0029516901D0014300E06F
S3250800E3E0814351617047000000100240044A0029D16901D0014300E08143D161704700003D
S3250800E40000100240044A0029116901D0014300E0814311617047000000100240044A002900
S3250800E420916901D0014300E0814391617047000000100240014908607047000040044242EF
S3250800E440F0B52A4A51682A4B11F00C014FF00F0503D0042901D0082901D0036026E0516811
S3250800E460546805EA914104F480340D2901D0891C00E00621BCB1D46A14F4803FD46A04F00E
S3250800E4800F0404F101040AD0D66AD76AC6F30316761CB3FBF6F3C7F30327BF1C7B43B3FBE0
S3250800E4A0F4F34B43D9E7134B594301605168124C05EA1111635C0168D940416053680725CD
S3250800E4C005EA1323E35C21FA03F38360536805EAD323E35CD940C1605268032303EA92322C
S3250800E4E0231F9A5CB1FBF2F10161F0BD0010024000127A0000093D00FC040020024600208C
S3250800E50053090949012B0BD0022B0BD0D1F8241002F01F02012393400B4200D00120704734
S3250800E5200968F5E7096AF3E700100240014908607047000080044242014908607047000007
S3250800E5403C04424202490A6A02430A62704700000010024010B5084C44F22001A06B0842AB
S3250800E56001D1400605D52F20FDF73EF90020A06310BD012010BD0000040D002070B50D469A
S3250800E5800646002403E0305D02F0F4FB641CAC42F9DB70BD70B50D460646002403E0305DE5
S3250800E5A002F0E8FB641CAC42F9DB0D2002F0E2FB0A2002F0DFFB002403E0305D01F0B6FC0D
S3250800E5C0641CAC42F9DB70BD0248018841F0100101807047042800400248018821F0100110
S3250800E5E00180704704280040034800880249091F098840EA014070471C28004010B5012105
S3250800E6004FF0C050FFF7F2FE4FF400742046FFF799FF0120FFF790FF0120FEF779FFFAF7E7
S3250800E62052FC0120FFF782FF6120FFF767FF0028FAD02046FFF786FF0120FFF77DFF00F0B3
S3250800E64023F800F019F849F63F4000F005F8BDE8104000F011B8000000B50246FFF7B4FF91
S3250800E6600449C2F303400880081D02805DF804EBFFF7B2BF08280040024801888906FCD5CA
S3250800E68070470000042800400448018821F00801018001880907FCD570470000042800404C
S3250800E6A0114910B50120C1F89801FEF73BF99020FEF776F90020FEF773F9FEF755F9FEF7C4
S3250800E6C031F99120FEF76CF9FEF7ECF8074C2080FEF7E8F86080FEF747F96088218840EA86
S3250800E6E001202080208810BD008021428400002010B510B3416801B38168F1B10378184903
S3250800E700002200BF02EB420404EBC20401EB041424789C4211D0521CD2B2022AF2D30022BE
S3250800E72002EB420303EBC20301EB03131B78FF2B05D0521CD2B2022AF2D3002010BD02EB95
S3250800E740420303EBC20201EB0214014620222046F9F73BFD012084F85400024810BD000093
S3250800E76044130020D8000020704772B6704762B67047000070B5FDF769FEFDF7F3FD002231
S3250800E780012804D0022804D0032802D002E0012200E002220A4900230C78A24202D08B61CE
S3250800E7A00A7070BD4D78AA4201D18B6170BD8A69521C8A61022AF9D34C708870F5E7000034
S3250800E7C02000002070B50D460446FFF70DFF216809B1616802E04119C4E90001814201D895
S3250800E7E0012070BD002070BD00210160416001207047000070B50F4D0224B5F8410028B107
S3250800E800B5F8430010B10024204670BD0A483C210646FFF7D7FF0028F6D03046FFF7E4FF7E
S3250800E820B5F8410020B10A20FCF7DEFF0124EBE70920F9E7CC0600209C340020084810B51A
S3250800E840C0780324012807D040B10420FCF7BEFF00B10224204610BD0124FBE70024F9E771
S3250800E86090230020084810B500790324012807D040B10320FCF7AAFF00B10224204610BD48
S3250800E8800024FBE70124F9E7902300202DE9F04142780378284E02EB032295B2284A378A0E
S3250800E8A00024264B92F82220AF4207D11B7A8B423CD1C2B30A46811C22482EE0778AAF42E5
S3250800E8C008D15B7A8B4231D16AB30A46811C1D48133022E0F78BAF4208D1DB7B8B4225D194
S3250800E8E00AB30A46811C1748773016E0378CAF4208D11B7C8B4219D1AAB10A46811C1148E8
S3250800E9007B300AE0768CAE4212D15B7C8B420DD14AB10A46811C0B487F30F9F756FC284663
S3250800E920FCF7BAFC05E0FFE7332402E0132400E031242046BDE8F081FA780108E678010852
S3250800E940A84400204D3500202DE9FF4F8046604800248DB0B0F842201F46A146042A03D26F
S3250800E960132011B0BDE8F08FB8F8013098F800105DBA71238DF8003098F800308DF801301A
S3250800E98098F801308DF8023098F8023004268DF803304FF0050B4FF4017A012907D0032913
S3250800E9A05ED002297AD00179012974D03BE0B8F8011083464DBA04211046FCF723F918B1BF
S3250800E9C0A5F50070033812D0BBF842000421FCF719F908B155450AD0BBF842000521FCF7A8
S3250800E9E011F9010040F207202ED085422CD19BF82210584631B3A5F50075033D1BD0012D34
S3250800EA000AD0042D0BD198F80300012802D83149887001E04FF001098DF8049005262D4915
S3250800EA2001201C3988703E80324669460F98F9F7CCFB204695E70121C1734FF4FA71ABF88E
S3250800EA405410E9E7332441E0A5F50071033903D0554501D0854201D1132437E0312435E026
S3250800EA60B8F8011080464DBA04211046FCF7CAF830B35545F2D198F822000028E2D01548A1
S3250800EA801C38817841B1002181701348007A8DF8040011E002E016E0242417E080460421C6
S3250800EAA01046FCF7AFF858B15545D7D198F822000028C7D08DF804900526A7F800B0B3E76F
S3250800EAC05545CBD1C8E70021017112243E80B0E7A8440020300B0020D435002004494BF607
S3250800EAE05C200880091D4AF65520088070470000B06C00400CB500212E48019100910268A9
S3250800EB0042F4803202604FF6FF72036803F400330093019B5B1C0193009B13B9019B934240
S3250800EB20F3D10268920342D50121009122490A6842F010020A600A6822F003020A600A684A
S3250800EB4042F002020A604168416041684160416841F480614160C16A184A1140C162C16AE7
S3250800EB60174A1143C162016841F08061016001680901FCD5416821F47C114160416841F4C5
S3250800EB80E8114160016841F08071016001688901FCD5416821F003014160416841F00201E1
S3250800EBA041604168C1F381010229FAD10CBD00910CBD0000001002400020024000F0FEFF0D
S3250800EBC014080100FFF78ABF0A4810B50078072804D0094800698047022809D10748D0E9AC
S3250800EBE001100A30814203D2BDE81040FEF730BF10BD0000682300205800002030240020E7
S3250800EC00014908720120704798060020014908710120704798060020032803D0042801D038
S3250800EC20002070470149C8710120704798060020012802D008B100207047024988710120E6
S3250800EC407047000098060020024A002110440172704700009C230020012802D008B1002093
S3250800EC607047024948710120704700009806002070B5FEF787FD002818D0124C0020124DAA
S3250800EC80124E608380B200EB400005EB800041687068F9F7BEFA0028608B08D000EB400017
S3250800ECA005EB8000806800B18047012070BD401C80B260831328E5D305A003F06FF80020A5
S3250800ECC070BD00008C010020C873010894200020416E20756E7265636F676E697A65642038
S3250800ECE0434D4420210A00001FB51E48FEF780FA00B101208DF800001B48FEF779FA00B16B
S3250800ED0001208DF804001948FEF772FA00B101208DF808001648FEF76BFA00B101208DF80B
S3250800ED200C0069461348FCF76DFE00B10120124C01A9E0700F480C38FCF764FE00B1012065
S3250800ED4020710C4802A90C30FCF75CFE00B101206070084803A91830FCF754FE00B101208F
S3250800ED60A0701FBDA0090020A8090020E0090020E8090020E423002090230020F0B5CF2255
S3250800ED800270002343700C7884700126C27006714F78477191F802C080F806C00223C27175
S3250800EDA00372CB7843720B7983720324C27204734B79437304258273C5738B790374052617
S3250800EDC042748674CB79C3740627027547750B7A83754B7AC3754FF0070C027680F819C005
S3250800EDE0897A81761B20F0BD054951F8062F40F8022F4A6842600A890281897A81727047D7
S3250800EE00D8350020F0B5002382F8003003EBC30400EB4404647834B144EA03251478660054
S3250800EE20641C14708D535B1CDBB2122BEED3107800281DD0002317E000200EE001EB4005E8
S3250800EE4031F810606C88F7B204F0FF0C674502D96E8021F81040401CC0B21478E41A641EB7
S3250800EE608442EBDC5B1CDBB21078401E9842E3DCF0BD000010B5FAF759F888B1FCF7C6F8D6
S3250800EE8000280CD0FCF740F8002808D0084890F83800C00602D5FBF733FB18B1012010BDB1
S3250800EEA004A000E00EA002F079FF002010BD0000040D0020424D53205468652043686172C9
S3250800EEC067696E672050686173652053746F70732041626E6F726D616C6C790A0D000000ED
S3250800EEE0434353204E6F204368617267696E6720416C6C6F7765646E0D0000000C4881686B
S3250800EF00491C81604168491C416081684FF47A72B1FBF2F302FB1311012902D1C168491C99
S3250800EF20C1600178002901D101210170704700007C0100200C484FF47A710068B0FBF1F0D1
S3250800EF40B0F1807F0ED220F07F414FF0E020491E4161064AF02182F8141D002181610721D4
S3250800EF6001617047FEE700000C0000200FE000E010B5FDF737FEBDE810404FF41F72024988
S3250800EF80024804F0E7BA00002815002000F00108124810B5016841F0010101604168104A0F
S3250800EFA01140416001680F4A11400160016821F480210160416821F4FE014160016821F085
S3250800EFC0A05101604FF47F0181600021C162FFF791FD05494FF00060086010BD00100240F1
S3250800EFE00000FFF0FFFFF6FE08ED00E00C4810B500880B4A0021243A02F02EFE0848303802
S3250800F000C068F9F7C2FB02460B4606480649F9F707FBF9F7CDFBFCF711FD0449088110BD89
S3250800F020500000209A99999999991340400C002010B5084C0121204600F04BF8002807D029
S3250800F04000F0A4FE2046BDE81040012100F034B810BD0000000400407FB50C4605460121B3
S3250800F0600220FFF7C3F9ADF800400020ADF80450104CADF80600ADF802006946204600F0FD
S3250800F0803FF801221146204600F02FF81D208DF80C0001218DF80D1003208DF80E008DF867
S3250800F0A00F1003A8FEF76EF90121204600F007F87FBD000000040040C943018270470029B6
S3250800F0C0018802D041F0010101E021F001010180704702460020138A92890B4202EA01020C
S3250800F0E002D0002A00D001207047002A828901D00A4300E08A4382817047818570470000E7
S3250800F10030B502881B4B1C4C98420DD0A0420BD0B0F1804F08D0194DA84205D0184DA84274
S3250800F12002D0184DA84203D122F070054A882A43154DA84206D0154DA84203D022F44075FA
S3250800F140CA882A4302808A8882850A88028598420AD0A04208D00E4A904205D00D4A904298
S3250800F16002D00D4A904201D1097A01860121818230BD0000002C0140003401400004004072
S3250800F18000080040000C004000100040001400400040014000440140004801400A48002127
S3250800F1A0428D4AB10722C273027B521CD2B20273102A00D1017370470177C173C1720176A9
S3250800F1C04174808CFDF744BA540B002070B51B4C0125002025756076E07B01280AD1607A74
S3250800F1E0102807D1FCF709FFE07B012802D1607A102807D0207908B1E07818B1A078012802
S3250800F20006D007E096202086E5760220A07001E0607930B1607A20B1E07B042803D1E08B2E
S3250800F22008B900F0F3FAE07A012806D1E07B062803D1BDE8704000F0E9BA70BD540B0020D7
S3250800F2402DE9F041274CA078012849D0264F3879012802D1E07A012842D0FDF723FA20851F
S3250800F26020483830FDF7E4F91E4E00253836307800F0F001A173E584A18CA7F842103D710E
S3250800F280A178012700F00F00022901D100B9A770E07A012801D100F0B9FAA07B00281FD128
S3250800F2A03078124B00F00F01A184012009E000BFE28C16F800C003F802C0521C401CE28424
S3250800F2C0C0B28842F4D900F06BF938B1E77429466174A08CBDE8F041FDF7BAB90921F7E7CA
S3250800F2E0BDE8F081540B0020A8440020A438002070B5194C0026A07801281CD00125657586
S3250800F300FDF7D0F9208504F13800FDF791F904F13800A1780078022900F00F0001D100B95F
S3250800F320A570E07A012801D100F070FA0B4866776570057170BD607F401CC0B260770228A5
S3250800F340F8D301F02BFC00F035F866770448A670E673067070BD0000540B0020A8440020D9
S3250800F360F40B002010B5104C207868B104F1380041782171807828B17F2800D97F20401CCA
S3250800F380C0B200E0012060712079E0706079A0710020207200F09CFA207A10B10320E0733F
S3250800F3A010BD0420FBE70000540B002000487047A438002007480021C1738170C172C175F4
S3250800F3C001760175417541768176C1760177017481757047540B002010B5064CA07AFDF759
S3250800F3E087F904F13800FDF763F94620A0850120607610BD540B002070B5164C0026072858
S3250800F400E08301D8667201E0102060720125A5702684E07D012805D00C206074FDF738F982
S3250800F420A67070BD607A10B1102803D004E000F0B9FA01E000F06CFAE571A07AFDF758F962
S3250800F44004483830FDF734F9E5734620A085657670BD0000540B002010B500F0D3FBBDE837
S3250800F460104000F0D3B900000B48417B29B101290FD002290FD100F0A7B9C18CA1F602017E
S3250800F48049428186408D072801D300F0A9B800F02DB900F079B97047540B002070B51F4DEC
S3250800F4A0A5F138042978687801F00F0140EA0120A08440F60201608588420BD90D216174AC
S3250800F4C0FDF7C6F80220207400F042FA00202074E07370BD0828FCD300F062F8B8B1104B49
S3250800F4E00220E18C2A5C401C5A54628D491C521E6285C0B2E1840728F3D901252573A08C78
S3250800F500FCF77CFDE572BDE8704000F021BA09216174A08CBDE87040FDF79AB88C0B00207D
S3250800F520A438002070B50F4B0F4DA3F13804187800F00F01A184012006E0E28C1E5CAE5470
S3250800F540521C401CE284C0B28842F6D900F028F830B100216174A08CBDE87040FDF778B8D6
S3250800F5600921F7E78C0B0020A43800200A480A494FF000020078A1F1380110F0F0008873AE
S3250800F580CA84CA740549C87603D0102803D1FFF785BFFFF7C7BF70478C0B0020A844002036
S3250800F5A00E4A00201146937B098D43B1102B0ED0202B0FD0302B09D1032907D305E0928C55
S3250800F5C0002A03D0521C914200D3012070470829FCD3FAE7528D072AF9D2F3E7540B00201F
S3250800F5E0F0B51E481E4E0121838E1E4C00F1380C072B1ED2C18601220EE000BFC58C1CF816
S3250800F600027067556D1CC584458D6D1E4585C58E6D1C521CC586D2B29A42EFD9428D0AB966
S3250800F62086F8211041730822C27301760021C184F0BD0122C38C1CF80250521CE5545B1C7A
S3250800F640C384438DD2B25B1E4385072AF2D91804000CEDD186F82110F0BD0000540B002003
S3250800F660A8440020A438002070B51F4C608E38B3607D002836D00025657504F13806257732
S3250800F680307810F0F000A0731CD010281AD0202828D1FFF785FFE8B13078217B00F00F000C
S3250800F6A0884219D16573FFF7DFFE9620608601202077607B002815D1BDE87040FFF76EBD2A
S3250800F6C003200AE00620607400F050F8BDE87040FFF74CBF092000E004206074BDE8704031
S3250800F6E000F044B870BD0000540B0020F0B51C4801231C4D868E418D00F138048E4215D307
S3250800F700CEB2012109E0C28C675CAF54521CC284428D521E491C4285C9B2B142F3D9408D16
S3250800F720002802D1104880F82130F0BDC38601210CE0C28C675CAF54521CC284428D521E94
S3250800F7404285C28E521C491CC286C9B2B142F0D9022141730821C17303760021C184F0BD72
S3250800F760540B0020A4380020A844002010B5054C0146A08CFCF76CFF0020E073E0722076B2
S3250800F78010BD0000540B002030B50D48017E002914D10C4C00F13803C18E07290AD8C28C15
S3250800F7A05D5CA554521CC284428D521E4285491CC186F1E7002141730721C17330BD00002D
S3250800F7C0540B0020A438002070B50E48017E002917D190F82A1000F138040B4D491C09E000
S3250800F7E0C28CE65CAE54521CC284428D521E42855B1CC386C38E8B42F2D900214173072109
S3250800F800C17370BD540B0020A438002070B52C4C00212246E37B0320527D092B1CD2DFE89F
S3250800F82003F0050C10141C202A383C00002A13D06175BDE87040FFF799BEBDE8704000F0EE
S3250800F84075BABDE8704000F037BA00F041F8207A002801D10420E07370BDBDE8704000F08F
S3250800F860F3B9A179491EC9B2A1710129F4D8E0736079A07170BD227D01203AB12175A17608
S3250800F8800721E17396216186207770BDE18D49B170BDBDE87040FFF7E7BE638E13B132B15F
S3250800F8A061750B206074BDE87040FFF75FBFFFF7DBFD607B0028EBD1BDE87040FFF76EBCFA
S3250800F8C0540B002001490120C8757047540B00200E48017A29B1012915D0022915D100F002
S3250800F8E03DB90A4AC179383241F020011170018CA1F6020149428186C08B072801D300F042
S3250800F90079B800F0B7B800F001B97047540B002030B50D480D4CC18BC1F3032242F010036C
S3250800F92000F13802137051700221038CE55C55545B1C0384C38B491C5B1EC9B2C383072993
S3250800F940F3D90821817230BD540B0020A438002010B5134C142204F13801207C40F03000C5
S3250800F9600870002048708A7060840320A072CC220A54401CC0B20728FAD90820A0720020A0
S3250800F980FCF7BCFEA07AFCF7B3FE05483830FCF78FFE0620E0734620E0850120A07610BD71
S3250800F9A0540B0020F0B51149012001F13804CA8B227003460E4F08E00D8C401CC0B27E5DB5
S3250800F9C0E6546D1C5B1C0D84DBB215469342F3D96A1C8A72072807D8CC222254401CC0B203
S3250800F9E00728FAD908208872F0BD0000540B0020A43800202DE9F0411C4C1D4904F1380269
S3250800FA00A38E072B1AD20125E58628460CE0268C8F5D1754761C2684E68B761EE683E68E77
S3250800FA20761C401CE686C0B29842F0D925720025E575FCF7E4FA2584BDE8F0810120238CD3
S3250800FA40CD5C15545B1C2384E38B401C5B1EC0B2E3830728F3D90820A072FFF7BDFC0420C5
S3250800FA60E073BDE8F04100F0BBB80000540B0020A43800202DE9F041224C234B04F1380120
S3250800FA80A28EE58B4FF00100AA4220D3EDB201220BE0268C401CC0B29F5D8F54761C268451
S3250800FAA0E68B761E521CE683D2B2AA42F1D9A572CC2202E00A54401CC0B20728FAD90820E5
S3250800FAC0A072FFF789FC0420E073BDE8F081E08601200CE0258C5E5D0E546D1C2584E58B1B
S3250800FAE06D1EE583E58E6D1C401CE586C0B29042F0D9022020720025E575FCF780FA2584EC
S3250800FB00E3E70000540B0020A438002070B5114CE07D01281CD1104A04F13803E08E072876
S3250800FB200AD8218C555C1D54491C2184E18B491EE183401CE086F1E70820A072FFF74CFCB3
S3250800FB40002020720420E073BDE8704000F048B870BD0000540B0020A43800202DE9F0413A
S3250800FB60174CE07D012828D194F83600A17FC2B20844C1B2A17204F13803124E0BE0258C41
S3250800FB80521CD2B2775D1F546D1C2584E58B6D1EE583401CE086E08E8842F0D3CC20072AAF
S3250800FBA003D89854521CD2B2F9E70820A072FFF713FC002020720420E073BDE8F081000020
S3250800FBC0540B0020A438002010B5FCF761FD03480021C1738170C175017510BD540B0020FD
S3250800FBE00748C179491CC9B2C171102901D10021C1710179002902D0C178491EC170704701
S3250800FC00540B00200F48417E012903D1818D09B1491E8185817E012903D1C18D09B1491EA2
S3250800FC20C185C17E012903D1018E09B1491E0186017F012904D1418E002901D0491E418686
S3250800FC4070470000540B002070B51A4C0126A08DD0B1207DA17D084326D00025657625756A
S3250800FC60E08B98B1207908B1E078A8B16079B0B1012814D002281AD016D9A079A0F10100CA
S3250800FC80A0714FF0050013E0304600E028466074BDE87040FFF798BF2570022008E0FFF73F
S3250800FCA017FE207A08B1A67570BDA57570BD0320E07370BD540B002070B51B4C208EB0B182
S3250800FCC0607D00282FD0002004F138016075097801F0F002A273302A25D1E07601F00F05CB
S3250800FCE0FFF75EFC28B1032D05D305200EE002200CE009200AE0022D07D0012D0BD0002D55
S3250800FD0011D1BDE87040FFF72DBB08206074BDE87040FFF759BF07206074FFF755FF952067
S3250800FD2020860120E07670BD540B00200B490122888D68B1087D002809D000200875487666
S3250800FD404B7A43B1102B02D10A700220C87370474A74104600E04874FFF736BF540B002026
S3250800FD60094A29B192680068904204D8101A04E09168016003E0C0431044884201D30120D7
S3250800FD8070470020704700007C0100200D4810B5407B012815D03220FBF718FD002810D1E5
S3250800FDA02A20FBF713FD00280BD1074C206801880648FFF7A2F9206840688047206880683B
S3250800FDC0206010BD30240020CC3400200004004030B52C4C2078012852D12B490122C868E8
S3250800FDE0401CC8600A70002323700524B0FBF4F504FB1504002C43D1002841D00A24B0FB1A
S3250800FE00F4F504FB15044A7004B98A701424B0FBF4F504FB150404B9CA703224B0FBF4F59D
S3250800FE2004FB150404B90A716424B0FBF4F504FB150404B94A714FF4FA74B0FBF4F504FB74
S3250800FE40150404B98A714FF47A74B0FBF4F504FB150404B9CA7140F2DC54B0FBF4F504FBF9
S3250800FE60150404B90A724FF4FA64B0FBF4F504FB150404B94A7241F27072904200D3CB6077
S3250800FE8030BD00007C010020181500200FB5124801880A2901D3002101800288009900EB1F
S3250800FEA00212516002889DF8041000EB0212117202889DF80D1000EB021251740188DDF85C
S3250800FEC0052000EB011141F8092FDDF809204A600188491C01800FBDA840002070B5104819
S3250800FEE0006800281BD1FAF76DFD002817D00D4C21886088814212D000250A2800D3658070
S3250800FF00608804EB0010001D0FC801F02AF906480121817080F82A506088401C608070BD40
S3250800FF20500B0020A8400020A844002010B5044C0146204601F0A8F820880006FCD510BD85
S3250800FF40004C00402DE9F041384C40F225573946204601F007F8364D002690B1204601F078
S3250800FF608FF8C1B2A88AC82804D2324A1154401CA88200E0AE820A292FD03946204600F003
S3250800FF80DAFF40F224473946204600F0EBFF38B1AE82204601F074F83946204600F0CBFFA3
S3250800FFA040F227752946204600F0DCFF18B12946204600F0C0FF40F226652946204600F0F6
S3250800FFC0D1FF18B12946204600F0B5FF0821204600F0C1FF012805D00BE0FEF749FEAE826D
S3250800FFE0BDE8F0810821204600F0A2FF204601F047F80421204600F0AEFF012806D10421DA
S32508010000204600F095FF204601F03AF80221204600F0A1FF0128E3D10221204600F088FF68
S325080100202046BDE8F04101F02BB80000004C00408C0100209A1D002070B5314D40F2255641
S325080100403146284600F08EFF2E4C98B1284601F017F8C2B2208B0021C82804D22A4B1A5415
S32508010060401C208300E02183E182E1703146284600F061FF40F224463146284600F072FF23
S3250801008040B1284600F0FCFF0120E0703146284600F051FF40F2266631462C46284600F06C
S325080100A061FF18B13146204600F045FF0821204600F051FF012806D10821204600F038FF72
S325080100C0204600F0DDFF0421204600F044FF012806D10421204600F02BFF204600F0D0FF57
S325080100E00221204600F037FF012808D10221204600F01EFF2046BDE8704000F0C1BF70BD52
S32508010100005000408C010020621E002010B5094C207F00280DD0E07F10280AD1A07F00F0B4
S3250801012037FA00202077BDE81040FF210248F8F765B810BDA8440020A438002010B5074C70
S32508010140207F002808D0E07F112805D104F12B0000F0AAFA0020207710BD0000A84400203F
S3250801016010B50A4C207F00280FD0E07F14280CD1032104F12B0000F0E7FA00202077BDE8C6
S325080101801040FF210248F8F739B810BDA8440020A438002010B5064C207F002806D0E07FCE
S325080101A0192803D100F0F6F80020207710BD0000A844002010B5064C207F002806D0E07F9A
S325080101C0222803D100F04CF90020207710BD0000A844002070B5104C207F00280ED0E07FA8
S325080101E027280BD194F82B0000250C4A04F12B01022804D0012000F0E1FA257770BD02209D
S3250801020000F0DCFA05482577801F84F8215040F8065F456070BD0000A8440020BA0B002034
S3250801022010B50A4C207F00280FD0E07F28280CD1022104F12B0000F0B7FB00202077BDE821
S325080102401040FF210248F7F7D9BF10BDA8440020A438002010B5094C207F00280DD0E07F5D
S325080102602E280AD106480088401E81B2054800F021F9002084F82100207710BDA844002053
S325080102807A0B0020A538002010B50A4C207F00280FD0E07F31280CD1032104F12B0000F023
S325080102A0F3FB00202077BDE81040FF210248F7F7A5BF10BDA8440020A438002010B5074CEC
S325080102C0207F002808D0E07F3E2805D104F12B0000F028F90020207710BD0000A844002014
S325080102E010B50A4C207F00280FD0E07F85280CD1012104F12B0000F0FDFB00202077BDE8BF
S325080103001040FF210248F7F779BF10BDA8440020A4380020044A81781170C078491C117033
S32508010320801C507070470000BA0B002006480178012908D141780C2903D20C3050F8210084
S325080103400047002101707047B80B002002490120087000F023BC0000B80B0020024900201A
S32508010360087000F01BBC0000B80B002070470000074801214177002180F8221000F8061F84
S32508010380C17241878177C17780F8211070470000A844002070B52F484178012959D91921CC
S325080103A001702D4C00214170B4F8420002281BD394F82B0004F12B0600F07F050B2D3DD2D4
S325080103C0DFE805F03C060627143C143C3C3C27002846FAF705FC80B3B4F8420003211FE000
S325080103E01E49FCF7AFF931E013212CE02846FAF7F7FB10B3B4F842000621FAF703FC00285A
S32508010400F2D0324629461548FBF700FD0328E7D811E02846FAF7E4FB78B1B4F84200022185
S32508010420FAF7F0FB0028DFD0324629460B48FBF7EDFC0028D4D1312101E0FFE71221207933
S32508010440012803D111B11920FCF760F90A20A4F8460070BD0E0C0020A8440020084700205B
S32508010460114810B5407801281DD9104C0321B4F84200FAF7C7FB78B10D48FBF74BFD032874
S3250801048003D30B49FCF75EF90AE02079012807D100202071312100E013212220FCF736F9DA
S325080104A01E20A4F8460010BD0E0C0020A84400200847002070B5064617480D464078012887
S325080104C028D9164C2079012824D1607F00220321FAF76AFBB8B1032D01D2132114E0AD1E19
S325080104E0A9B23046FEF7D2F908B101460CE00C486E2101703178417071788170014603207E
S32508010500FCF720F903E07F212E20FCF7FFF82820A4F8460070BD00000E0C0020A844002068
S325080105200847002070B5054616484078012827D9154C0221B4F84200FAF764FBC8B12978B2
S3250801054011F07F0F03D0207901280ED015E00846FAF752FB88B10D487E2101702978417019
S3250801056001460220FCF7EEF807E000202071122100E013213E20FCF7C9F80A20A4F846002D
S3250801058070BD00000E0C0020A8440020084700202DE9F04707464148417801297BD91021DF
S325080105A001703F4C002580464570B4F842000221FAF728FB002865D007F07F06012E07D08C
S325080105C0022E05D0032E03D02079012856D05DE0607F4FF00109032804D001281AD002287A
S325080105E01FD019E0022E17D1207901284ED1FAF70FFB68B1E07B58B16677FEF7E3FA84F868
S325080106000C90C82084F8009084F8200078213AE0222138E0022E06D0032E0CD0012E07D078
S3250801062009E0032EFAD1207901282FD17E212AE0FCF7D6FAE5736677A4F8405084F8225049
S32508010640A5716574032E05D084F8245084F8255084F827503846FAF7CFFAB8B11148502157
S325080106600170477085703221C17080F80490F421417106200B49FCF765F807E0257112217D
S3250801068001E008E013211020FCF740F80A20A8F80400A4F84600BDE8F08700000E0C0020ED
S325080106A0A8440020084700202DE9F04107462248417801293ED911210170002545701E21FC
S325080106C01E4C81800221B4F84200FAF79BFA50B3387800F07F00FAF77BFAF0B1FAF798FA5D
S325080106E0C8B13878FAF788FA154E38B1512030703878707031460220FCF724F811480179E7
S32508010700012902D105713570757001202070C82084F820000BE0222106E02079012806D1EB
S325080107202571122100E013211120FBF7EFFF0A20A4F84600BDE8F0810E0C0020A844002054
S32508010740084700207044002070B519494A78012A2CD914220A701E228A8001784278090494
S32508010760807801EB0221134C0D180421B4F84200FAF748FA98B16FF07F40854208D1FAF7A1
S3250801078049FA0D49542008700120FBF7DBFF0AE02079012807D100202071312100E013213D
S325080107A01420FBF7B3FF0A20A4F8460070BD00000E0C0020A8440020084700202DE9F05FFF
S325080107C0DFF8D8A1002490469AF801000E46012876D973480179012972D181460122407F16
S325080107E01146FAF7E1F900287ED0307800254FF0010BAAF10A07012807D002283FD0B9F8A4
S325080108004200022871D2132451E03D70A8464C46B9F842000221FAF7F5F90028F3D0E0784D
S32508010820012809D05F4D672028703078687094F82200012802D004E0372438E0A07901281A
S3250801084002D0607C18B10CE0C5F8028009E053480938FBF7C3FA84F811B0D7F80100C5F8A9
S32508010860020087F800B084F806B067218AF800108AF801804B490620FBF764FF1BE089F85E
S325080108801150B9F842000621FAF7BCF90028BAD099F82810032906D8387810B1012813D026
S325080108A013E0032900D33624387858B11CB121462720FBF72BFF1E20AAF80400A9F84600C2
S325080108C0BDE8F09F2424F2E73D70364C334904222560A58009392046F7F7B4FC88B3307810
S325080108E02E4A401EC0B201E056E053E0521F111FFBF71EFA20B1122447F8015FBD80D6E70C
S32508010900717888F80010B17888F80110F17888F80210317988F80310204940460422491FE0
S32508010920F7F790FC002848460CD090F82810FF2902D2491C80F82810C9B202291BD83524D9
S32508010940DAE725E080F8285067212170327862703278022A0DD0022280F823208AF8001019
S325080109608AF8015089F822B00E490220FBF7EAFE03E00122F0E7032903D047F8015FBD8037
S3250801098099E736240A2180F8291089F803B0B3E72424B1E712248AE77F2488E70E0C0020F1
S325080109A0A8440020084700202DE9F041334F0646682038703248417801295CD9282101701C
S325080109C01E21304C81800122607F1146FAF7ECF80025C0B3B4F842000321FAF713F998B32C
S325080109E0FAF716F988B3307810F07F01707805D0032903D0207901282BD039E0012805D0F5
S32508010A00032803D02079012820D031E011B1032907D00DE0012884F8245009D084F8255071
S32508010A2006E00121012884F8241001D084F825103078FAF7E1F8D8B1307878700F4902203F
S32508010A40FBF780FE14E00BE008E005E0257131210BE02571122108E0222106E0132104E0A6
S32508010A602079012804D125717F212820FBF74EFE0A20A4F84600BDE8F08100000847002083
S32508010A800E0C0020A8440020F8B50646164A0020ADF8000050780D46012823D931201070D2
S32508010AA0124C1E209080207901281BD10122607F1146FAF779F840B16B460D4A2946304634
S32508010AC0FDF742FF010001D104E07F213120FBF71DFE04E00649BDF80000FBF733FE0A20E8
S32508010AE0A4F84600F8BD00000E0C0020A84400200847002070B5054625484178012946D9BC
S32508010B00852101701E21234C81800122607F1146FAF74AF8002670B3B4F842000221FAF729
S32508010B2071F830B3FAF774F850B1287800F07F0001280BD0022805D02079012816D023E03F
S32508010B4022211EE0012084F8270001E084F827602878FAF751F8B8B10F48C521017029780B
S32508010B60417001460220FBF7EDFD0DE02671122107E0132105E0FFE72079012804D12671A5
S32508010B807F218520FBF7C2FD0A20A4F8460070BD0E0C0020A84400200847002004480021F5
S32508010BA0022201704270012282708180704700000E0C002010B5084C207F00280BD0E07FBE
S32508010BC000F00EF800202077E077BDE81040FF210248F7F713BB10BDA8440020A438002012
S32508010BE0084910B5497801290BD9074C2179012904D1002121711121FBF788FD0A20A4F8F3
S32508010C00460010BD0E0C0020A84400202DE9F0411446054669B1092927D13348017800291F
S32508010C2023D000210170BDE8F041FF212F48F7F7E5BA2F4802274178012906D0022914D1BD
S32508010C4021782C4E102923D025E005460178207801F1400282420AD12046272904D14178CE
S32508010C60012901D1FFF756FB6F70BDE8F0817F28FBD160788142F8D1A078782804D0FFF7D4
S32508010C806DFB03206870F0E71E20A8800420F9E747706078B0772178174B184AF177002006
S32508010CA01F5C8F4208D1342901D0362902D11449098829B9507003E0401CC0B20C28EFD369
S32508010CC00C2801D10B2050700A4814212B300746F7F794FA1422611C3846F7F776FA0120B9
S32508010CE03077A6F84250C0E7550B0020A43800200E0C0020A844002056790108B80B0020EA
S32508010D007E0B002001490120487070470E0C002070B5154C40F22551204600F023F900283F
S32508010D200ED0204600F0ACF9C2B2104881890B0406D44C044FF0000306D50A2A01D0838196
S32508010D4070BD41F400410DE00D2A09D0C1F30D04074D491C89B22A558181C729EFD870BDC6
S32508010D6041F48041818170BD003801408C0100200C1B002010B5044C0146204600F084F9A3
S32508010D8020880006FCD510BD0044004070B5304C40F225563146204600F0E4F82D4D88B1CA
S32508010DA0204600F06DF9EA89C0B2FE2A04D22A498854521CEA8101E00020E8813146204616
S32508010DC000F0B9F840F224463146204600F0CAF840B1204600F054F90120687031462046CE
S32508010DE000F0A9F840F226652946204600F0BAF818B12946204600F09EF80821204600F07C
S32508010E00AAF8012806D10821204600F091F8204600F036F90421204600F09DF8012806D184
S32508010E200421204600F084F8204600F029F90221204600F090F8012808D10221204600F0B8
S32508010E4077F82046BDE8704000F01AB970BD0000004400408C010020D41B002070B5314D86
S32508010E6040F225563146284600F07CF82E4C98B1284600F005F9C2B2608A0021C82804D209
S32508010E802A4B1A54401C608200E061822182A1703146284600F04FF840F22446314628460E
S32508010EA000F060F840B1284600F0EAF80120A0703146284600F03FF840F2266631462C46C6
S32508010EC0284600F04FF818B13146204600F033F80821204600F03FF8012806D10821204658
S32508010EE000F026F8204600F0CBF80421204600F032F8012806D10421204600F019F8204625
S32508010F0000F0BEF80221204600F025F8012808D10221204600F00CF82046BDE8704000F05C
S32508010F20AFB870BD004800408C010020D21C0020C943018070470A0A01219140C9430180F3
S32508010F4070470029818902D041F4005101E021F40051818170470246002012880A4200D022
S32508010F600120704730B501F01F0201240025C1F3421304FA02F2012B0FD0022B0FD0838A2A
S32508010F804FEA11210088134204FA01F400EA040001D000B10125284630BD8389F0E7038AA6
S32508010FA0EEE710B5C1F3421301F01F040121A140012B07D0022B07D01430002A026805D0B4
S32508010FC00A4304E00C30F8E71030F6E78A43026010BD000030B50446008A85B00D464CF61A
S32508010FE0FF710840E98801432182A1894EF6F3100140A8882A8910436A890A431043A08136
S32508011000A08A4FF6FF410840A9890143A1826846FDF716FA1948844201D1039800E0029871
S32508011020A189090400EBC00101EB0010296801D5490000E08900B0FBF1F06422B0FBF2F109
S3250801104009010B096FF018056B4300EB8300A3891D044FF0320306D503EBC000B0FBF2F0F4
S3250801106000F0070005E003EB0010B0FBF2F000F00F000843208105B030BD000000380140F4
S325080110808088C0F308007047C1F308018180704710B500F02BF9BDE81040FDF737B900F0B0
S325080110A04DBA000004480088034A0449121F128842EA0040C8607047BC6C0040940B00206F
S325080110C002F0E5BE02F01CBF0A484FF0E022816819B99169084B594381609169826843F26E
S325080110E0856311441A44826088B202EB820140EA01407047940B00200DE37A0570470000B3
S32508011100034900200978C90700D0012070470000300B0020034900200978890700D501208D
S3250801112070470000300B002001460020A1F5E062B43A00D1012070470FB41FB50DF12301FF
S32508011140069800909DF822208DF804200DF10500F7F73BF89DE80F0000F03EFA1FBC5DF8C2
S3250801116014FB0FB585B000208DF808009DF8182005998DF80A2000918DF809000DF119015A
S325080111800DF10B00F7F721F8684602F0B3FC09B000BD0000074810B54178002909D1012179
S325080111A04170FCF751F9F9F755FFBDE81040FAF715B810BD940B002010B52A48284CC168DB
S325080111C0E2792948F7F701F82748227827A16B38F6F7FBFF2448627828A15D38F6F7F5FF6D
S325080111E02148A27828A15138F6F7EFFF1E48227928A12B38F6F7E9FF1B48E27828A145382B
S32508011200F6F7E3FF184862792CA12138F6F7DDFF1548A2792CA11738F6F7D7FF1248A27AF9
S325080112202FA15F30F6F7D1FF0F48217A0A30F6F7E5FF0D4800216B3800F8E81F41708C2110
S325080112400171A02141711421017250214172132101738821417319210174417410BD000098
S32508011260E6780108940B002043350020323130393134302D535A303100000000383932362C
S32508011280202020202020000044435520202020202020000048573A312E302E4300000000EA
S325080112A053573A312E30302E435F3234303230345F383932365F30300000000078787878A9
S325080112C0787878780000000078787878787878787878787878787878787878787800000047
S325080112E05232583030303031000000002DE9F05F644CDFF894B1654920785D4640F00100C7
S325080113002070DBF80400F7F702F8F7F72AFADFF880A1A0729AF8100060725E48808F010A1F
S32508011320E1722073E868F7F71CFA010A6173A07359480126022700780025DFF860910728ED
S3250801134066D0D9F810008047022863D0E573DFF8508198F8030001285ED000285ED00420DF
S32508011360FAF734FA00B1677498F80400012857D0002857D00320FAF729FA00B127744F4668
S325080113804849D9F80000F6F7C2FFF7F7EAF9010AA174E0749AF80E00C8B3002020750120F8
S325080113A0FAF714FA217860F3041121F0E00020703020FAF70BFA617860F300016170312008
S325080113C0FAF704FA617860F3410161700320FAF7FDF9617860F3820161700320FAF7F6F943
S325080113E0617860F3C30161700420FAF7EFF9617860F3041161700420FAF7E8F961784646B3
S3250801140060F34511617098F8010088B90EE00BE0E6739CE7E7739AE76574A5E76674A3E718
S325080114202674ACE72574AAE70120B7E7B07810B141F0400001E021F0400020F0800060709B
S32508011440A570DBF80C00F7F78CF9A0803078A07178688047E0711448257200780228207818
S3250801146003D240F00200207006E020F00200207002D940F0040001E000F0FB002070BDE82E
S32508011480F09F0000D4350020400C00200000204130240020CC06002068230020580000202F
S325080114A09023002000401C46940B00200848094910F8EC2FCA7042780A714279037902EB91
S325080114C00322CA80427A007A02EB002008817047D8340020300B002030B5164885B00168A3
S325080114E0001D0068814223D01249134A10390024086120464FEA0D0300EBC00102EB41018A
S32508011500097B092903D1411C1955641CE4B2401CC0B21228F0D3074812210C3084720B3097
S325080115200546F6F76BFE224669462846F6F74DFE05B030BD240B0020EC3500202DE9F041C5
S32508011540214C0127207820B9FFF736FEFEF710FF27701E4D0026287890B195F8200020B1C1
S32508011560401E85F82000BDE8F08119482E700168184A01F4E06111430160BFF34F8FFEE721
S325080115806088401C80B26080022807D36680FEF7DDFEEF71EE7600F055F8E680A088401C41
S325080115A00004000CA08004D0A680FEF7BFFEFBF76DF8FEF793FCFAF793FFF9F78FFABDE8C4
S325080115C0F041FEF7D3BE0000AC0B0020A84400200CED00E00400FA050FB40098A0F5E06155
S325080115E0DF3907D0A0F5E061343903D080B204B000F04CB812480188322901D30021018049
S325080116000288009900EB0212516002889DF8041000EB0212117202889DF80D1000EB0212F8
S3250801162051740188DDF8052000EB011141F8092FDDF809204A600188491C018004B0704763
S325080116404C4100202DE9F0410D4C00270D4E0E4D10E0322800D367806088307004EB0010C6
S32508011660001D0FC8FCF724FA6088401C60802868401C2860218860888142EAD1BDE8F08199
S325080116804C410020A40B0020A80B00200D4910B50978C90710D00B4900230839A1F114043E
S325080116A00A68B0F5827F08D0A0F58070113803D122F002000860238110BD22F00100086021
S325080116C0E38010BD300B00202DE9FE4F15460E460746FBF787FADFF8ACC2AB4C002F63D000
S325080116E0012F7DD19CF80800E246002878D13078F178727840EA0160B178090441EA02211E
S3250801170008436061F7F796FCFBF76CFA2A469FA0616900F043FBD4E9050181427ED0A0615A
S32508011720E169A5F10D0901EB0903C3F30A02D90A9CA0E36100F032FBFAF7FEF8218CE0698D
S32508011740DFF890B2B1EBD02F0BD0C10A5844C70A2184FF023946A0A000F020FB3846FAF7D4
S3250801176069F84FEAE97109EB9170C0F38708371DA807B0F1804F0CD09EA000F00FFB70191F
S325080117800322FF210938F6F732FD08F1010000F0FF087D480024426A02EB0B010091C1695E
S325080117A04FF0010B41627CE03579257072796270F088317A40BA000440EA0123707A034331
S325080117C0636071892181307BF77B96F80D8040EA0760B77B3F0447EA08273843E06000E062
S325080117E056E0378A27824FF0FF36A6610026E6614FF6FF786662A4F820808CF80860CDE9F0
S3250801180000100297294681A000F0C8FA2089228AE1688DE807006278217800E0ADE08A4802
S32508011820636800F0BBFABDE8FE4FF7F735BC002557F824100098FAF755F8042808D06D1C4D
S32508011840EDB2032DF4D381A0009900F0A7FA1DE00098006801901CB1A8F10100844206DBFC
S32508011860DDE9001357F8242081A000F097FA57F82410019881420DD085A000F08FFADDE92B
S32508011880001357F824207AA000F088FA8AF808B0BDE8FE8F0098001D0090032D03D2641CD1
S325080118A0E4B24445C3D3FBF79DF91FFA89F15546BAF82C20301DF7F777FC334CA88502460E
S325080118C021897CA000F06AFAFBF78CF9E1686069884250D12089AA8D904204D0BDE8FE4FF3
S325080118E07DA000F05BBA002785A000F057FA8D4E3046F9F79FFFDFF8308230464146F9F7D5
S32508011900F1FF042807D07F1CFFB2032FF5D3314686A000F043FA376831463B46424654A0A2
S3250801192000F03CFA47451AD17E4F00263F1D38466168F9F7D7FF042807D0761CF6B2032E31
S32508011940F5D3394682A000F029FA3E683946334689A0626800F022FA6068B04202D085F856
S3250801196008B095E7FBF73EF9F7F764FB8BA000F015FAFBF74DFDF9F791FFBDE8FE4FFBF7E4
S3250801198031B900008C010020E41A00200A0D43757272204261673A25642C206C656E202513
S325080119A0640A0D0057726974652D616464723A20736563746F722025642C2C6F66667365CC
S325080119C074202564202C7265636C656E202530640D0A000000600208343443757272204553
S325080119E0726173652D2D616464723A202530780D0A0000000A0D6C6173742D2D2D2D2D62EC
S32508011A006167212121212121210A0D000D0A3636365570642D2D747970653A2564202C766E
S32508011A2065723A25642C54627974653A25642C204372633A25642C5061673A25642C506CF0
S32508011A40656E3A25640D0A006479010821323221212121212121212157726974652D466157
S32508011A60696C2D616464723A202530780D0A000061646472202530782C2C57726974652071
S32508011A802530782C2C72656164202530780D0A000A0D207265616476616C20213D205570F9
S32508011AA064646174615B695D2921212121210A0D00000000313232557064486561642E466F
S32508011AC0696C654372633D2530782C544372633D2530780D0A000000557064486561642E19
S32508011AE046696C6543726320213D2054437263202121212072657475726E210D0A000000BA
S32508011B002121217570642D696E666F21212057726974652D746F74706167202564200D0A28
S32508011B2000000000005802084433221155706444617461466C6167212057726974652D46AE
S32508011B4061696C2D616464723A202530780D0A002121217570642D696E666F21212057728A
S32508011B606974652D4661696C2D616464723A202530780D0A00000000316164647220253024
S32508011B80782C2C5772697465202530782C2C72656164202530780D0A00000000323275702D
S32508011BA0642D616C6C207772697465204F4F4B4B212172657374617274212121212121217F
S32508011BC0212121210D0A000030B50D46094CC1B041F20D01A4F8051001462A46E01DF6F7CA
S32508011BE0F4FA658040AA69462046F9F7BBFA41B030BD00002A1F0020FEE7000070B50E4DB3
S32508011C000224286F816A884730B1286F816A884700B10024204670BD084805210546FCF7F0
S32508011C20D1FD0028F6D02620F9F7DEFD2846FCF7DBFD0124EEE70000CC0600206C340020E3
S32508011C4010B50C46801AF6F771FD2146F6F791FBF6F787FD80B210BD2DE9F041194D01EB80
S32508011C604106294601EB8604904615F8262061880027CAB199B11420B1FBF0F06080F6F79E
S32508011C8063FD4FF06632104BF6F758FC6FF00B02F6F735FDF6F78CFDA060C8F800006780BA
S32508011CA005F82670BDE8F08122790844521CD2B222716080142AF5D1012005F82600277140
S32508011CC0F0E70000500C002066660A4010B50121CC022046FCF796FB2046BDE81040002171
S32508011CE0FCF790BB07490020086007490878401CC0B208701E2803D802497F2008390860F5
S32508011D0070470000082C00407801002043E0322100BF00BF00BF00BF00BF00BF00BF00BF82
S32508011D2000BF00BF00BF00BF00BF00BF00BF00BF00BF00BF00BF00BF00BF00BF00BF00BFA4
S32508011D4000BF00BF00BF00BF00BF00BF00BF00BF00BF00BF00BF00BF00BF00BF00BF00BF84
S32508011D6000BF00BF00BF00BF00BF00BF00BF00BF00BF00BF00BF00BF00BF00BF00BF00BF64
S32508011D8000BF00BF00BF00BF00BF491E11F0FF01BED1401EC0B20028B9D170470FB4054B36
S32508011DA010B503A9044A029800F044F910BC5DF814FB0000F13F0108F40400200FB4084BF7
S32508011DC010B504A902AA039800F034F9044602A9002000F0B2FC204610BC5DF814FB0000D5
S32508011DE03B27010830B528B1144C031F002021680A4605E0084630BD9A4203D81046526849
S32508011E00002AF9D1002800D041680BD00468A3EB0005A54204D11B681C440346046002E016
S32508011E20436000E023603AB11C68D51AA54203D115682C441C6052685A6030BD140C00206A
S32508011E402DE9F04782460F4C10480D4E0E4F001B4FF0000820F007054FF0010900221146B3
S32508011E60504602F0CDFD002802D1306810B10020BDE8F0873C60C4E90058C6F80090EDE7AE
S32508011E80180C00208C470020140C00208867002002E008C8121F08C1002AFAD1704770479E
S32508011EA0002001E001C1121F002AFBD1704700002DE9FF5F82B00021DDE90430020DDDF8CD
S32508011EC040B0034318D044F61050A2F2FF3242431514119801281FD0A5EB0B00401C5FEAC7
S32508011EE0000A4FF000064E4FDFF83891B046504615D5CAF1000413E0119801244AA301283B
S32508011F0001D16FEA0B010298119AC0E90031C0E9024206B0BDE8F09FCBF10000DFE70446B9
S32508011F200021404A491842EB0450CDE9001012E0E00707D032463B4640464946F6F7FEFA9C
S32508011F408046894632463B4610461946F6F7F6FA06460F466410002CEAD1DDE90401DDE9C5
S32508011F600023BAF1000F06DAF6F7E8FA42464B46F6F7E4FA05E0F6F753FB42464B46F6F7BC
S32508011F804FFB04460E460022284BF6F747FD03D84FF0FF30014607E00022254B204631469E
S32508011FA0F6F725FAF6F721FD102409E0002C0ADB0A220023F6F742FC039B30321A55641E62
S32508011FC050EA0102F2D1641C039AC4F111031444119A012A03D0012208430DD10AE008438A
S32508011FE004D000204FF0110B119072E7A3EB0B056D1E0DE05B4504DD4FF0000205F10105B5
S3250801200004E003DA4FF00002A5F10105002AECD002981199C0E90231C0E9004579E70000BF
S32508012020000014400000F03F300000000000F0430000E03F2DE9FF4F95B09A4688460646E9
S325080120400025EEE1252877D100242746F94A0121039400E0044316F8013F203B01FA03F09D
S325080120601042F7D130782A2811D06FF02F033078A0F13002092A16D8039A44F0020402EB7B
S32508012080820203EB42021044761C0390EFE758F8042B0392002A03DA504244F40054039060
S325080120A044F00204761C30782E2816D116F8010F44F004042A280DD06FF02F023078A0F10E
S325080120C03003092B09D807EB870302EB4303C718761CF3E758F8047B761C30786C280FD033
S325080120E006DC4C2817D068280DD06A2814D104E0742810D07A280FD10DE044F400140AE0AB
S3250801210044F4801401E044F440147278824202D104F58014761C761C307866280BD013DC45
S32508012120582877D009DC002875D04528F6D04628F4D047281AD193E118E0632835D0642830
S3250801214079D0652812D18BE1702873D008DC6728F1D069286FD06E280DD06F2806D1ACE0FF
S3250801216073282CD0752874D0782853D05246179990476D1C54E1C4F30250022809D0032801
S325080121800DD0D8F8001004280DD00D6008F1040846E1D8F80010EA17C1E90052F6E7D8F847
S325080121A000100D80F2E70D70F0E718F8041B8DF8001000208DF80100EB46012003E058F857
S325080121C004BB4FF0FF3061074FF0000102D40DE009F101018946B9420FDA8145F8DB1BF8FD
S325080121E009100029F4D108E009F1010189468142FADB1BF809100029F6D103985346A0EBA3
S32508012200090721463846179A00F080FA284400EB090507E044E008E10DE01BF8010B5246A2
S3250801222017999047B9F10109F7D2534621463846179AF2E039E00A21C4F302524FF0000BF1
S325080122400091022A06D058F8040BC117032A09D00AE023E008F1070020F00702F2E80201BC
S32508012260904605E000B2C117042A01D140B2C117002906DA0A460021404261EB02012D22A6
S3250801228002E0220504D52B228DF80420012203E0E20701D02022F7E7914657E00A2100E05E
S325080122A010214FF0000B00910BE010214FF0000B44F004040827009103E008204FF0000B4C
S325080122C00090C4F30252022A05D058F8040B0021032A08D008E008F1070020F00702F2E8F3
S325080122E00201904603E080B2042A00D1C0B24FF0000922072AD53278702A07D0DDF800C050
S325080123008CF0100C5CEA0B0C05D00EE040228DF80420012208E050EA010306D030238DF8F4
S3250801232004308DF8052002229146009B83F0080353EA0B030AD150EA010201D1620705D524
S3250801234030228DF804204FF001097F1E3278582A04D039A20C920CAA02920BE03BA2F9E722
S325080123605B46009AF6F76AFA0C9B9B5C029A521E0292137050EA0102F2D1029804A9081A98
S3250801238000F1200B600702D524F4803400E001275F4502DDA7EB0B0000E0002000EB0B01E9
S325080123A0009003984944401A0390E00306D453462146179A039800F0A9F90544002706E078
S325080123C001A85246C05D179990476D1C7F1C4F45F6DBE0030CD553462146179A039800F080
S325080123E095F9054404E030205246179990476D1C0099481E00900029F5DC08E00298029975
S3250801240052460078491C0291179990476D1CBBF10001ABF1010BF1DC5BE100F065F90544A0
S32508012420761C307800287FF40DAE19B02846BDE8F08F0000092801003031323334353637D4
S32508012440383961626364656600000000303132333435363738394142434445460000000005
S32508012460600700D4062708F1070020F00700F0E80223804603F0004C5FEA0C0001D097A06F
S3250801248009E0200501D596A005E0E00701D095A001E0AFF24C001390307823F00043652845
S325080124A00CD006DC452809D046281DD047287FD13BE0662818D067287AD136E00021112F0D
S325080124C001DB112000E0781CCDE9000104A90CA8FFF7EEFCDDE90D010C9A4FF0000B07F1B8
S325080124E00109109200914EE04FF000400097CDE9011004A90CA8FFF7DBFCDDE90D020C9BDB
S325080125000F994FF0000B91461093009211B9791C00EB0109B7EB090003D4C0F1FF3B07F1F5
S325080125200109A9EB0700019042E0012F00DA01270021112F01DD112000E03846CDE900017D
S3250801254004A90CA8FFF7B4FCDDE90D010C9A00914FF0000BB946109221070FD4009A4A453B
S3250801256003DA914601E0A9F10109B9F1010F05DD109AA9F10101515C3029F4D0B84202DA91
S3250801258010F1040F03DA0121CDE9011010E0002803DC8344A9EB000102E0411C494500DD55
S325080125A08946A0EB0B00401C01904FF000400290200705D40198484502DB4FF0FF300190A7
S325080125C000208DF84B0002980DF14B07B0F1004F25D002200C902B200D90029800280CDADF
S325080125E0404202902D200D9007E00A210298F6F70FF93031029007F8011D0C99481E0C9076
S325080126000029F2DC02980028EFD1791E0D980870307800F0200040F0450007F8020D11A88A
S32508012620C01BC01D02901398007800B1012000EB0901019801EBE071029801440398401AAD
S32508012640401E0390E00306D453462146179A039800F05CF805441398007818B152461799B0
S3250801266090476D1CE00323D553462146179A039800F04CF805441BE0BBF1000F07DB009817
S32508012680584504DD1098179910F80B0001E0179930205246904701980BF1010B401E05F1FD
S325080126A00105019004D12E205246179990476D1CB9F10001A9F10109DEDC05E017F8010BA0
S325080126C05246179990476D1C0299481E02900029F4DC53462146179A03989EE62D000000BA
S325080126E02B000000200000002DE9F041044600251E461746880404D405E039462020B0470A
S325080127006D1C641EF9D52846BDE8F0812DE9F041044600251E469046C80301D5302700E085
S325080127202027880404D505E041463846B0476D1C641EF9D52846BDE8F0810A68531C0B6054
S3250801274010707047F0B40C4905244A680E68531C93FBF4F504FB1535B54203D1F0BC07A09C
S32508012760FFF71CBB044D0835A85493FBF4F004FB10304860F0BC7047E40A00204576656E9B
S32508012780742071756575652069732066756C6C0A00000000F0B58DB001F0BBF82E4E002571
S325080127A02E4C24E09DF824300AAA03A80899F7F761FA8DF81F5001203070079803AF0090C4
S325080127C097E80F0000F0D4F901280ED12348142203A91438F5F7F9FC2048CDE9015614385C
S325080127E0016900910FC800F079F9FAF7FBF9676827B309AB0AAA08A90020B8470028D1D106
S325080128001CE000BF9DF824300AAA03A80899F7F731FA8DF81F50FEF773FC30B1079803AE63
S32508012820009096E80F0000F033F9079803AE009096E80F00FEF780FCFAF7D4F9E66936B17E
S3250801284009AB0AAA08A90120B0470028DAD100F0B9FF0DB0F0BD0000EC000020C81400204B
S3250801286070B520211B48F5F7C9FC1A4830213038F5F7C4FC01F046F8FAF730FAFAF766FA6D
S32508012880144A1549303A0020FAF718FB10B113A0FFF784FA0F4A1049183A34390120FAF774
S325080128A00DFB10B113A0FFF779FA0A4C303CE56825B100231A4619461846A847646A002C16
S325080128C007D0A4460023BDE870401A4619460120604770BDF81400204401002063616E3108
S325080128E020D0ADD2E9B3F5CABCBBAFB3C9B9A60D0A00000063616E3220D0ADD2E9B3F5CAB9
S32508012900BCBBAFB3C9B9A60D0A00000000B50D49A1B041F20B020020A1F80520401C80B288
S325080129202828FBD3502048800749087C401C087406A0FFF733FA20AA69460248F8F712FCFD
S3250801294021B000BD2A1F0020B020002053656E642063656C6C2074656D70200A0D0000002A
S3250801296010B51149A2B041F20C02A1F80520002001F2EA2213180C18401C93F8973080B28A
S32508012980E3710828F6D3082048800849087C401C087407A0FFF702FA20AA69460248F8F7F3
S325080129A0E1FB22B010BD00002A1F0020B020002073656E6420626D735F73746174655F69E0
S325080129C06E666F0A0D00000010B51249A2B041F20A02A1F80520002001F2EA2200EB4003D2
S325080129E00C181344401C93F8213080B2E3712828F4D3282048800849087C401C087407A014
S32508012A00FFF7CCF920AA69460248F8F7ABFB22B010BD00002A1F0020B020002053656E6412
S32508012A202063656C6C2074656D70200A0D0000002DE9F05F0024134EDFF84CB0DFF84CA03A
S32508012A40054640F227474FF00109A04656F83410286888420FD106EBC400416809B12846FB
S32508012A6088472868B84204D15846FBF7BDFE8AF80C90C5F80080641C64B2102CE6D3BDE843
S32508012A80F09F000010050020B4340020302400200FB4142210B502A90D48F5F796FB0C4C54
S32508012AA01422214601F51270F5F78FFB80210948F9F7F7F808480168204688471421204622
S32508012AC0F5F79CFB0020206010BC5DF814FB0000F00C0020001001400C0500200FB470B50E
S32508012AE0214C0A9D607814280BD200EB800004EB8000142204A9001DF5F767FB6078401C66
S32508012B006070059941F6EC4218480024B2EB114F10D19DF81B10102904D0132902D011295C
S32508012B2003D005E09DF81E1001E09DF81C1081700A210EE041F6EB42B2EB114F0AD19DF88E
S32508012B401B108278914203D114210161847001E032210161054800210C30FDF701F92C7045
S32508012B6070BC5DF814FB0000A40D0020980000200FB4142270B504A92748F5F726FB264D73
S32508012B8026484FF0FF366C68C461A0B2A0F57441563903D0304670BC5DF814FB41F6EC41E3
S32508012BA0B1EB144F03D0491EB1EB144F06D11A49142201F17800F5F708FBEBE718498C4204
S32508012BC01AD018498C4217D017498C4214D017498C4211D016498C420ED016498C420BD0B2
S32508012BE015498C4208D015498C4205D014498C4202D014498C420CD10749142201F1B40090
S32508012C00F5F7E3FA0449AA7A00230B31204600F091FB0020BFE70000DC0C002098000020A4
S32508012C2056F4261856F4011856F4071856F4081856F40A1056F4121856F41D1856F41F08FF
S32508012C4056F41A1056F41A1810B5134C13490020C4E900010421217260720520A072FF2245
S32508012C60082104F10B00F5F7C2FA0D4A32F8411F5088E172090AC0F57A6021736073000A55
S32508012C80A073107908B1022000E00120E073BDE81040014800F00CBF680D0020F45610185A
S32508012CA0CC0600202DE9F04101462E4C002504220823022604F10B0001293CD002294FD1EC
S32508012CC02949C4E9005122726572A372FF220821F5F78DFA254F0120E07237F8330F20734D
S32508012CE0000A60737888C0F57A60A073000AE073B8882074000A6074B879A074204600F09C
S32508012D00D7FE0320F8F7BBFAE672F888000A2073387A0A306073B7F80900A073000AE073AC
S32508012D20B7F80B002074000A6074A574BDE8F0410C4800F0BDBE0E49C4E9005122726572EA
S32508012D40A372FF220821F5F752FA1020E0720D2020736573A673FF20E07325740620E3E79F
S32508012D60BDE8F081680D0020F456EB1CCC060020F456EC1C2DE9F04101462D4C00250422B2
S32508012D800823022604F10B00012938D002294CD12849C4E9005122726572A372FF2208211E
S32508012DA0F5F725FA244F0120E07237F8460F2073000A60737888A073000AE073B8882074DB
S32508012DC0000A607497F82600A074204600F070FE0320F8F754FA97F82600C0F16400A7F8B0
S32508012DE00700E6722073000A6073A573E57325746574A574BDE8F0410D4800F059BE0F4970
S32508012E00C4E9005122726572A372FF220821F5F7EEF91020E072092020736573A673FF20BA
S32508012E20E073257411206074E3E7BDE8F0810000680D0020F456EB1CCC060020F456EC1C88
S32508012E4070B50C4C05460C490020C4E900010421217260720220A072FF22082104F10B0070
S32508012E60F5F7C5F9E572280A20732046BDE8704000F01EBE680D0020F45627182DE9F04F83
S32508012E8085B0054614216846F5F7B8F9714C08210026042204F10B004FF0100B4FF0070948
S32508012EA04FF00208012D7CD0022D7BD16A4B9246C4E9006322726672A172FF22F5F797F90C
S32508012EC0664D0127E772A8782073E87860732879A0736879E073E8882074000A6074287A5D
S32508012EE0A074204600F0E4FD0320F8F7C8F984F80B802889000A2073A87A6073E87AA073E6
S32508012F00287BE073687B20746674A674204600F0CFFD0320F8F7B3F90320E072277384F8D6
S32508012F200D80A87CA073E87CE073287D2074687D6074A87DA074204600F0BAFD0320F8F7BD
S32508012F409EF94748FF22112180F887616846F5F74EF984F80BA0E87D2073287E6073A673F7
S32508012F609DF80000E0739DF8010020749DF8020060749DF80300A074204600F099FD03200A
S32508012F80F8F77DF90520E0729DF8040020739DF8050060739DF80600A0739DF80700E07310
S32508012FA001E03FE03BE09DF8080020749DF8090060749DF80A00A074204600F079FD0320A2
S32508012FC0F8F75DF90620E0729DF80B0020739DF80C0060739DF80D00A0739DF80E00E073D3
S32508012FE09DF80F0020749DF81000607484F812B0204600F05DFD0320F8F741F984F80B90C0
S325080130000A2121730B21617384F80E90E020E073FF2020746074A0740E4800F049FD05B099
S32508013020BDE8F08F0F4BC4E9006322726672A172FF220821F5F7DBF884F80BB03120207350
S32508013040667384F80E90FF20E073267484F81180A674E1E7680D0020F456EB1CCC0600209B
S3250801306028150020F456EC1C70B50B4C05460B490020C4E900010421217260720120A072EC
S32508013080FF22082104F10B00F5F7B1F8E5722046BDE8704000F00CBD680D0020F45609107F
S325080130A010B5134C13490020C4E900010421217260720720A072FF22082104F10B00F5F7BA
S325080130C096F80D4890F86C10E17230F8661F2173090A61734188A173090AE173017921742C
S325080130E0407960742046BDE8104000F0E1BC0000680D0020F4561C18CC06002070B5484D8D
S3250801310048490020C5E900010421297268720720A872FF22082105F10B00F5F768F82B2083
S32508013120F8F754FB404C18B92C20F8F74FFB28B194F85B0020F00300401C03E094F85B0067
S3250801314020F0030084F85B002D20F8F73FFB18B90C20F8F73BFB28B194F85B0020F00C0002
S32508013160001D03E094F85B0020F00C0084F85B002E20F8F72BFB002894F85B0020F03000B4
S3250801318000D0103084F85B000B20F8F71FFB002894F85B0020F0C00000D0403084F85B000F
S325080131A00E20F8F713FB18B91A20F8F70FFB28B194F85C0020F00300401C03E094F85C00D6
S325080131C020F0030084F85C0094F85900012894F85C0020F00C0000D1001D84F85C0094F891
S325080131E05A00012894F85C0020F0300000D1103084F85C0014F84F0FE87260780A302873BB
S32508013200A0786873E0780A30A8732079E873207B2874607B6874BDE87040014800F048BC8B
S32508013220680D0020F4561318CC06002070B53E4D3E490020C5E900010421297268723C4C5B
S32508013240A972204694F86C1090F86100642920F0030000D1401C84F861002F20F8F7B6FA55
S32508013260002894F8610020F0C00000D0403084F861001A20F8F7AAFA18B90E20F8F7A6FAE2
S3250801328028B194F8620020F00300401C03E094F8620020F0030084F862000B20F8F796FA7D
S325080132A0002894F8630020F0030000D0401C84F863000320F8F78AFA18B90420F8F786FAD0
S325080132C028B194F8630020F00C00001D03E094F8630020F00C0084F863002E20F8F776FA64
S325080132E0002894F8640020F0030000D0401C84F864000120F8F76AFA002894F8640020F0EC
S325080133000C0000D0001D84F8640014F8610FE87260782873A0786873E078A873BDE87040C1
S32508013320014800F0C5BB0000680D0020F4561910CC0600202DE9F0411F4616460C46054626
S32508013340F7F73AFA574A2846A91A574D90424FD022DC564AA0EB0201904276D00BDC54490D
S32508013360401871D05349C8426BD12078A876A86B40F0080064E05048081825D0B0F5C02F3D
S325080133805FD13A4631462046F7F7F8F8002858D0A86B40F0020053E0B1F5202F46D0B1F53A
S325080133A0901F52D0B1F5A81F5ED0B1F5F01F48D121463246032E00DD03223B48F4F705FF40
S325080133C0A86B40F480403BE02078E87060782871A0786871E078A8712079E8716079287294
S325080133E0A0796872E079A872A86B40F0010027E0208868826088A882B4F904004FF47A619A
S32508013400884202DDA0F57A6001E0C0F57A60E882B4F90600884202DDA0F57A6001E0C0F54A
S325080134207A602883A86B40F0040009E03A4631462046F7F773F8002803D0A86B40F01000C4
S32508013440A863BDE8F08100E01CE0207885F82300607805F8240FA0786870E078A8706869EF
S3250801346040F020006861ECE7207905F8340F60796870A079A870E079E870686840F04000A5
S325080134806860DEE7207885F82700607805F8280FA0786870E078A870286940F0800028611E
S325080134A0CFE7000056F40818040D002056F41A10AA0BE0F7000015F8000019F870B50F4C0E
S325080134C08318A34201D9032070BDA2B1012400230BE005780E78AE4204D0FF2D01D00220C7
S325080134E070BD0024401C491C5B1C9342F1D3012C01D0012070BD002070BD000000000208F8
S32508013500F8B501210820FAF789FF03248DF8024014250F4F8DF803504FF48066ADF80060A1
S3250801352069463846F8F736FB8DF802407400ADF800408DF8035069463846F8F72BFB31467E
S325080135403846F8F7AEFB21463846F8F7AAFBF8BD000C01402DE9F0418846054614462249A6
S325080135602044884202D90120BDE8F081CCB3E00700D0541C224641462846FFF79FFF00283D
S32508013580F2D0012080F31088F8F7D6F93520F8F74BF9E80AC002F8F74DF9074640F2E73069
S325080135A0401E80B2FCD200260FE000BF08EB460118F81600497840EA01212846F8F776F991
S325080135C00746042804D1AD1C761CB6EB540FEDD3F8F764F9002080F31088042F02D00220D1
S325080135E0C2E7FFE70020BFE70000020810B54FF0000140B1054C2046F6F71CFE2046F6F756
S3250801360003FB012010BD024CF5E70000006800400064004030B4022814D20B4A00EB800382
S3250801362002EB83021569002D0CD00A7A8B7A042A06D00C6801F10B022146AC4630BC604796
S325080136404C68F7E730BC7047940F002010B538B1044800BFF6F792FE042800D1FF2010BD44
S325080136600148F7E7006800400064004030B4022815D20C4A00EBC00302EB83040122E368ED
S325080136808A4013420BD09343064AE36000EB8003483252F82320002A01D030BC104730BC19
S325080136A0704700004C0F002010B518B1F6F7F4F8012010BDF6F718FDFAE7000010B5832821
S325080136C012D10A4C207C01280ED0A4F13000C16A09B1012088470120207404480021BDE89E
S325080136E010401430FCF73CBB10BD0000F814002070B500291DD10F4E0546002406EB041037
S325080137000168A94203D100210C30FCF729FB641CA4B2022CF2D30848817F002909D0017C66
S32508013720022906D100218177BDE870401830FCF717BB70BDF0000020F8140020044B00EB5A
S32508013740C00203EB820200219160FFF74FBF00004C0F0020022811D2094900EB800201EBDD
S3250801376082018A68002A09D0054B00EBC001483B03EB8101C96801B10121104770470000C0
S32508013780940F002010B50446022817D2FAF7EDFF0B4804EB840100EB8100C16809B12046DC
S325080137A08847FAF7E4FF064804EBC401483800EB8100C168002901D00021C16010BD000037
S325080137C0940F00202DE9F047254F4FF00008454607F1300606EB05142078012802D002288F
S325080137E02DD036E0A089062803D21E4931F8101000E0C621201DFCF7B3FAF8B1FAF7B5FFD9
S32508013800A089401CA08105EB450007EBC000D0F80CC0BCF1000F04D000231A461946284698
S32508013820E047022020704FF00109FAF7A0FF04F108000021FCF794FA84F80E9009E004F130
S3250801384008006721FCF78CFA18B1A4F80C8084F800806D1CEDB2022DBCD3BDE8F087000061
S32508013860C8140020B07301082DE9F041022802D30020BDE8F0810C4E00EBC00706EB87040D
S325080138800125A560002565712371E27026F827102146E560FFF708FF18B10220A060012003
S325080138A0E7E7A560E4E700004C0F002070B50646022807D20D4806EBC60400EB8405A868D8
S325080138C0022801D0002070BD05F110000446F6F7B1F921463046FFF7B9FEFF28F3D0012213
S325080138E0E96882401143E96070BD00004C0F00200EB58DE807006946014803F0FAF80EBD7A
S325080139003C12002010B500F089F8BDE8104000F033B810B500F042F8BDE8104000F088B810
S3250801392030B54FF0FF34E8B1124A002352F83350854208D102EBC300416011B9002042F827
S325080139403300002030BD5B1C142BEFD351B1002352F8335045B102EBC3056D6825B15B1CE1
S32508013960142BF5D3204630BD42F8330002EBC3004160E6E7BC0F002010B54FF4267106487B
S32508013980F4F73CFC04492823A0310C2201F5F07003F088F8002010BDBC0F00203EB5104C6E
S325080139A004F5207515E06946284603F087F8DDF80000002154F83120824207D104EBC10106
S325080139C04B6833B1DDE90112984702E0491C1429F0D3284603F056F80028E4D000203EBD9C
S325080139E0BC0F002000280CD00B4A002101EB410302EB83039B682BB1491C89B21429F5D32C
S32508013A000020704701EB410302EB83018860002042F82300084670475412002010B5F02159
S32508013A200248F4F7EBFB002010BD0000541200202DE9F84300216846FCF792F9009818B3E8
S32508013A40012821D0DFF84880002500BF05EB450108EB810458F82160A76896B18FB1201D68
S32508013A603146FCF77DF901280BD1A06838B160680099091AB1FBF6F101FB06006060204622
S32508013A80B8476D1C142DE1D30020BDE8F883000054120020002803D002C00021FCF760B9EA
S32508013AA07047002803D00068002800D0012070471CB50F490C68C4B1017A002304290ED052
S32508013AC0D0F80020CDE90023427A52B10023042909D0016800F10B020020A0471CBD42683D
S32508013AE0F0E7837AF3E74168F4E700201CBD0000C81400207CB50446FDF70CFB38B9207A8F
S32508013B00042830D0D4F80000FDF70EFB68B31C48856935B3207A0022042828D0D4F8001090
S32508013B20CDE90012617A21B30023042823D0216804F10B020120A84798B1207A04281CD027
S32508013B402568104E002400BF06EB04100168A94203D100210830FCF703F9641CA4B2022C0F
S32508013B60F2D300207CBD6068CEE701207CBD6168D6E7A37AD9E76168DAE76568E1E70000BF
S32508013B80C8140020F00000200A4810B5418D49B1002141850848F9F73CFB08A0BDE8104030
S32508013BA0FEF7FCB8012141850348F9F712FB09A0F4E700008C01002088090020BFAAC6F418
S32508013BC04143BDBBC1F7CEC2B6C8BCCCB5E7C6F70D0A0000B9D8B1D54143BDBBC1F7CEC2C1
S32508013BE0B6C8BCCCB5E7C6F70D0A0000094810B5418C41B100214184F9F746FC06A0BDE808
S32508013C001040FEF7CBB801214184F6F761FE07A0F5E700008C010020BFAAC6F4BDBBC1F717
S32508013C20BCCCB5E7C6F70D0A00000000B9D8B1D5BDBBC1F7BCCCB5E7C6F70D0A000000003E
S32508013C40704700000B4810B5C48C00210A4A01234CB1C184D3710948F9F7DBFA08A0BDE8B4
S32508013C601040FEF79BB8C384D1710448F9F7B1FA06A0F4E78C010020902300207009002093
S32508013C80BFAAC6F443433143500D0A00B9D8B1D543433143500D0A000B4810B5048D00214F
S32508013CA00A4A01234CB1018513720948F9F7B1FA08A0BDE81040FEF771B803851172044877
S32508013CC0F9F787FA07A0F4E78C0100209023002080090020BFAAC6F44343325F43430D0AE2
S32508013CE000000000B9D8B1D54343325F43430D0A00000000F9F78CFB0B4810B5048C0021AA
S32508013D000A4A01234CB1018493710948F9F781FA08A0BDE81040FEF741B80384917104487A
S32508013D20F9F757FA08A0F4E78C0100209023002060090020BFAAC6F4D6B1C1F7BCCCB5E721
S32508013D40C6F70D0A00000000B9D8B1D5D6B1C1F7BCCCB5E7C6F70D0A0000000070477047C4
S32508013D60704700000A4810B5818C49B1002181840848F9F74EFA08A0BDE81040FEF70EB859
S32508013D80012181840348F9F724FA07A0F4E700008C01002078090020BFAAC6F4C9FDD1B951
S32508013DA0C4A3BFE90D0A0000B9D8B1D5C9FDD1B9C4A3BFE90D0A000070477047704700001C
S32508013DC00D4810B5C18B61B10021C1830B48F9F720FA0B48F9F71DFA0AA0BDE81040FDF7AD
S32508013DE0DDBF0121C1830548F9F7F3F90448F9F7F0F908A0F1E700008C0100207809002096
S32508013E0068090020BFAAC6F4B8DFD1B9C4A3BFE90D0A0000B9D8B1D5B8DFD1B9C4A3BFE951
S32508013E200D0A00002DE9F04104460E460D20FCF77DF80A20FCF77AF8002510E02078F8F7B7
S32508013E40DDFB01462078F8F7D1FB07460846FCF76DF83846FCF76AF86D1CADB2641CB542BC
S32508013E60ECD30D20FCF762F8BDE8F0410A20FCF75DB8002142F6DE6304E01A46521EFDD1D6
S32508013E80491C89B28142F8D37047FFF739BB2DE9F04115460C460646F8F734FEA020F8F734
S32508013EA007FEF8F757FE98B9200AF8F701FEF8F751FE68B9E0B2F8F7FBFDF8F74BFE38B940
S32508013EC0F8F720FEA120F8F7F3FDF8F743FE20B1F8F72EFE0020BDE8F08100246F1E09E03A
S32508013EE0BC4201D0012000E00020F8F7B3FD3055641CA4B2AC42F3D3F8F71AFE0120EAE71C
S32508013F002DE9F041164607460C4600252AE035B1E00618D1F8F70CFE0620F7F7B0F9F8F7C7
S32508013F20F1FDA020F8F7C4FDF8F714FE88B9200AF8F7BEFDF8F70EFE58B9E0B2F8F7B8FDBC
S32508013F40F8F708FE28B9785DF8F7B2FDF8F702FE20B1F8F7EDFD0020BDE8F081641C6D1C31
S32508013F60A4B2ADB2B542D2D3F8F7E2FD0120F3E770B5174D0526A5F1080423E000F068FD6A
S32508013F80E8B92168685C491C91FBF6F206FB12112160062813D2DFE800F0120306090C0F9D
S32508013FA0F7F738FB0EE0F7F775FB0BE0F7F77CFB08E0F7F739FB05E0F7F780FB02E005A056
S32508013FC0FDF7ECFE00F044FD0028D7D070BD0000EC0A0020556E6B6E6F776E206576656EF3
S32508013FE0742069732069676E6F7265640A0000002DE9F041134C0546C1B22046FDF744F836
S3250801400020880006FCD5104890F8A810012906D10E4E0027B178022904D080F8A8702846D0
S32508014020BDE8F0810A4C0B48E179962903D24554491CE171F3E7FDF7C7FD307C401C307436
S32508014040E771ECE7004C004028150020B02000208C010020E819002038B51248006F016B5D
S3250801406088478DF8000069460F48F7F7CBFC0F4C0F4D012801D068B111E002212846FAF7E5
S32508014080A1FB60B1E07B401CE0732846FAF7ACFB012038BD0020E0732846FAF7A5FB0020AC
S325080140A038BD0000CC06002014240020682300208C340020134810B590F83800C0070DD0A3
S325080140C011484179012907D0022141710FA000BFFDF764FE012010BD12A0F9E717480069DC
S325080140E08047022801D0022010BD15480A210446FAF768FB0028F7D02046FAF775FB032001
S3250801410010BD0000040D00207C230020424D535F50524F544F43414C5F4742323031310A78
S325080141200D000000424D535F50524F544F43414C5F4742323031350A0D000000580000207F
S325080141404C340020104810B500698047022802D0012810D008E00D490020C8730C48006F02
S32508014160016A8847042801D0002010BD09A0FDF715FE012010BD88210B48F4F73FF80BA0A5
S32508014180FDF70CFE022010BD5800002068230020CC060020BDF8C8EBD6B1C1F7B3E4B5E734
S325080141A0C1F7B3CC0D0A000044340020BDF8C8EBBDBBC1F7B3E4B5E7C1F7B3CC0D0A0000F1
S325080141C00D4810B5806B44F2010108420BD0F7F7ADFA3D210848F4F711F888210748F4F754
S325080141E00DF8012010BD064800698047022801D0022010BD002010BD040D0020443400209F
S32508014200580000200D4810B5C078AA2809D0FAF7A1F958B10A480069804702280BD00320DC
S3250801422010BD08A0FDF7BAFD012010BD0CA0FDF7B5FD022010BD002010BD0000040D002002
S325080142405800002052455620445F43445A5F48414E44494E475F43524D2041410A0D0000F4
S3250801426052656164792D537461746520526563656976656420546865204368617267696EA8
S32508014280672050696C652041626F7274204D6573736167650A0D000010B5FAF75BF948B1E7
S325080142A0FAF7E8FD50B1074800698047022807D0032010BD04A0FDF771FDF9E7012010BDD4
S325080142C0002010BD5800002052756E6E696E672D53746174652052656365697665642054A0
S325080142E06865204368617267696E672050696C652041626F7274204D6573736167650A0DE1
S3250801430000000000214810B5807EAA2808D0FAF721F950B12820F7F759FA002821D108E021
S325080143201BA0FDF73BFD012010BD20A0FDF736FD17E00620F7F74AFA98B91C20F7F746FAA8
S3250801434078B92120F7F742FA58B90920F7F73EFA38B90A20F7F73AFA18B92620F7F736FAE0
S3250801436008B1032010BD1F4800698047022801D0052010BD1C483C210446FAF723FA0028C0
S32508014380F7D02046FAF730FA042010BD040D002043445A5F5F43524F20414120746F204319
S325080143A068617267696E670A0D00000053746172742D537461746520526563656976656474
S325080143C020546865204368617267696E672050696C652041626F7274204D657373616765A3
S325080143E00A0D0000580000206434002010B5064805210446FAF7E6F9002803D02046FAF7C2
S32508014400F3F9012010BD00007C34002000B5F4F739FC0520FFF72DFD5DF804EBFAF740B99B
S32508014420072070477047022070470000124810B5018F49040DD500218163104901204871E9
S325080144400F480088FEF7FCFCBDE810400DA0FDF7A5BC0A4840F6B83108300446FBF780FC29
S32508014460002808D00CA0FDF799FC2046BDE810400021FBF775BC10BD040D00207C2300209C
S32508014480CC060020445F43445A5F48414E44494E475F43484D0D0A004E4F2048616E647346
S325080144A068616B65205369676E616C0A0D00000000207047704701207047704703207047C8
S325080144C00848007928B1012807D0022808D1F7F73BBB02210448F7F7FBBA0348F7F724BB1A
S325080144E0704700007C2300207D2E010805207047F6F7B2BA042070472DE9F041304E002589
S3250801450006F12807F07C012811D1F6F793FA70B1FDF774FB58B9F4F709FD40B1FAF76AF9AA
S3250801452028B93879012802D1F4F724FE0546254C284694F83810490707D4F17C012901D040
S32508014540B9B12BE0A17EAA2928D0FEF78DFD1E48006F816A8847012528B1387918B9BD7130
S325080145601A48F8F756FEF574A06B20F00400A06314E013481430007920B1012807D00228F5
S325080145800CD108E006211248F7F7A2FA06E01048F7F7CAFA02E00620F7F7D6FAA06B8107F3
S325080145A002D520F0020007E0000706D509A0FDF7F5FBA06B20F00800A063BDE8F081000071
S325080145C068230020040D0020CC06002060090020A52C010843445A5F48414E44494E475F03
S325080145E043524D2041410A0D000000000620704738B51A48006FB0F90200002800DA404247
S32508014600ADF8000069461648F7F7FCF900B1012014490979012902D108B1F6F783F91148CD
S32508014620322144380446FBF79BFB012806D10020FEF7FCFD00212046FBF792FB0948FA214A
S3250801464034380446FBF78CFB012806D10020FEF727FD00212046FBF783FB38BDCC06002005
S32508014660082400209023002070B505460846F7F79BFD040062D00420812D2CD00CDC042DAB
S3250801468017D0802D5AD194F85400032856D3E16C002953D0802043E0822D13D0832D4DD15C
S325080146A094F85410032949D394F8911002292DD033E094F85400032840D32046BDE8704072
S325080146C0F8F768B894F85400032837D3E16C002934D0822024E094F8541003292ED394F8DE
S325080146E0911002290DD194F8901094F84420914200D2032084F89100227804210120FFF73A
S32508014700F7F8E16C002919D0812009E084F89100227804210120FFF7EBF8E16C19B1832032
S32508014720BDE870400847207800F09AFA2078BDE8704000231A46194600F0DCBA70BD70B503
S325080147400C460546F7F730FD00281ED090F85410022906D8C168002917D02846BDE870408B
S32508014760084781290AD0002C0FD1802180F854102A46BDE870400120FFF7BAB8002C04D080
S32508014780812180F854102A46F3E770BDFFF7D7BF10B50446F7F708FD002813D090F8541090
S325080147A0022906D8C16800290CD02046BDE810400847832180F854102246BDE8104001200B
S325080147C0FFF796B810BD00002DE9F0411D4617460E468046F7F7E8FC040030D094F85400E2
S325080147E003282CD3802802D1032084F8540094F84000C00706D0A36C0BB32A463946304677
S3250801480098471CE00F48691E2A4606600571072903D83946401DF3F7D8FC04F15800094940
S32508014820054602F066F9284602F034F938B1822084F85400014642460120FFF759F801208D
S32508014840BDE8F081A414002010B50C46F7F7ACFC002815D090F89120E1B2022A01D0032AAB
S325080148600ED190F898208A420AD1052180F8911090F85410032903D3BDE81040F7F78ABF0A
S3250801488010BD0020401C80B23C28FBD3704700002DE9F047504C1420012684F86C0041F246
S325080148A088302080A670E670002525714FF0030884F805804FF47A70E08041F26800208156
S325080148C04220A0725920E0724420207354206073A573E5732674022767741920A0740B20C6
S325080148E0E0740A2020756575A5751020E07525766576112239A104F11A00F3F766FC3CA162
S32508014900A4F134000A6840F85F2F496841604FF4D27024F8330F4FF4FA70608041F224303E
S32508014920E0806E202072C820A4F809004FF47A60A4F80B006573E0814FF416702082A774D8
S32508014940A4F81350A4F81550B4F81700DFF8AC906FF30B0000F5A270A4F8170014F8180F18
S325080149606FF0310720F0F000103004F8020B3C202080A6703A4649460A20FDF761F9E0705F
S3250801498084F804803A4649460520FDF759F960710420A071E57125726572A572E5722573BE
S325080149A065732674A4F8115004F8135F6420607140F25910E08040F2631020813A46494666
S325080149C01920FDF73DF9A0723A4649461C20FDF737F9E072BDE8F087CC0600204C5650434F
S325080149E035323739584E44303133383138000000533030314830303100000000CDCCCC3D53
S32508014A002DE9F0410B3020F00706104D19E02068B04215D3B0420AD9871B201DD4F804802C
S32508014A20F3F7D3FBA019C0E90078286004E060682860201DF3F7C9FB201D2660BDE8F08155
S32508014A40251D2C68002CE2D10020F7E7140C00200448D0E90010814201D1012070470020B2
S32508014A6070470000E40A002010B50E4C62785AB100206070E168C4E9030120700A20B1FB0E
S32508014A80F0F080B2A08010BDFFF7C0FCE1680844E0602078411C2170092801D30120607005
S32508014AA0A08810BD7C00002086B0FAF771FA4FF4004162B60803F8F7A1FCFAF73BFA6846BD
S32508014AC0F9F7BEFCF8F74EFCF8F766F9F8F7B4F8FFF7DBF9F4F75CFBF4F72AF9F4F7F6F808
S32508014AE04FF47A3002F058F84FF4E13002F0B0F840F2CF2140F2F310FAF7AEFAFFF7C8FEDE
S32508014B00FCF7D0FAF8F77AF8FDF7AAFE3A493BA0FDF744F9F9F772FDF5F75EFEF6F740FF6A
S32508014B20394F3A4E0124BC73002535723848F8F750FBF4713748F8F76CFBF8F7A5FC364C30
S32508014B40FBF746F9FDF726FE207801281BD06078012831D0A078012834D0E07801283CD07D
S32508014B60207901283FD06079012840D0E0790128E6D1E571F4F7F0FBF9F7CAF8F9F710FB31
S32508014B80FCF708FBDCE72570B87B08B1F4F772F9F4F786FBFCF783FA204E306880477068F5
S32508014BA08047B0688047F0688047F7F77FF8FAF79BF8F5F7EFFEC3E76570F9F7DBFDF8F729
S32508014BC011F8BDE7A5700220F7F70CFB1449C860FCF75EFAF9F742FBB2E7E570F6F764F8B9
S32508014BE0F6F7CEF9ACE72571F8F766FBA8E76571FFF7BEF9A4E70000BC730108B0E6B1BE9F
S32508014C00BAC52025730D0A007C230020902300208009002070090020181500206C0000208A
S32508014C20400C002070B53AB10C4B84189C4203D8A3F50074A04202D24FF0FF3070BD31B1FE
S32508014C40002302E0CD5CC5545B1C9342FAD3011B92B289B2FCF736FA002070BD084700206B
S32508014C6070B50546F7F7A0FA040003D094F85400022801D8002070BD022084F85400E168EB
S32508014C8009B12846884794F8910018B3D4F8A8204AB906E00428D4F8A4000AD00321904738
S32508014CA018E0226DB2B10528F4D10021D4F8A400F5E70121F3E72946304601F0FFFE68B1B4
S32508014CC0D4F8A8200AB9226D42B10321D4F8A400904703E004F1940504F17006304601F03E
S32508014CE0D1FE0028E7D0202104F19000F3F786FA012070BD2DE9F0411D4616460F46804658
S32508014D00F7F752FA04002CD094F85400012828D9D4F804C0BCF1000F23D02B463246394699
S32508014D204046E047E8B1D4F88C1031B194F84530182204F1700001F0B5FE94F84000C007FD
S32508014D4009D1D4F8881031B194F84530102204F1580001F0A7FE032084F854000120BDE855
S32508014D60F0810020FBE710B5F7F71EFA002801D090F8540010BD2DE9FF411E4615460F46DA
S32508014D80F7F712FA04000ED094F8540002280AD94DB194F84000C00705D104F158008046C1
S32508014DA001F070FE18B1002004B0BDE8F0816946404601F083FE0028F6D0009838609DF878
S32508014DC0040030709DF80420501E072804D828460DF10501F3F7F9F994F85400822802D143
S32508014DE0032084F854000120DEE72DE9F04786B01D46DDE90E9816460F46F7F7D5F9040008
S32508014E000BD094F85400022807D9082D05D804F17000824601F03EFE18B1002006B0BDE80E
S32508014E20F087F9F7A2FC94F85400832801D0032802D2F9F79CFCF0E7CDF8148000978DF82F
S32508014E400550CDF8109016B900208DF805009DF80520501E072804D831460DF10600F3F778
S32508014E60B4F9FF208DF804006946504601F041FE94F8910010B92046F7F78CFCF9F777FC34
S32508014E800120CBE700207047104910B500230C464FF480520846640705D0C01D20F007002F
S32508014EA0411AD1EB02020A49C1E900038118084A0839A2F1140221F0070111604B600B6053
S32508014EC00B1AC0E900139360536010BD44240020080B002030B5134900E011460A68824206
S32508014EE0FBD34B685C18844204D1406818444860084600E000BF43681C18944209D1094C96
S32508014F00143C2468A24209D052681A4442600A6812680260814203D0086030BD0460F9E7B2
S32508014F2000BF30BD080B002070B5274D04460026286898B100BFA4B104F00700C0F11000D1
S32508014F40C1438C423CD82118002939DD6868814236D81D4814300246146806E0FFF794FF67
S32508014F60E9E700BF2CE02046144662688A4202D22268002AF7D12A68944221D00668226890
S32508014F80026060680836421A102A05D9601842606160FFF79FFF00E000BF61686868401A25
S32508014FA06860AA68904201D2A86000E000BF41F00040606000202060E868401CE86000E017
S32508014FC000BF304670BD0000F40A00202DE9F04F9BB00546402107A8F3F710F9FE4F4FF0C8
S32508014FE0000AADF85CA087F810A0B5F805804FF6FF7BA8F5004020381ED0A8F5004021387E
S325080150001AD0DFF8D8930126F54CB8F5004F7CD05FDCB8F5D06F01F0F4844ADCB8F5607F63
S3250801502074D03FDCB8F1800F77D0B8F5C07F6ED0B8F5207F33D192E06A882E461446B2F530
S32508015040967F04D8E448E91D3830F3F7BEF8E24821463830FEF7E6FE301930F8025CA01EB7
S3250801506081B23046F4F7B6F8064602462946DDA0FCF794FEB54202D0E0A001F0D0BCD649F5
S3250801508008F1E00887F811A008F0FF0022463831FCF71AFBE149642088830420B8701BB050
S325080150A0BDE8F08FB8F5906F6AD0B8F5B06FF6D17DE0B8F5286F01F0B184F0DCB8F5F06FA5
S325080150C0F9D0B8F5086FF6D0B8F5186FE7D101F0A5BC48F20701A8EB01008845F7D009DC81
S325080150E06FF4004040440628D9D2DFE800F02F38474960F8062806D0D1DC0128E7D00228E0
S32508015100E5D00328CBD1C6A002E006E036E01DE0FCF744FE87F810A0C1E7E879012801D05C
S32508015120C6A0AAE7BE7084F8766044F86CAFAC49C4F804A0A4F808A0A8682060E868606059
S32508015140BE7089F800606C31C1A02DE2E879012801D0C7A091E70220B870C9A08DE7E97961
S32508015160CCA0FCF71BFED048D5F8091040F8011FB5F80D108180E97B817190E7CBA07CE7EC
S32508015180D0A0FCF70BFE287A01280ED0D3A1D5A0FCF704FE287A002881D1A04846710178D9
S325080151A00029B9D10421017079E7D1A1EFE7DFF86C8288F80660E87990B1CFA0FCF7EEFD55
S325080151C0E87901280ED00028A6D12C7ACEA02146FCF7E4FDD14888F804400D2C7ED057E3CC
S325080151E0CFA0EBE72F7AD2A03946FCF7D7FD012F76D0022F75D005F109000290042F71D00D
S32508015200072F70D0062F6FD0082F6ED0092F6DD00A2F6CD00B2FB0D00C2F69D00D2F68D094
S325080152204FF00A080E2F7DD00F2F7CD0102F7BD0112F7AD0122F79D0132F78D0142F77D048
S32508015240162F76D01D2F75D01E2F74D01F2F73D0202F72D0212F71D0222F70D0232F6FD0BD
S32508015260242F6ED0252F6DD0262F6CD0272F6BD0282F6AD0292F69D02A2F68D02B2F67D097
S32508015280302F66D0312F7DD0322F7CD0332F7BD0342F7AD0352F79D0362F78D0372F77D0AF
S325080152A0502F76D0512F75D0522F74D0532F73D0542F72D0552F71D0562F70D0572F6FD0B7
S325080152C0582F6ED0592F6DD05A2F6CD0602F6BD0612F6AD0622F69D0632F0BE0D9E2D9E21F
S325080152E054E166E16CE17AE181E19AE289E1A7E1B4E1C0E15BD0642F87D0652F58D06D2F08
S3250801530057D040F22F206E2F54D06F2F53D0702F52D0712F51D0722F50D0732F4FD0742FAD
S325080153204ED017E0B5E1C2E1CCE1ECE102E20EE21AE22FE23BE24AE259E282E293E2A2E2D4
S32508015340A9E2A9E2A9E2A9E2A9E2A9E2A9E2A9E2A9E2A9E2752F34D0762F33D0772F32D0D8
S32508015360782F31D0792F30D07A2F2FD07B2F2ED07C2F2DD07D2F2CD07E2F2BD07F2F2AD0DE
S32508015380802FDDE091E291E291E291E291E291E291E291E291E291E291E291E291E291E248
S325080153A091E291E291E291E291E291E291E291E291E291E291E291E291E291E291E291E2AE
S325080153C091E291E291E291E291E291E291E291E291E291E291E291E2B02000207D010020CC
S325080153E0281500200A0D44637263202530782C56637263202530780A0D0000000A0D2028A4
S325080154004463726320213D2056637263292072657475726E21212121210A0D008C01002083
S325080154205265636569766520444542554720444344432061636B0A0D0000000072656769D8
S32508015440737465726564206661696C65640A0D0072656769737465726564207375636365B9
S32508015460737365642C436F64652025730A0D00004C6F67696E204661696C65640A0D000083
S325080154804C6F67696E205375636365737365640A0D000000686561727420636F756E7420AE
S325080154A025640A0D00000000BC0C0020726563656976652073746174652064617461200A4D
S325080154C00D00000072656365697665206368617267652064617461200A0D000044697361D1
S325080154E0626C65006368617267652025730A0D00456E61626C650000706172616D207772D0
S325080155006974650A0D0000005265616420706172616D206E756D2025640A0D002A1F0020DD
S32508015520706172616D20726561640A0D00000000706172616D20616464722025780A0D00D8
S3250801554071D0812F70D0822F6FD0832F6ED0842F6DD0852F6CD0862F6BD0872F6AD0882FB4
S3250801556069D0892F68D08A2F67D08B2F6FD08C2F6ED08D2F6DD08E2F6CD08F2F7FF4CCAD75
S32508015580B5F80910A4F8DA11DDA048E1697A39B988F8056098F8002012B9042288F800200E
S325080155A0012904D0DCA1DEA0FCF7F8FB77E5E0A1F9E7687A012801D0DFA05EE5E2A05CE5DF
S325080155C00446F2F738FE82B2102A214605D2E248F2F7FBFD2146E1A021E1E5A0E4E76D7A7B
S325080155E0EAA02946FCF7DAFBA4F8695019E16D7AEDA02946FCF7D2FB24F84D5F6580A58017
S32508015600F4E70446F2F717FE82B2102A214615D2D1481038F2F7D9FD2146E9A0FCF7BEFBE0
S3250801562089F80060E2E7F8E3F8E3F8E3F8E3F8E3F8E3F8E3F8E3F8E3F8E3F8E3E6A0EEE0F4
S32508015640687A012807D084F887A0EAA00CE0EFE3EFE3EFE3EFE384F88760F6E7687A0128AD
S3250801566005D084F889A0E9A0FCF798FBBEE784F88960EEA0F8E7697A642903D284F88A10C0
S32508015680F2A0CCE0F7A0FCF789FB5A2084F88A00ACE76D7A4046B5FBF0F108FB1152B5FB88
S325080156A0F8F1F6A0FCF77AFB84F88B509EE76D7AF8A02946FCF772FB05EB8500400084F899
S325080156C08C0093E7B5F80950F8A02946FCF766FBB4F8592005EB8500B2EB400F04D90BEAFC
S325080156E04000A4F8830081E705EB85004100F3A0FCF754FB34F8590F143880B2B0FBF8F1A3
S325080157006085F5A050E7B5F80950F8A02946FCF745FBB4F85B2005EB8500B2EB400F04D924
S325080157200BEA4000A4F8850060E705EB85004100F3A095E0B5F80950F7A02946FCF72EFBD7
S3250801574005EB85010BEA4100A4F859004EE7B5F80950F6A02946FCF721FB05EB85010BEADF
S325080157604100A4F85B0041E76C7AF5A02146FCF715FBF8488178202901D920218170C9B2CC
S3250801578001EBC10100EB4101A1F807408178491C817084E4B5F809004146B0FBF1F2B0FB12
S325080157A0F8F108FB1202A4F86300EBA066E2687A012803D0022801D0EDA05EE484F88D0057
S325080157C0012802D0F0A1F1A029E0F5A1FBE7687A00EB80010BEA41004146B0FBF1F2B0FBD8
S325080157E0F8F108FB1202A4F85300EEA046E2B4F89010B4F85320687A914213D94546B2FBB1
S32508015800F5F2B1FBF5F1EDA0FCF7C8FAB4F853000A3880B2B0FBF5F1A4F89000F2A0FCF709
S32508015820BDFA41E200EB80010BEA41004146B0FBF1F2B0FBF8F108FB1202A4F89000F0A061
S325080158401CE2687A00EB80010BEA41006421B0FBF1F201FB1202B0FBF1F1A4F8B300EFA029
S32508015860FCF79CFA1BE4687A00EB80010BEA41006421B0FBF1F201FB1202B0FBF1F1A4F8C1
S32508015880B100EDA0FAE1697AA4F8B710F1A0C6E733E333E333E3E5E1F1E1FDE105E20DE2CE
S325080158A034E23BE249E258E268E274E284E288E28CE290E2A2E2C2E2CEE2DFE2F9E213E387
S325080158C01EE31EE31EE31EE31EE31EE31EE31EE31EE31EE31EE31EE31EE31EE31EE31EE3A9
S325080158E01EE31EE31EE31EE31EE31EE31EE31EE31EE31EE31EE31EE31EE31EE31EE300008A
S32508015900536F6343616C6962726174696F6E202025642020200A0D0064697361626C6500D7
S325080159206368617267696E672025730A0D000000656E61626C6500006F70656E2072656CCA
S3250801594061790A0D00000000636C6F73652072656C61790A0D00000038150020626C7565C8
S32508015960746F6F7468206E616D652025730A0D00626C7565746F6F7468206E616D65206D36
S32508015980697374616B652025730A0D00486561727420426561742054696D65202564202080
S325080159A07365630A0D0000004F76657254656D7056616C75652025642020200A0D00000037
S325080159C05379735061726150696C65442E736E3A25730A0D0000000053797350617261501C
S325080159E0696C65442E736E206661756C742025730A0D0000517569636B2043686172676599
S32508015A0020456E61626C650A0D000000747269636B6C65204368617267696E6720536F6383
S32508015A2020456E61626C6520300A0D00747269636B6C65204368617267696E6720536F6313
S32508015A4020456E61626C6520310A0D00747269636B6C654368617267696E67536F632564A9
S32508015A600A0D0000747269636B6C654368617267696E67536F632039300A0D007472696378
S32508015A806B6C6520706F7765722025642E25646B770A0D00747269636B6C6520637572724B
S32508015AA0656E742564410A0D00000000426D734D6178566F6C742564200A0D002564204217
S32508015AC06D734D6178566F6C74202564206661696C640A0D00000000426D52657175697205
S32508015AE065566F6C74202564200A0D00426D734D617843757272656E74202564200A0D00A2
S32508015B00726571202564206F766572206D6178202564200A0D000000426D734D6178566F56
S32508015B206C74202564200A0D00000000426D734D617843757272656E742564200A0D0000AB
S32508015B4073657474696E6720736F63282564290A0D000000A4170020754261744D61784510
S32508015B606E657267792025642E25640A0D0000004368617267696E674D6F64652046617596
S32508015B806C740A0D00000000435600004368617267696E674D6F64653A2573200A0D0000B5
S32508015BA0434300004F766572506F776572203A25642E25646B77680A0D000000526571750F
S32508015BC0697265506F776572202564206B77204F766572506F776572203A25646B772C669E
S32508015BE061756C740A0D000052657175697265506F776572202564206B77200A0D000000FD
S32508015C0052657175697265506F776572203A25642E25646B77680A0D000000004261745227
S32508015C2061746564566F6C74616765203A25642E2564560A0D0000004261744D61784368F6
S32508015C4061726765566F6C203A25642E2564560A0D000000426174436F756E74203A25645B
S32508015C600A0D0000B5F809004146B0FBF1F2B0FBF8F108FB1202A4F85F00B1A058E3B5F854
S32508015C8009004146B0FBF1F2B0FBF8F108FB1202A4F85900B1A04BE36D7AB5A02946FCF71A
S32508015CA07DF8323584F8B55044E36D7AB7A02946FCF774F8323584F8B650F8E3687A84F823
S32508015CC0B000012810D0022810D0032810D0042810D0052810D0062810D0072810D0082881
S32508015CE010D0FF2810D0E2E3AFA0BDE4B4A0BBE4B9A0B9E4BFA0B7E4C4A0B5E4C9A0B3E419
S32508015D00CEA0B1E4D5A0AFE4DAA0ADE4B5F80900A4F85D00B0FBF8F1DCA080E5697AA1F1C5
S32508015D200A005A2803D884F89310DDA077E5E5A0FCF734F884F893A0B9E3B5F8091040F60A
S32508015D40C412A1F57A70904205D8A4F8A610B1FBF8F1E2A063E5E9A061E5687A012808D0CC
S32508015D6084F8A8A094F8A800012805D0EDA1EFA055E584F8A860F5E7F3A1F8E7B5F809003E
S32508015D804146B0FBF1F2B0FBF8F108FB1202A4F86300EFA0CCE2B5F8090000EB80010BEAE1
S32508015DA041004146B0FBF1F2B0FBF8F108FB1202A4F88E00ECA0BBE2697AA4F84D10F1A013
S32508015DC02DE5697AA4F84F10F4A028E5697AA4F85110F8A023E5687A012809D084F892A011
S32508015DE094F89200012806D0AFF61011F7A016E584F89260F4E7AFF60811F7E71121F948C7
S32508015E00F2F7FCF9F74855F8091F953840F8951F69684160298901810EE0CEE3D3E3D8E372
S32508015E20DCE3E0E3E4E3E8E3ECE3F0E3F0E3F0E3F0E3F0E3F0E3F0E3EBA00299EFE4E94881
S32508015E4055F8091F953840F89F1FA9888180A9798171EBA00299E2E4687A012809D084F869
S32508015E6074A100BF94F87401012805D0ECA1EEA0D5E484F87461F5E7F0A1F8E7B5F8091009
S32508015E80A1F13000FC2806D201EB81010BEA4100A4F8750102E0EDA0FBF780FFB4F875116D
S32508015EA04046B1FBF0F208FB1212B1FBF8F1F0A03EE2B5F80910A1F10B00592806D201EBAB
S32508015EC081010BEA4100A4F8770102E0EFA0FBF765FFB4F877114046B1FBF0F208FB1212B1
S32508015EE0B1FBF8F1F3A023E2697AA1F10B008B2802D2A4F87911ECE1E8E1B6E3B1E3BDE3D6
S32508015F00F2E1F6E1FAE116E230E238E240E253E266E279E293E2AFE2C2E2DBE2EAE2F9E2C1
S32508015F20FEE202E307E30BE30FE313E317E31BE31FE323E327E32BE32FE333E337E3000073
S32508015F40546F74616C4361706163697479203A25642E256441480A0D00000000426D734D57
S32508015F606178566F6C743A25642E2564760A0D00754261744D617854656D70506C7573356C
S32508015F8030203A2564200A0D00000000754261744D696E54656D70506C75733530203A25DA
S32508015FA064200A0D000000007563426174547970653AC7A6CBE1B5E7B3D8200A0D000000F5
S32508015FC07563426174547970653AC4F8C7E2B5E7B3D8200A0D0000007563426174547970F8
S32508015FE0653AC1D7CBE1CCFAEFAEB5E7B3D8200A0D0000007563426174547970653AC3CC94
S32508016000CBE1EFAEB5E7B3D8200A0D007563426174547970653AEEDCCBE1EFAEB5E7B3D8C5
S32508016020200A0D007563426174547970653AC8FDD4AAEFAEB5E7B3D8200A0D007563426196
S3250801604074547970653ABEDBBACFCEEFEFAEC0EBD7D3B5E7B3D8200A0D0000007563426137
S3250801606074547970653AEED1CBE1EFAEB5E7B3D8200A0D007563426174547970653AC6E4E6
S32508016080CBFBB5E7B3D8200A0D000000546F74616C566F6C746167653A256420200A0D00DD
S325080160A052657175697265566F6C74616765446966666572656E63652825642956200A0DD0
S325080160C000000000202825642956206F7665722072616E6765200A0D0000000053696D7583
S325080160E06C6174656443757272656E74426174566F6C74202564560A0D00000053696D7534
S325080161006C6174656443757272656E74426174566F6C74202564562D2D3130302D33353018
S32508016120560A0D00434C4F534500000025732044656275675F506167655F66756E6374690A
S325080161406F6E200A0D0000004F50454E00000000754261744D6178456E6572677920256425
S32508016160202E2564200A0D0053746F70566F6C74616765203A25642E2564205620200A0D23
S32508016180000000004F76657254656D703056616C75653A256420200A0D0000004F766572DB
S325080161A054656D703156616C75653A256420200A0D0000004F76657254656D703256616C6B
S325080161C075653A256420200A0D0000005369676E616C4C6F7373466C616720257320200A41
S325080161E00D000000BD1500205665686963686C65496E666F28302D39293A25730A0D00000D
S325080162005665686963686C65496E666F2056494E2831302D3137293A25730A0D000000007E
S325080162206561737900000000576F726B4D6F64656C20257320200A0D0000000070726F6643
S32508016240657373696F6E616C00000000444352657175697265566F6C742025643A4F7665BB
S32508016260722834382D333030292020200A0D0000444352657175697265566F6C743A2564DD
S325080162802E2564205620200A0D00000044435265717569726543757272656E742564413A20
S325080162A04F7665722831302D31303041292020200A0D00004443526571756972654375727D
S325080162C072656E74256441200A0D0000ECA0FBF765FDB4F879114046B1FBF0F208FB1212A4
S325080162E0B1FBF8F1EEA023E0697A84F87B11F2A013E5697A84F87C11F5A00EE5B5F80910BA
S32508016300A1F13000CA2806D201EB81010BEA4100A4F87D0102E0F3A0FBF740FDB4F87D1146
S325080163204046B1FBF0F208FB1212B1FBF8F1F6A0FBF734FDBBE0B5F80910A1F114005A283C
S3250801634006D201EB81010BEA4100A4F87F0102E0F4A0FBF723FDB4F87F114046B1FBF0F2BE
S3250801636008FB1212B1FBF8F1F7A0E1E7687A962801D284F8810194F88111FAA0CDE4687A37
S32508016380962801D284F8820194F88211FBA0C4E4687A01280AD084F890A100BF94F890018E
S325080163A0012806D0AFF6CC61F9A0B6E484F89061F4E7AFF6C461F7E7687A01280AD084F879
S325080163C087A100BF94F88701012806D0AFF6F461F5A0A2E484F88761F4E7AFF6EC61F7E790
S325080163E0687A01280AD084F888A100BF94F88801012806D0AFF61C71EFA08EE484F8886199
S32508016400F4E7AFF61471F7E7687A032804D884F88901012803D005E084F889A147E0EBA062
S32508016420FBF7BCFC94F88901022802D1ECA0FBF7B5FC94F88901032839D1EEA055E494F8C3
S325080164408901B5F80950012803D12946EEA0FBF7A5FC94F88901022803D12946F0A0FBF70B
S325080164609DFC94F88901032803D12946F2A0FBF795FCA4F88A511AE0687A01280AD084F809
S325080164808CA100BF94F88C01012806D0AFF6B471EFA042E484F88C61F4E7AFF6AC71F7E786
S325080164A0687A012808D002280AD003280DD089F800601BB0BDE8F08F84F89761EBA014E417
S325080164C0022084F89701EEA00FE4032084F89701F0A00AE4B5F80910A4F89811A1F1C902D9
S325080164E0824205D201EB81020BEA4200A4F85900EDA012E4B5F80910A1F1C902824205D216
S3250801650001EB81020BEA4200A4F85D00A4F89A11EDA00BE4B5F80910A4F89C11F2A005E480
S32508016520B5F80910A4F89E1103E0B5F80910A4F8A011F7A00EE4B5F80910A4F8A2113AE08D
S32508016540B5F80910A4F8A41135E0B5F80910A4F8A61130E0B5F80910A4F8A8112BE0B5F804
S325080165600910A4F8AA1126E0B5F80910A4F8AC1121E0B5F80910A4F8AE111CE0B5F8091093
S32508016580A4F8B01117E0B5F80910A4F8B21112E0B5F80910A4F8B4110DE0B5F80910A4F80B
S325080165A0B61108E0B5F80910A4F8B81103E0B5F80910A4F8BA11DEA007E4B5F80910A4F817
S325080165C0BC11E3A006E4B5F80910A4F8BE11FEF7DBBFB5F80910A4F8C011F8E7B5F80910DA
S325080165E0A4F8C211F3E7B5F80910A4F8C411EEE7B5F80910A4F8C611E9E7B5F80910A4F8CC
S32508016600C811E4E7B5F80910A4F8CA11DFE705E009E00DE011E015E019E01DE0B5F8091067
S32508016620A4F8CC11D3E7B5F80910A4F8CE11CEE7B5F80910A4F8D011C9E7B5F80910A4F8CD
S32508016640D211C4E7B5F80910A4F8D411BFE7B5F80910A4F8D611BAE7B5F80910A4F8D8117B
S32508016660B5E788F804A0A0F802A051468246418000F050FB0027DFF8F0B2A0E1C1E10000F3
S3250801668044434D6178506F7765722564203A4F76657228312D31356B2909200A0D000000F2
S325080166A044434D6178506F7765723A25642E2564206B77090A0D000044435F496E6475639C
S325080166C074616E636554656D70202564200A0D0044435F4947425454656D70202564200AB5
S325080166E00D00000044434D6178566F6C74202564563A4F7665722834382D32303056292065
S3250801670020200A0D0000000044432044434D6178566F6C743A25642E2564205620200A0DD3
S325080167200000000044432044434D617843757272656E7425643A4F7665722832302D31319B
S3250801674030292020200A0D0044432044434D617843757272656E743A25642E256420412028
S32508016760200A0D0043617061636974616E636554656D7031202564200A0D00004443426FA8
S325080167807854656D7032202564200A0D00000000446F75626C65426174746572794D6F6474
S325080167A0652025730A0D000056494E205472616E732025730A0D0000426C75655369676E99
S325080167C0616C4C6F737325730A0D00004368617267654D6F64652D2D6B77680A0D00000003
S325080167E04368617267654D6F64652D2D74696D650A0D00004368617267654D6F64652D2D72
S32508016800534F430A0D0000004368617267654D6F64652D6B7768282564290A0D0000000036
S325080168204368617267654D6F64652D74696D65282564290A0D0000004368617267654D6FA7
S3250801684064652D534F43282564290A0D000000006869676820766F6C74616765206D6F644B
S32508016860756C652025730A0D00000000536F6353696D756C61547970652D310A0D0000004D
S32508016880536F6353696D756C61547970652D320A0D000000536F6353696D756C6154797074
S325080168A0652D330A0D0000000A0D20536F6353696D756C614D6178566F6C74202025642072
S325080168C05620200A0D0000000A0D20536F6353696D756C614D696E566F6C74202025642083
S325080168E05620200A0D0000000A0D20536F6343616C6962726174696F6E566F6C742020250E
S32508016900642028302E31295620200A0D000000000A0D20536F6343616C6962726174696F01
S325080169206E566F6C7420202564205620200A0D00536F6343616C6962726174696F6E566F4D
S325080169406C7420202564205620200A0D00000000536F6343616C6962726174696F6E2020E5
S32508016960256420200A0D0000E8010020E819002690F809901BF8362049464A4519D10BEB70
S32508016980C60828A098F80120FBF708FABAF8023004F10900534498F801201844D8F8041043
S325080169A0F1F713FCBAF8021098F801000844AAF80200761CF6B2612EDCD37F1CFFB2A742DF
S325080169C0D4D3BAF80220A11C1144AAF8021041F20501AAF80510E9798AF8071050468AF864
S325080169E00840002105E06A184318527A491C5A72C9B2A142F7D317AA07A91348F4F7B2FBD4
S32508016A0057E5E8790128FBD184F8B9A078210F48F1F7F4FBF8F7ACFA0DA000E012A0FBF773
S32508016A20BDF946E57265616420706172616D2061646472203078257820706172616D206CBC
S32508016A40656E2025640A0D002A1F0020E215002052656365697665207265636F726473201F
S32508016A6061636B0A0D0000005265636569766520444344432073746174652061636B0A0D29
S32508016A8000000000418819B1806808B1002070470120704741880088814201D30120704744
S32508016AA00020704710B50380002444808160828002FB0312C0E90321416110BD10B5044680
S32508016AC040880B4698B1A06888B1A28818466169F1F77BFBA088616901446161E26891423E
S32508016AE001D3A16861616188491E618010BD002010BD10B5044640882288904213D2A068BD
S32508016B0088B1A2882069F1F760FBA188206908442061E168884201D3A06820616088401C04
S32508016B206080012010BD002010BD000010B5F2F7EBF80F4C18B100206060012010BDF7F71A
S32508016B4053FD6060A1682731216088420ED309480078072808D0084800698047022803D03C
S32508016B600020E073022010BD0120FAE7002010BD302400206823002058000020016842680B
S32508016B8009BA12BAC0E9002170470168426809BA12BAC0E90021704730B5044687B001212B
S32508016BA00420F7F73BFC01214804F7F71FFC0420ADF8100003208DF812001820224D8DF847
S32508016BC0130004A92846F4F7E5FF0820ADF8100048208DF8130004A92846F4F7DBFF2620A6
S32508016BE08DF8140001218DF815108DF816108DF8171005A8F6F7C6FB0020ADF80400009412
S32508016C00ADF80600ADF80800ADF80C000C200F4CADF80A0069462046FAF7DCF9012240F2F6
S32508016C2025512046FAF7BDF9012240F224412046FAF7B7F901212046FAF783F98021204605
S32508016C40FAF776F907B030BD000801400044004070B5054686B001211120F7F7DFFB012171
S32508016C60C804F7F7C3FB4FF48060ADF8100003248DF812401820244E8DF8130004A9304652
S32508016C80F4F788FFF014ADF8100048208DF8130004A93046F4F77EFF34208DF814008DF8BD
S32508016CA015408DF8164001208DF8170005A8F6F769FB0020ADF80400ADF80600ADF80800B9
S32508016CC0ADF80C000C20114CADF80A00009569462046FAF77FF901212046FAF732F90122E2
S32508016CE040F225512046FAF75CF9012240F226612046FAF756F9012240F224412046FAF79E
S32508016D0050F906B070BD000000100140004C0040FDF788BF254810B5B0F859100A22B1FB05
S32508016D20F2F323490B80B0F85B30B3FBF2F34B80B0F88330B3FBF2F30B82B0F85330B3FB83
S32508016D40F2F30B83B0F88E30B3FBF2F38B82B0F88530B3FBF2F34B8290F88B30B3FBF2F318
S32508016D608B7690F88C30B3FBF2F3CB76B0F89030B3FBF2F3CB82B0F8B130B3FBF2F4B0F8DE
S32508016D80B340B4FBF2F4B3FBF2F2CC838A8390F8B620323A81F8212090F8B520323A81F8A8
S32508016DA0202090F8790181F8220010BD28150020C420002070B5174E002500BF05EB450016
S32508016DC000EBC50006EB001494F8540003281BD394F89100012803D122780421FCF788FDA5
S32508016DE094F8910002280FD194F8AC00401CC0B284F8AC00022807D3032084F89100227861
S32508016E0004210120FCF774FD6D1CEDB2022DD5D370BD000044130020D8FF0000F8339F4332
S32508016E20D9FF000058699543DAFF0000BA298C43DBFF0000C77B8343DCFF000071BD7643A3
S32508016E40DDFF0000A09A6743DEFF000000805943DFFF0000E75B4C43E0FF0000E71B404357
S32508016E60E1FF00001BAF3443E2FF00005A042A43E3FF00008B0C2043E4FF00001DBA164347
S32508016E80E5FF000042000E43E6FF0000B6D30543E7FF00007B54FC42E8FF0000C3F5ED42F5
S32508016EA0E9FF00005879E042EAFF000068D1D342EBFF0000E6EEC742ECFF0000AFC5BC428D
S32508016EC0EDFF0000C749B242EEFF00002E70A842EFFF0000B22E9F42F0FF0000C07B96428D
S32508016EE0F1FF00008A4E8E42F2FF0000AB9E8642F3FF00009AC87E42F4FF000007307142F8
S32508016F00F5FF0000FE656442F6FF0000645D5842F7FF0000230A4D42F8FF0000C5604242C3
S32508016F20F9FF00006D563842FAFF000048E12E42FBFF0000B5F72542FCFF000000911D4283
S32508016F40FDFF0000DDA41542FEFF00009F2B0E42FFFF0000011E0742000000005A750042C0
S32508016F6001000000A156F441020000005474E841030000005238DD4104000000FC98D2418C
S32508016F80050000004A8CC84106000000D509BF4107000000CE08B64108000000D881AD41F7
S32508016FA009000000916DA5410A00000039C59D410B000000758296410C0000008A9F8F4111
S32508016FC00D000000F01689410E00000088E382410F00000069007A4110000000B7D16E410F
S32508016FE0110000006132644112000000CE195A41130000006F815041140000007C61474198
S325080170001500000039B43E41160000001973364117000000F6972E41180000004F1E2741C7
S3250801702019000000000020411A000000DA3819411B00000028C412411C000000939D0C414E
S325080170401D00000020C106411E000000022B01411F00000025AFF74020000000D786ED407B
S3250801706021000000A1D6E340220000009E98DA4023000000E7C6D14024000000145CC94056
S32508017080250000001153C14026000000DFA6B94027000000FC52B240280000001153AB40D5
S325080170A029000000DBA2A4402A000000963E9E402B0000007D2298402C0000000A4B924066
S325080170C02D000000E1B48C402E000000E65C87402F00000010408240300000002CB77A40CE
S325080170E0310000006059714032000000D06168403300000092CB5F4034000000109257403F
S3250801710035000000DEB04F4036000000E2234840370000002EE740403800000027F73940B0
S3250801712039000000DF4F33403A00000063EE2C403B0000006CCF26403C000000B3EF204055
S325080171403D000000984C1B403E00000054E315403F0000001CB1104040000000D0B30B4070
S3250801716041000000A7E8064042000000D34D024043000000BEC1FB3F44000000FB3FF33F9A
S32508017180450000001B12EB3F460000002B35E33F47000000E8A4DB3F480000005F5ED43F77
S325080171A0490000004A5ECD3F4A000000B6A1C63F4B0000000326C03F4C0000003EE8B93F40
S325080171C04D00000075E5B33F4E000000041CAE3F4F000000A488A83F50000000062AA33FE8
S325080171E05100000037FD9D3F520000009300993F530000002332943F54000000EF8F8F3F47
S325080172005500000001188B3F5600000008C9863F5700000062A1823F580000002D3E7D3FA1
S3250801722059000000AE81753F5A0000004E0B6E3F5B0000001FD7663F5C0000002AE35F3FA6
S325080172405D000000CF2C593F5E00000018B2523F5F00000065704C3F600000001765463F56
S3250801726061000000DE8E403F620000001CEB3A3F63000000D977353F640000006E34303F35
S3250801728065000000931D2B3F66000000A032263F670000009F71213F6800000040D91C3F10
S325080172A0690000008C67183F6A000000331B143F6B000000E5F20F3F6C00000052ED0B3F7C
S325080172C06D0000002D09083F6E000000CC45043F6F00000038A1003F700000009335FA3EFC
S325080172E0710000006362F33E720000008FC7EC3E730000007862E63E740000007F30E03E74
S3250801730075000000A531DA3E76000000FA61D43E770000007FC1CE3E78000000944DC93EF5
S32508017320790000003A06C43E7A00000082E7BE3E7B0000006BF1B93E7C0000005721B53EEF
S325080173407D0000009678B03E00008A02020002007602B60302000500840340060200050009
S325080173600E063A07020005001C076009020005000000000069380108AD3801083D370108FA
S32508017380000000000000000000000000000000000100000069380108AD3801083D370108C8
S325080173A00000000000000000000000000000000030003000300030003000C600413430550E
S325080173C03238000000000000010000002C7A0108413C010801000000C87901085F3D01080E
S325080173E001000000C07901085D3D010801000000207A0108613D010801000000187A0108B1
S32508017400BD3D0108010000000C7A0108BB3D010801000000D0790108B93D01080100000076
S32508017420307A0108F53C010801000000B8790108C13D010801000000407A0108F93C01080C
S3250801744001000000387A0108ED3B010801000000A8790108653D010801000000547A010882
S32508017460453C010801000000487A0108993C010801000000607A0108893B01080100000017
S32508017480F4790108B1D0000801000000DC79010889D0000801000000007A010859D4000865
S325080174A001000000E8790108A1A8000800C1814001C0804101C0804100C1814001C0804177
S325080174C000C1814000C1814001C0804101C0804100C1814000C1814001C0804100C181408D
S325080174E001C0804101C0804100C1814001C0804100C1814000C1814001C0804100C181406D
S3250801750001C0804101C0804100C1814000C1814001C0804101C0804100C1814001C080414C
S3250801752000C1814000C1814001C0804101C0804100C1814000C1814001C0804100C181402C
S3250801754001C0804101C0804100C1814000C1814001C0804101C0804100C1814001C080410C
S3250801756000C1814000C1814001C0804100C1814001C0804101C0804100C1814001C08041EC
S3250801758000C1814000C1814001C0804101C0804100C1814000C1814001C0804100C18140CC
S325080175A001C0804101C0804100C1814000C0C101C30302C2C60607C705C5C404CC0C0DCD4C
S325080175C00FCFCE0E0ACACB0BC90908C8D81819D91BDBDA1A1EDEDF1FDD1D1CDC14D4D5150C
S325080175E0D71716D6D21213D311D1D010F03031F133F3F23236F6F737F53534F43CFCFD3D6C
S32508017600FF3F3EFEFA3A3BFB39F9F83828E8E929EB2B2AEAEE2E2FEF2DEDEC2CE42425E54B
S3250801762027E7E62622E2E323E12120E0A06061A163A3A26266A6A767A56564A46CACAD6DAB
S32508017640AF6F6EAEAA6A6BAB69A9A86878B8B979BB7B7ABABE7E7FBF7DBDBC7CB47475B58B
S3250801766077B7B67672B2B373B17170B0509091519353529296565797559594549C5C5D9DEB
S325080176805F9F9E5E5A9A9B5B99595898884849894B8B8A4A4E8E8F4F8D4D4C8C44848545CB
S325080176A087474686824243834181804000000000807E010801000000E47D010802000000A1
S325080176C0B47D010803000000607D010804000000747D010805000000647F01080600000083
S325080176E01C7C010807000000087F010808000000187F0108090000004C7D01080A000000B6
S32508017700407C01080B000000947C01080C000000E87C01080D000000887D01080E000000CF
S32508017720947D01080F000000307D010810000000FC7E010811000000207E010812000000FE
S32508017740587E010813000000487E010814000000D07E010815000000C07E0108160000007C
S32508017760E07E010817000000687E0108180000009C7E010819000000347E01081A00000064
S32508017780A47D01081B000000F07E01081C0000004C7F01081D000000607C01081E0000000E
S325080177A0747C01081F000000887C010820000000287F010821000000587F010822000000A2
S325080177C0507C010824000000F47C010825000000007D010826000000107D0108270000009A
S325080177E0287C0108280000003C7D0108290000003C7F01082A000000D47D01082B00000047
S32508017800C07C01082C000000A47C01082D000000DC7C01082E000000B07E01082F0000009D
S32508017820207D010830000000F47D010831000000087E010832000000C47D0108330000007A
S325080178408C7E01080007070209030C020E0200008711C1008793C20016179100171791001A
S325080178608873C0000C401F000D401F0000401F0001401F0002401F0003401F0004401F0082
S3250801788005401F0006401F0007401F0008401F0009401F000A401F0000008A0202000200E2
S325080178A07602B6030200050084034006020005000E063A07020005001C07600902000500BE
S325080178C000000E001A00260040004A0054006B0075008800CA00D400E000E400E800EC00CF
S325080178E0F000F400F8000C0A0A18080815081140080A020202020202020087F18AF197F14C
S3250801790089F189F093F195F180F190F110F08CF184F100A001A0802F812F822F832F842FC1
S3250801792090F110F08CF184F100A001A0812F822F832F0000130055005F006B006F0073005D
S3250801794077007B001100400008000A000200020002000200020010111419222E273E31285D
S32508017960857F00000D0A3737375570642D2D747970653A253078202C7665723A2530782C20
S3250801798054627974653A2530782C204372633A2530782C5061673A2530782C506C656E3A1E
S325080179A02530780D0A0000005265616C7948696768343030000000004B43353600000000CA
S325080179C04F464644434443004F4E44434443000053455441504E50574400000041435F72F9
S325080179E045634C4F53450000414352656C61794F4646000041435F72454F50454E00000075
S32508017A00414352656C61794F4E00000053455441504E55534552000054455354424D53000D
S32508017A20524541444D41535300000000534554005265736574000000414363757400000028
S32508017A40444363757400000043433243435265616C79000043433143505265616C790000C2
S32508017A6047554E54656D705265616C790000000052657365727665643100000048414E44EE
S32508017A800000000049444C450000000052554E4E494E470053544F5000000000494E49541E
S32508017AA00000000053544152540000006368617267655F4D6F64655F3132560052454144A7
S32508017AC0590000005265736572766564000000005265736572766174696F6E5F41435F63C7
S32508017AE068617267655F6D6F6465000044435F6368617267655F6D6F6465000041435F64D1
S32508017B0069736368617267655F6D6F646500000044435F6469736368617267655F6D6F64DD
S32508017B20650000004E6F726D616C5F6D6F64650052656D6F74655F636F6E74726F6C5F6DCC
S32508017B406F6465006368617267655F626174746572795F686561745F6D6F64650000000015
S32508017B6052656D6F74655F626174746572795F686561745F6D6F64650000000044656661BB
S32508017B80756C745F6D6F64650000000041435F4368617267696E670044435F4368617267AC
S32508017BA0696E670041435F4368617267000000004E6F726D616C5F4F7065726174696F6E37
S32508017BC00000000041435F6368617267655F636F6E6E65637400000041435F646973636812
S32508017BE0617267655F636F6E6E6563740000000048616C665F636F6E6E65637400000000CA
S32508017C004E6F5F636F6E6E6563740000436F6E6E6563745F4661756C74000000534F432025
S32508017C203130302500000000B3E4B5E7D7AED6D0D6B9B1A8CEC428C6FAD3C3290000000000
S32508017C40B3E4B5E7D0E8C7F3B5E7D1B9CEAA3000564355B9A4D7F7C4A3CABDD2ECB3A30087
S32508017C60424D53C8C8B9DCC0EDBCD3C8C8D2ECB3A3000000424D53C8C8B9DCC0EDD6C6C0FE
S32508017C80E4D2ECB3A3000000424D53BEF9BAE2CAA7D0A700B5E7B3D8B8DFCEC2D4A4BEAF8D
S32508017CA000000000B3B5D4D8B4A2C4DCD7B0D6C3C0E0D0CDC7B7D1B9B1A8BEAF0000000080
S32508017CC0B3B5D4D8B4A2C4DCD7B0D6C3C0E0D0CDB9FDD1B9B1A8BEAF00000000534F43B58E
S32508017CE0CDB1A8BEAF000000534F43B9FDB8DFB1A8BEAF00424D53CDA8D1B6B3ACCAB10032
S32508017D00B3E4B5E7D7AECDA8D1B6B3ACCAB10000B3B5C1BECEB4C9CFB8DFD1B900000000A4
S32508017D20B3E4B5E7D7AED6D0D6B9B1A8CEC40000424D53C4DAB2BFCDA8D0C500434D4C2065
S32508017D40B2CECAFDB2BBBACFCACA0000B3E4B5E7B5E7C1F7D0E8C7F3B9FDB5CD0000000012
S32508017D60D6B1C1F7BCCCB5E7C6F7D5B3C1ACB9CAD5CF0000BDBBC1F7BCCCB5E7C6F7D5B31F
S32508017D80C1ACB9CAD5CF0000424D53C5F6D7B2B9CAD5CF00424D53C4DAB2BFBEF8D4B5B90A
S32508017DA0CAD5CF00424D53CDE2B2BFBEF8D4B5B9CAD5CF00CAE4C8EBC7B7D1B9B9CAD5CF4E
S32508017DC0000000004B4C3330B8DFD1B9D1B9B9CAD5CF00004B4C3330B5CDD1B9B9CAD5CF9B
S32508017DE000000000CAE4C8EBB9FDD1B9B9CAD5CF00000000B0E5D4D8CEC2B6C8B9FDB8DF10
S32508017E00B9CAD5CF00000000D6B1C1F7C7B9D7F9CEC2B6C8B9FDB8DFB9CAD5CF000000001B
S32508017E20424D53D7DCB5E7D1B9BCECB2E2B9CAD5CF000000B5A5CCE5B5E7D1B9BCECB2E2A8
S32508017E40B9CAD5CF00000000424D53CEC2B6C8BCECB2E2B9CAD5CF00424D53B5E7C1F7BCA7
S32508017E60ECB2E2B9CAD5CF00B3B5D4D8B4A2C4DCD7B0D6C3B9FDB3E4B9CAD5CF00000000AE
S32508017E80CEB4B6A8D2E5B9CAD5CF0000B3ACB3F6B6A8D2E5B9CAD5CF00000000BDBBC1F7A1
S32508017EA0B3E4B5E7BFDACBF8BDF4B9CAD5CF0000B3E4B5E7B9FDC1F7B9CAD5CF0000000084
S32508017EC0B8BABCABBDD3B4A5C6F7B9CAD5CF0000D5FDBCABBDD3B4A5C6F7B9CAD5CF0000E7
S32508017EE0D4A4B3E4BDD3B4A5C6F7B9CAD5CF0000B5E7B3D8C8C8CAA7BFD80000424D53D422
S32508017F00A4B3E4CAA7B0DC00B5A5CCE5B5E7D1B9B9FDB8DF00000000B5E7D0BECEC2B6C864
S32508017F20B9FDB8DF00000000B5A5CCE5B5E7B3D8C7B7D1B9BEAFB8E60000000043435320A7
S32508017F40BDFBD6B9B3E4B5E700000000424D53BDFBD6B9B3E4B5E700564355BDFBD6B9B354
S32508017F60E4B5E700CAE4C8EBB9FDC1F7000000004B433100595831004B433200595832005F
S32508017F8048565F4453475F434845434A5F3200004B4333004B4335004B4338004B43390099
S32508017FA043414E315F5354420000000043414E325F53544200000000454C535F4F464600FD
S32508017FC048565F4453475F434845434A0000000043414E325F454E00454C535F4F4E000025
S32508017FE04D43555F52554E005057335F335600005057355600000000434F4E475F52580015
S32508018000434F4E475F54580028800108000000201C0C0000708A0008E48501081C0C00206A
S325080180206C7B0000A01E01088133E80384A24A04400901020304060708090237A613B9C490
S3250801804014084DC31B0859041AD50C13A9A41C08EDEF041ABC1412D2021D08023E01180AAE
S32508018060494801083F4701088D041A91041AC904411A14E8B26429F89AF46C00091CD5FB24
S32508018080B3B5D0ADD2E963030A1EBD360108F104092A3401484BFFFFBC01281A02E413F0D1
S325080180A0045B2001085A03082305101348151B2004081A38082306021A75081A07081A91E5
S325080180C0081A08281A93081A09201A28081A0A101AAF081A0F081AB4081A0E081AB3081AD2
S325080180E00D081AB2081A0C081AB1085A0B601A13481A83101A12081A81081A11081AAD08C7
S325080181001A10081AAB081A140829281A16081A8B101A18381AD8081A1F0813DA201B201ED2
S32508018120081ADC081A1D081AB5181A20081AE2101A21081AE0081A22081ADF185A24601A24
S3250801814023081A87085A27481A26081AE5281A25081AE4081A28201A85181A29101ABB086E
S325080181601A2A101ACE081A2B101AD0085A30881A31081AD8301A32181A75101A33081A77F5
S32508018180081A34081A79081A35081ABA0823360A1ABD082337071AC7081A5018139C161BB6
S325080181A02051401A9D081A52081A9F081A53181AA1081A54081AA3081A55081AA4081A56DB
S325080181C0201AA5081A57081AA7081A58181AA9081A59081AAA081A5A081AB8081A60081AD9
S325080181E0AF081A61081AB0081A62081AB1081A63381AB2081A65101AB4081A66081AB508C0
S325080182001A6D081ABF081A6E201AC0081A6F081AC2081A70081AC4081A71081AC6081A7261
S32508018220081AC8081A73081ACA081A74081ACC081A75081ACE081A76081AD0081A77081A74
S32508018240D2081A78081AD4081A79081AD6081A7A081AD8081A7B081ADA081A7C081ADC0847
S325080182601A7D081ADE081A7E081AE0081A7F081AE2081A80081AE4081A81081AE6081A821A
S32508018280081AE8081A83081AEA081A84081AEC081A85081AEE081A86081AF0081A87081A24
S325080182A0F2081A88081AF4081A89081AF6081A8A081AF8081A8B081AFA081A8C081AFC08D7
S325080182C01A8D081AFE081A8E081112171B208F081A02088145020406082D010203040420AB
S325080182E00B06070809312A01080401132DD51B0809081A750823310313F9DA1B0857081A24
S32508018300AD101A58081AF1081A59081331D61B085D081A69081A5F081A8908239B051AA9AA
S32508018320081AE6101AC9082AE72812D71B0880181A59081A11581325DB6408270463340708
S325080183405ADF088117B1440108D9A5140879A639A8811AB7181AF514DA45181A27184B0D28
S32508018360A7189A611C1ABD181A2118DAA51C1AF5181A41141A09105A1D1829201AED181A61
S3250801838055181A91049A31481EED450108691401101A2130DAB58C411AB5181ABB041A2DEA
S325080183A0041AC1041AF9042AF10419481A25081B45411819041FB54001080542041D43014E
S325080183C00899081AED081A5914C11331EC14083DC31B08590813C5C41B080D0813E9BF1B14
S325080183E00819081AED081A01081AE508017013980682201EB07B01088C041A98041E847A94
S3250801840001089C041A7C041ABC041AA4041A8C042A940C1920111D7C0108F0081AC4041A1A
S32508018420D8041A0C102A7030190C1A24041ADC0C1AFC041AEC041A10101AD0081AAC041AB4
S32508018440300C1A44042A603C1910722813A7BC7308328BADCB0C1A8D0C720A1351B07308F6
S325080184600513C78A6B0814248AC70C9A890C8B25AA0C1305D50218081301D21408BFD11B2B
S3250801848008E90439253C0C014018990C9A020C118A800C39055A0818290669249A04182912
S325080184A03D690C293C3C100140502912690C2905593C5A106C398029051924390C292419A1
S325080184C00C49B589549A209C29776954494D490C39185A143C29616948011713C1CF1408FB
S325080184E040081B204C041354091620707F0108120A1B2078081A0C081A90081A18081A945D
S32508018500081A24081A98081A30081A9C081A3C081AF0081A48081AE0081A54081A74081A32
S3250801852060081A7C081A6C081AE8081A78081AAC081A84081AD0081A90081AD8081A9C0824
S325080185401AB8081AA8081AA0081AB4081AC0081AC0081A80081ACC081AF8081AD808114E09
S3250801856080010815D1AC1A5804690C9A640C9A700C9A7C0C9A880C1A94045A750C1AA0042B
S325080185804B29D20C9AAC0C9AB8309AC40C9AD00C9ADC0C9AE80C9AF40C1112094C20D9D0DB
S325080185A00C9A0C0C1A180C69249A240C1A300C01340316F40102631F022F021E0D010108D4
S325080185C03D041A61041A95041AB5041E55020108D5081ABD081A89041A21041AE1040528FA
S309080185E0B50B0108BF
S9030000FC
